:020000040000FA
:10000000000002204510020039100000DD1002003F
:100010003D100000D90A000045100000000000005B
:100020000000000000000000000000005D10000063
:1000300049100000000000004D100000311C0200BB
:10004000551000005510000055100000551000001C
:10005000551000005510000055100000551000000C
:1000600055100000551000005510000055100000FC
:1000700055100000551000005510000055100000EC
:10037000DFF80CD021F00AF900480047312B0200C9
:100380000000022081B08DF8030001B0704700BF6B
:1003900081B08DF803008DF8021001B0704700BFE6
:1003A00081B0ADF8020040F2C011C2F2000101209C
:1003B000087001B0704700BF80B582B00190009115
:1003C0000198009900F006F80198009900F046F8AD
:1003D00002B080BD82B0019000910198006840F2A7
:1003E000DF71884230D0FFE70198006840F2237146
:1003F000884229D0FFE70198006840F224718842C2
:1004000022D0FFE701980068B0F58A6F1CD0FFE7A3
:100410000198006840F25341884215D0FFE70198E7
:10042000006840F2544188420ED0FFE7019800680E
:1004300040F28731884207D0FFE70198006840F218
:10044000EF31884207D1FFE740F2BA11C2F2000152
:1004500001200870FFE702B0704700BF82B0019032
:1004600000910198006841F21431C8F200018842FD
:1004700046D1FFE701980079012841D1FFE70198B3
:100480004079E8BBFFE700988068082837D1FFE78C
:10049000009800680078012831D1FFE700980068D3
:1004A000407802282BD1FFE7009800688078032865
:1004B00025D1FFE700980068C07804281FD1FFE726
:1004C000009800680079052819D1FFE700980068B6
:1004D0004079062813D1FFE7009800688079072843
:1004E0000DD1FFE700980068C079082807D1FFE721
:1004F00040F2BB11C2F2000101200870FFE7FFE7E4
:1005000002B0704740F2BC11C2F20001086801302D
:10051000086000EE100AB8EE400AB7EE001AB4EE1A
:10052000410AF1EE10FA0DD1FFE740F2BC11C2F220
:1005300000010020086040F2B911C2F20001012060
:100540000870FFE7704700BF80B588B006900120B3
:100550008DF81700069800880146039120B1FFE747
:100560000398B72826D068E040F2C412C2F2000215
:1005700040F23370506040F20000C2F20000906020
:100580000020019010800821917001210FF0DEF809
:1005900001980FF059FA0220029017F09DFE029880
:1005A00040F6B83117F0F2FDFFE7FFE70699B720F4
:1005B0000880FFE740F2B910C2F20000007801287D
:1005C00004D0FFE700208DF81F003FE0FFE740F276
:1005D000C110C2F200000178013101700078FF28DB
:1005E00001D1FFE728E040F2C110C2F2000000781C
:1005F00040F20001C2F20001087040F2C411C2F2E0
:10060000000104200FF054FC002004900490FFE748
:10061000049842F20F71884205D8FFE7FFE704987B
:1006200001300490F4E70FF085FE40F2B911C2F2F8
:10063000000100200870B8E7FFE700208DF81700E0
:100640000699088003208DF81F00FFE79DF91F0021
:1006500008B080BD80B586B0049001208DF80F00F1
:10066000049800880146029120B1FFE70298E02833
:100670000ED01CE00020019001210FF067F80198D6
:100680000FF0E2F9FFE7FFE70499E0200880FFE7B9
:1006900040F2BA10C2F200000078012804D0FFE74F
:1006A00000208DF817000BE0FFE7FFE7FFE70020D1
:1006B0008DF80F000499088003208DF81700FFE7DC
:1006C0009DF9170006B080BD80B50FF017FF40F20E
:1006D000BB10C2F20000007880BD00BF80B586B0BC
:1006E000049001208DF80F000498008801460291C3
:1006F00020B1FFE70298FE2813D02DE000200190E2
:1007000001210FF023F801980FF09EF9022040F626
:10071000B83117F03BFDFFE7FFE70499FE200880A2
:10072000FFE7FFF7D1FF012804D0FFE700208DF895
:1007300017001AE0FFE740F2BB10C2F20000007899
:10074000012807D1FFE740F2BB11C2F200010020EF
:10075000087000E0E0E7FFE700208DF80F00049943
:10076000088003208DF81700FFE79DF9170006B0F9
:1007700080BD00BF80B586B0049001208DF80F00C9
:10078000049800880146029130B1FFE7029840F2D8
:100790001311884212D020E00020019001210EF0B8
:1007A000D5FF01980FF0ACF8019810F003FCFFE7BB
:1007B000FFE7049940F213100880FFE740F2B810F9
:1007C000C2F200000078012804D0FFE700208DF875
:1007D00017000BE0FFE7FFE7FFE700208DF80F00B1
:1007E0000499088003208DF81700FFE79DF9170092
:1007F00006B080BD80B586B0049040F2D012C2F23F
:10080000000241F22210C8F20000506040F20800DD
:10081000C2F20000906000200090108008219170CA
:10082000012101910EF092FF00980FF00DF90220C6
:1008300040F6B83117F0AAFC01988DF80F00049823
:1008400000880146029130B1FFE7029840F2391169
:10085000884207D034E0FFE7FFE7049940F23910FF
:100860000880FFE740F2B910C2F2000000780128CA
:1008700004D0FFE700208DF817002AE0FFE740F2E0
:10088000D011C2F2000105200FF012FB40F2B911A5
:10089000C2F200010020087040F2DC10C2F2000039
:1008A0000168013101600068642807D1FFE740F268
:1008B000DC11C2F200010020086000E0CCE7FFE795
:1008C00000208DF80F000499088003208DF8170090
:1008D000FFE79DF9170006B080BD00BF80B584B06A
:1008E000029001208DF807000298008801460091CF
:1008F000E0B1FFE70098B0F5AB7F3BD0FFE7009891
:1009000040F2571188424FD0FFE70098B0F5AC7F16
:1009100064D0FFE7009840F25911884278D0FFE791
:100920000098B0F5AD7F00F08D80A0E040F204218A
:10093000C2F200010020088040F20621C2F200014C
:10094000088040F20821C2F20001088040F20A212A
:10095000C2F20001088040F20C21C2F200010880BE
:10096000022017F03DFDFFE7FFE702994FF4AB705F
:100970000880FFE740F20420C2F20000FFF7E4FD28
:10098000012804DCFFE700208DF80F0078E0FFE786
:1009900040F20421C2F2000100200880FFE7029922
:1009A00040F257100880FFE740F20620C2F2000034
:1009B000FFF750FE012804DCFFE700208DF80F0050
:1009C0005EE0FFE740F20621C2F20001002008804D
:1009D000FFE702994FF4AC700880FFE740F208206F
:1009E000C2F20000FFF77AFE012804DCFFE70020D6
:1009F0008DF80F0044E0FFE740F20821C2F2000149
:100A000000200880FFE7029940F259100880FFE7B4
:100A100040F20A20C2F20000FFF7ACFE012804DC1D
:100A2000FFE700208DF80F002AE0FFE740F20A21DF
:100A3000C2F2000100200880FFE702994FF4AD7078
:100A40000880FFE740F20C20C2F20000FFF7D2FE60
:100A5000012804DCFFE700208DF80F0010E0FFE71D
:100A600040F20C21C2F20001002008807CE7002047
:100A70008DF807000299088003208DF80F00FFE72A
:100A80009DF90F0004B080BD704700BF704700BFE4
:100A900084B08DF80F0002918DF80720009301209B
:100AA00004B0704782B08DF80700ADF80410ADF8BF
:100AB000022002B0704700BF81B08DF803008DF8AE
:100AC000021001B0704700BF704700BF704700BF01
:100AD000704700BF704700BF80B5002010F0BAFA21
:100AE00038B9FFE740F2B811C2F2000101200870E6
:100AF000FFE780BD80B500F043FE80BD80B500F00B
:100B000051FE80BD80B500F03BFE80BD80B500F099
:100B100049FE80BD80B500F033FE80BD80B500F099
:100B200041FE80BD80B500F02BFE80BD80B500F099
:100B300039FE80BD80B500F023FE80BD80B500F099
:100B400031FE80BD80B500F01BFE80BD80B500F099
:100B500029FE80BD80B500F013FE80BD80B500F099
:100B600021FE80BD80B500F00BFE80BD80B500F099
:100B700019FE80BD80B500F003FE80BD80B500F099
:100B800011FE80BD80B500F0FBFD80BD80B500F09A
:100B900009FE80BD80B500F0F3FD80BD80B500F09A
:100BA00001FE80BD80B500F0EBFD80BD80B500F09A
:100BB000F9FD80BD80B500F0E3FD80BD80B500F09B
:100BC000F1FD80BD80B500F0DBFD80BD80B500F09B
:100BD000E9FD80BD80B500F0D3FD80BD80B500F09B
:100BE000E1FD80BD80B500F0CBFD80BD80B500F09B
:100BF000D9FD80BD80B500F0C3FD80BD80B500F09B
:100C0000D1FD80BD80B500F0BBFD80BD80B500F09A
:100C1000C9FD80BD80B500F0B3FD80BD80B500F09A
:100C2000C1FD80BD80B500F0ABFD80BD80B500F09A
:100C3000B9FD80BD80B500F0A3FD80BD80B500F09A
:100C4000B1FD80BD80B500F09BFD80BD80B500F09A
:100C5000A9FD80BD80B500F093FD80BD80B500F09A
:100C6000A1FD80BD80B500F08BFD80BD80B500F09A
:100C700099FD80BD80B500F083FD80BD80B500F09A
:100C800091FD80BD80B500F07BFD80BD80B500F09A
:100C900089FD80BD80B500F073FD80BD80B500F09A
:100CA00081FD80BD80B500F06BFD80BD80B500F09A
:100CB00079FD80BD80B500F063FD80BD80B500F09A
:100CC00071FD80BD80B500F05BFD80BD80B500F09A
:100CD00069FD80BD80B500F053FD80BD80B500F09A
:100CE00061FD80BD80B500F04BFD80BD80B500F09A
:100CF00059FD80BD80B500F043FD80BD80B500F09A
:100D000051FD80BD80B500F03BFD80BD80B500F099
:100D100049FD80BD80B500F033FD80BD80B500F099
:100D200041FD80BD80B500F02BFD80BD80B500F099
:100D300039FD80BD80B500F023FD80BD80B500F099
:100D400031FD80BD80B500F01BFD80BD80B500F099
:100D500029FD80BD80B500F013FD80BD80B500F099
:100D600021FD80BD80B500F00BFD80BD80B500F099
:100D700019FD80BD80B500F003FD80BD80B500F099
:100D800011FD80BD80B500F0FBFC80BD80B500F09A
:100D900009FD80BD80B500F0F3FC80BD80B500F09A
:100DA00001FD80BD80B500F0EBFC80BD80B500F09A
:100DB000F9FC80BD80B500F0E3FC80BD80B500F09B
:100DC000F1FC80BD80B500F0DBFC80BD80B500F09B
:100DD000E9FC80BD80B500F0D3FC80BD80B500F09B
:100DE000E1FC80BD80B500F0CBFC80BD80B500F09B
:100DF000D9FC80BD80B500F0C3FC80BD80B500F09B
:100E0000D1FC80BD80B500F0BBFC80BD80B500F09A
:100E1000C9FC80BD80B500F0B3FC80BD80B500F09A
:100E2000C1FC80BD80B500F0ABFC80BD80B500F09A
:100E3000B9FC80BD80B500F0A3FC80BD80B500F09A
:100E4000B1FC80BD80B500F09BFC80BD80B500F09A
:100E5000A9FC80BD80B500F093FC80BD80B500F09A
:100E6000A1FC80BD80B500F08BFC80BD80B500F09A
:100E700099FC80BD80B500F083FC80BD80B500F09A
:100E800091FC80BD80B500F07BFC80BD80B500F09A
:100E900089FC80BD80B500F073FC80BD80B500F09A
:100EA00081FC80BD80B500F06BFC80BD80B500F09A
:100EB00079FC80BD80B500F063FC80BD80B500F09A
:100EC00071FC80BD80B500F05BFC80BD80B500F09A
:100ED00069FC80BD80B500F053FC80BD80B500F09A
:100EE00061FC80BD80B500F04BFC80BD80B500F09A
:100EF00059FC80BD80B500F043FC80BD80B500F09A
:100F000051FC80BD80B500F03BFC80BD80B500F099
:100F100049FC80BD80B500F033FC80BD80B500F099
:100F200041FC80BD80B500F02BFC80BD80B500F099
:100F300039FC80BD80B500F023FC80BD80B500F099
:100F400031FC80BD80B500F01BFC80BD80B500F099
:100F500029FC80BD80B500F013FC80BD80B500F099
:100F600021FC80BD80B500F00BFC80BD80B500F099
:100F700019FC80BD80B500F003FC80BD80B500F099
:100F800011FC80BD80B500F0FBFB80BD80B500F09A
:100F900009FC80BD80B500F0F3FB80BD80B500F09A
:100FA00001FC80BD80B500F0EBFB80BD80B500F09A
:100FB000F9FB80BD80B500F0E3FB80BD80B500F09B
:100FC000F1FB80BD80B500F0DBFB80BD80B500F09B
:100FD000E9FB80BD80B500F0D3FB80BD80B500F09B
:100FE000E1FB80BD80B500F0CBFB80BD80B500F09B
:100FF000D9FB80BD80B500F0C3FB80BD80B500F09B
:10100000D1FB80BD80B500F0BBFB80BD80B500F09A
:10101000C9FB80BD80B500F0B3FB80BD80B500F09A
:10102000C1FB80BD80B500F0ABFB80BD80B500F09A
:10103000B9FB80BDFFE7FEE7FFE7FEE7FFE7FEE75E
:10104000FFE7FEE7FFE7FEE7FFE7FEE7FFE7FEE774
:10105000FFE7FEE700BFFFE700BFFDE7FFE7FEE7B2
:10106000BFF34F8F4EF60C51CEF20001086800F42A
:10107000E0600422C0F2FA5210430860BFF34F8FC1
:10108000FFE700BFFDE7000080B582B00190FFE7F9
:10109000019840B9FFE745F26860C0F20200742190
:1010A00000F042F83EE001980068CE2808D3FFE740
:1010B00045F26860C0F20200752100F035F831E0B9
:1010C00000200090FFE7009801990968884228D223
:1010D000FFE701984068009A00EBC20130F9320046
:1010E000C97800F027F801984068009900EBC1002A
:1010F0008078012808D1FFE701984068009930F90D
:10110000310000F065F807E001984068009930F977
:10111000310000F08DF8FFE7FFE700980130009004
:10112000D1E7FFE702B080BD82B001900091FFE7F8
:10113000FEE700BF80B582B0ADF806000091FFE782
:10114000BDF9060010F10D0F09DCFFE745F26860FC
:10115000C0F202004FF49D71FFF7E6FF36E0BDF9E3
:101160000600CD2809DBFFE745F26860C0F2020007
:1011700040F23B11FFF7D8FF28E00098102809D370
:10118000FFE745F26860C0F202004FF49E71FFF77E
:10119000CBFF1BE0BDF9060000280AD4FFE700984A
:1011A0000001BDF906104EF20042CEF20002885452
:1011B0000BE000980001BDF8061001F00F014EF69B
:1011C0001452CEF200028854FFE7FFE702B080BD60
:1011D00080B582B0ADF80600FFE7BDF90600B0F1BA
:1011E000FF3F08DCFFE745F26860C0F20200E12142
:1011F000FFF79AFF1AE0BDF90600CD2808DBFFE7EC
:1012000045F26860C0F20200E221FFF78DFF0DE0B9
:10121000BDF9061001F01F02012090404A094EF26C
:101220000011CEF2000141F82200FFE702B080BDBC
:1012300080B582B0ADF80600FFE7BDF90600B0F159
:10124000FF3F09DCFFE745F26860C0F202004FF49F
:101250008671FFF769FF1FE0BDF90600CD2809DBA5
:10126000FFE745F26860C0F2020040F20D11FFF79F
:101270005BFF11E0BDF9061001F01F020120904054
:101280004A094EF28011CEF2000141F82200BFF36C
:101290004F8FBFF36F8FFFE702B080BD80B584B082
:1012A000ADF80E00029101924EF60850CEF2000009
:1012B00000680090FFE7BDF90E0010F10F0F08DC89
:1012C000FFE745F26860C0F20200AA21FFF72CFF99
:1012D00035E0BDF90E00CD2808DBFFE745F2686078
:1012E000C0F20200AB21FFF71FFF28E04EF60850C6
:1012F000CEF20000006841F23401C0F20201096838
:10130000884208D2FFE745F26860C0F20200AE21D1
:10131000FFF70AFF13E0019848B1FFE70098BDF915
:101320000E1000EB8100006C01990860FFE7029845
:101330000099BDF90E2001EB82010864FFE704B0BB
:1013400080BD00BF80B582B0ADF8060000200090DF
:10135000FFE7BDF9060010F10D0F09DCFFE745F2CC
:101360006860C0F2020040F27311FFF7DDFE29E071
:10137000BDF90600CD2809DBFFE745F26860C0F241
:1013800002004FF4BA71FFF7CFFE1BE0BDF9060073
:1013900000280AD4FFE7BDF906004EF20041CEF264
:1013A0000001405C000900900BE0BDF8060000F071
:1013B0000F004EF61451CEF20001405C000900907F
:1013C000FFE7FFE7009802B080BD00BF80B582B0A4
:1013D000ADF80600FFE7BDF90600B0F1FF3F09DCFC
:1013E000FFE745F26860C0F202004FF4D571FFF7E5
:1013F0009BFE1BE0BDF90600CD2809DBFFE745F2A7
:101400006860C0F2020040F2AB11FFF78DFE0DE004
:10141000BDF9061001F01F02012090404A094EF26A
:101420008021CEF2000141F82200FFE702B080BD2A
:1014300080B584B00390002001908DF80B000398D4
:1014400038B1FFE7FF2000211022012320F06AF9C4
:101450004BE044F29C30C0F202000068002843D008
:10146000FFE744F29C30C0F20200006800900020C8
:101470000190FFE7019800990968884233D2FFE79D
:1014800000984068019A00EBC20130F932004968C7
:101490000022FFF703FF00984068019A00EBC201A9
:1014A00030F93200C978FFF745FE0098406801998D
:1014B00000EBC1008078012808D1FFE70098406860
:1014C000019930F93100FFF783FE07E0009840688A
:1014D000019930F93100FFF7ABFEFFE7FFE7019814
:1014E00001300190C6E7FFE7FFE704B080BD00BF11
:1014F00080B582B0ADF806008DF8051000208DF89B
:101500000400BDF90600CC2806DCFFE7BDF90600A3
:1015100010F10F0F0ADCFFE7FF2000211122022348
:1015200020F000F901208DF804000FE09DF805007F
:10153000012805D1FFE7BDF90600FFF749FE04E0E9
:10154000BDF90600FFF774FEFFE7FFE79DF8040012
:1015500002B080BD80B584B0ADF80E0002910020CD
:101560008DF80700BDF90E00CC280ADCFFE7BDF9B5
:101570000E0010F10E0F04DBFFE7029810280AD3CB
:10158000FFE7FF2000211222022320F0CBF80120E8
:101590008DF8070005E0BDF90E000299FFF7CAFDBE
:1015A000FFE79DF8070004B080BD00BF80B584B0A0
:1015B000ADF80E00029100208DF80700BDF90E0075
:1015C000CC2806DCFFE7BDF90E0010F10F0F0ADC96
:1015D000FFE7FF2000211322022320F0A3F80120BF
:1015E0008DF8070015E0029858B9FFE7FF200021A9
:1015F00013220123009320F095F800988DF807003E
:1016000006E0BDF90E00FFF79DFE02990860FFE7B6
:10161000FFE79DF8070004B080BD00BF80B584B02F
:10162000ADF80E000291019200208DF80300BDF983
:101630000E00CC2806DCFFE7BDF90E0010F10F0FFD
:101640000ADCFFE7FF2000211422022320F06AF8C1
:1016500001208DF8030006E0BDF90E000299019A01
:10166000FFF71CFEFFE79DF8030004B080BD0000FB
:1016700080B500F0B1F840F68821C2F200010020E8
:10168000086080BD80B584B08DF80F000291012004
:101690008DF807009DF80F000146009120B1FFE78B
:1016A0000098012806D00BE00299002008608DF810
:1016B000070006E0029800F0E5F88DF8070000E06A
:1016C000FFE79DF8070004B080BD00BF80B586B07D
:1016D0008DF817000491039201208DF80B009DF8FE
:1016E00017000146019120B1FFE7019801280BD0B6
:1016F00011E003990120086004990868013008602E
:1017000000208DF80B0007E00498039900F0E2F840
:101710008DF80B0000E0FFE79DF80B0006B080BDE0
:1017200080B584B08DF80F000291002001909DF8E3
:101730000F000146009120B1FFE70098012803D077
:1017400007E00298019005E0029800F00DF9019081
:1017500000E0FFE7019804B080BD00BF80B582B013
:101760008DF8070000919DF80700012804D1FFE7DC
:10177000009800F037F900E0FFE702B080BD00BF3D
:1017800040F68820C2F20000006810B9FFE772B688
:10179000FFE740F68821C2F20001086801300860C6
:1017A000704700BF40F68820C2F20000006840B1D8
:1017B000FFE740F68821C2F200010868013808609E
:1017C000FFE740F68820C2F20000006810B9FFE78A
:1017D00062B6FFE77047000080B582B0002001903C
:1017E000019943F29050C0F2020050F8210028B94C
:1017F000FFE70121084600F01BF817E0019A43F2C9
:101800009050C0F2020050F82200406840F68C214F
:10181000C2F2000141F8220000F020F8019A40F6DF
:101820009021C2F2000101208854FFE702B080BD80
:1018300080B582B08DF807008DF80610FFE79DF89F
:10184000060040B1FFE745F29C60C0F20200D521DE
:1018500000F0E6F800E0FFE702B080BD4EF21401B0
:10186000CEF200016FF07F4008604EF21801CEF218
:101870000001002008604EF21001CEF200010520A8
:101880000860704780B584B0039000208DF80B008D
:101890000190019940F69020C2F20000405C0128BE
:1018A00005D0FFE702210846FFF7C2FF04E000F081
:1018B00007F803990860FFE79DF80B0004B080BDAE
:1018C00081B04EF21800CEF200000068009000983F
:1018D00001B0704780B584B00390029100208DF86C
:1018E00007000090009940F69020C2F20000405C92
:1018F000012805D0FFE703200221FFF799FF04E04C
:101900000398029900F006F8FFE79DF8070004B07D
:1019100080BD00BF83B0029001914EF21800CEF25C
:1019200000000068009000980299096888420ED96A
:10193000FFE74EF21400CEF2000000680099401A52
:1019400002990968084401300199086006E002988C
:1019500000680099401A01990860FFE70098029911
:10196000086003B0704700BF80B586B005900020C6
:101970000490039002900190019940F69020C2F2E9
:101980000000405C012805D0FFE704200221FFF79A
:101990004FFF24E005984EF68171C0F298118842FD
:1019A00005D3FFE704200121FFF742FF16E0059869
:1019B000019A40F68C21C2F2000151F82210A0FBDE
:1019C0000101039102900298039944F24022C0F26F
:1019D0000F0200231FF088FB0490FFE7FFE7049845
:1019E00006B080BD80B582B00190002000900099C3
:1019F00040F69020C2F20000405C012805D0FFE7CD
:101A000005200221FFF714FF08E00198009A40F634
:101A10008C21C2F2000141F82200FFE702B080BD34
:101A200082B001900091FFE7FEE7000080B582B030
:101A3000019040F2F010C2F20000007848BBFFE7CE
:101A4000019800F02FF801281BD1FFE744F278201D
:101A5000C0F20200006840F2EC11C2F200010091F5
:101A6000086000F035F800F05FF800980068406901
:101A700000F078FB40F2F011C2F200010120087082
:101A800006E040F2EC11C2F2000100200860FFE71E
:101A900006E065200022132311461FF043FEFFE7F6
:101AA00002B080BD80B582B0019001208DF80300A6
:101AB000019848B1FFE700228DF80320652011232B
:101AC00011461FF02FFEFFE79DF8030002B080BD16
:101AD00081B040F2EC10C2F20000006808B3FFE7EA
:101AE00000200090FFE7009840F2EC11C2F20001E4
:101AF00009684968884213D2FFE7009840F2EC1168
:101B0000C2F200010968C96851F8302040F69C21F2
:101B1000C2F200018854FFE7009801300090E2E72C
:101B2000FFE701B0704700BF81B040F2EC10C2F295
:101B30000000006808B3FFE700200090FFE700986E
:101B400040F2EC11C2F2000109688968884213D2A0
:101B5000FFE7009840F2EC11C2F200010968096940
:101B600051F8302040F69421C2F200018854FFE77A
:101B7000009801300090E2E7FFE701B0704700BF36
:101B800080B582B0019001208DF8030000F00AF8C2
:101B9000012801D1FFE700E0FFE79DF8030002B054
:101BA00080BD00BF80B582B08DF8070001208DF8A0
:101BB000060040F2F010C2F20000007850B9FFE7D2
:101BC00000218DF806109DF8072065200F231FF0D7
:101BD000A9FDFFE79DF8060002B080BD80B582B088
:101BE000019001208DF803000220FFF7DBFF0128A0
:101BF00023D1FFE7019800F025F801281BD1FFE76A
:101C000040F2EC10C2F2000000680069019A40F650
:101C10009421C2F20001895C00EBC100416840F6EA
:101C20009820C2F200000160006800F0B7FA0020BE
:101C30008DF8030000E0FFE700E0FFE79DF80300F8
:101C400002B080BD80B582B0019001208DF8030004
:101C500040F2EC10C2F200000068A0B1FFE701986A
:101C600040F2EC11C2F2000109688968884209D388
:101C7000FFE700218DF80310652002220B231FF0DF
:101C800051FDFFE703E000208DF80300FFE79DF81A
:101C9000030002B080BD00BF80B582B001208DF886
:101CA00007000320FFF77EFF01280DD1FFE700F0BA
:101CB00011F8012806D1FFE700F086FA00208DF820
:101CC000070000E0FFE700E0FFE79DF8070002B033
:101CD00080BD00BF80B582B001208DF8070000F004
:101CE00089FA012809D0FFE700218DF80710652047
:101CF00003220E231FF016FDFFE79DF8070002B038
:101D000080BD00BF80B582B002208DF8070004209E
:101D1000FFF748FF01280ED1FFE700F06BFA01281A
:101D200004D1FFE700208DF8070003E001208DF8C3
:101D30000700FFE700E0FFE79DF8070002B080BD65
:101D400080B582B003208DF80700FF208DF80600D3
:101D500000208DF805000E208DF804000520FFF707
:101D600021FF01282DD1FFE700F096FA8DF806003B
:101D7000FFE79DF805009DF80410884220DAFFE790
:101D80009DF806009DF8052044F65871C0F2020146
:101D900011F8121088420CD1FFE79DF8051044F6A7
:101DA0005870C0F2020000EB410040788DF8070047
:101DB00006E0FFE79DF8050001308DF80500D8E743
:101DC00000E0FFE79DF8070002B080BD80B582B05B
:101DD0004FF0FF3001900620FFF7E4FE012804D108
:101DE000FFE700F0A3FA019000E0FFE7019802B0DE
:101DF00080BD00BF80B50720FFF7D4FE012803D1C6
:101E0000FFE700F045FA00E0FFE780BD80B582B053
:101E100001900820FFF7C6FE012836D1FFE70198A0
:101E200000F036F801282ED1FFE7FEF7B3FF40F2AD
:101E3000EC10C2F200000068C068019A40F69C21D4
:101E4000C2F20001895C00EBC100007901460091FB
:101E5000032814D80099DFE801F002060A0E0020DA
:101E600000F0CCF90CE0012000F0C8F908E00220F5
:101E700000F0C4F904E0032000F0C0F900E0FFE73F
:101E8000FEF78CFF00E0FFE700E0FFE702B080BD57
:101E900080B582B0019001208DF8030040F2EC1073
:101EA000C2F200000068A0B1FFE7019840F2EC1117
:101EB000C2F2000109684968884209D3FFE700219E
:101EC0008DF80310652008220C231FF02BFCFFE780
:101ED00003E000208DF80300FFE79DF8030002B047
:101EE00080BD00BF80B582B00190019880B1FFE74E
:101EF0000199B3200880019965204880019901204B
:101F0000087101990220487101990020887106E04A
:101F100065200021092210231FF004FCFFE702B016
:101F200080BD00BF80B582B000208DF807000B2077
:101F3000FFF738FE012820D1FFE700F081F90146C4
:101F40000091032814D80099DFE801F002060A0E78
:101F500000208DF807000FE001208DF807000BE04E
:101F600002208DF8070007E003208DF8070003E04A
:101F700000208DF80700FFE700E0FFE79DF807006D
:101F800002B080BD80B582B08DF8070000208DF8CA
:101F900006000C20FFF706FE01281DD1FFE700F028
:101FA0001FF8012817D1FFE79DF8070020B9FFE7C8
:101FB000002000F0BFF90AE09DF80700012804D1D5
:101FC000FFE7012000F0B6F900E0FFE7FFE701209E
:101FD0008DF80600FFE7FFE79DF8060002B080BD20
:101FE00080B582B001208DF80700032000F0B0F822
:101FF00048B9FFE700218DF8071065200C22142353
:102000001FF09CFBFFE79DF8070002B080BD00BFFA
:1020100080B50D20FFF7C6FD012803D1FFE700F0D2
:10202000A3F9FFE780BD00BF80B582B08DF807003F
:1020300000208DF806000E20FFF7B4FD01281DD109
:10204000FFE700F01FF8012817D1FFE79DF8070010
:1020500020B9FFE7002000F08BF90AE09DF80700A7
:10206000012804D1FFE7012000F082F900E0FFE73A
:10207000FFE701208DF80600FFE7FFE79DF8060067
:1020800002B080BD80B582B001208DF8070000F05D
:102090005FF848B9FFE700218DF8071065200E2290
:1020A00014231FF04BFBFFE79DF8070002B080BD33
:1020B00080B50F20FFF776FD012803D1FFE700F080
:1020C00071F9FFE780BD00BF80B582B08DF80700D1
:1020D0008DF806108DF8052000208DF804001020E2
:1020E0008DF803001120FFF75DFD01282DD1FFE7DA
:1020F000FFE79DF804009DF80310884224DAFFE70B
:102100009DF807009DF8042044F67471C0F20201A6
:1021100001EB4201497888420FD1FFE79DF8041096
:1021200044F67470C0F2020010F811009DF8061019
:102130009DF8052000F03AF906E0FFE79DF804005D
:1021400001308DF80400D4E7FFE702B080BD00BF86
:1021500080B582B08DF807009DF8070000F06AF99D
:1021600002B080BD80B582B00190019898B1FFE7C0
:1021700000F098FC0198006801F060FF0198406849
:1021800001F0FCFF0198806801F092FC0198C068A2
:1021900000F08EFBFFE702B080BD00BF80B582B0CB
:1021A0000190019868B1FFE70198006800F0FCFD1C
:1021B0000198406801F050FE0198806800F044F9F1
:1021C000FFE702B080BD00BF80B582B00020019063
:1021D00001F0F0F901280AD0FFE701F0DFFA0190E1
:1021E0000199032001F09CF801F0BAFEFFE702B06C
:1021F00080BD00BF80B501F0C5F980BD80B582B05B
:102200008DF807009DF8070001460091032814D8B7
:102210000099DFE801F002060A0E002002F026F81D
:102220000CE0012002F022F808E0022002F01EF883
:1022300004E0032002F01AF800E0FFE702B080BDDE
:1022400080B582B000208DF8070001F0C7FE01467E
:102250000091032814D80099DFE801F002060A0E65
:1022600000208DF807000FE001208DF807000BE03B
:1022700002208DF8070007E003208DF8070003E037
:1022800000208DF80700FFE79DF8070002B080BD31
:1022900080B5FEF7E5FE80BD80B584B007208DF8DF
:1022A0000F0000208DF80E008DF8070001F0ACFF44
:1022B0000006002804D5FFE707208DF80F0030E066
:1022C00001F0A2FF4BF6E7610840029000208DF874
:1022D0000E00FFE79DF80E001F2821D8FFE70298A7
:1022E0009DF80E10C840C00798B1FFE79DF80E009A
:1022F0008DF80F009DF8070001308DF807009DF85C
:102300000700022804D3FFE755208DF80F0007E0EF
:10231000FFE7FFE79DF80E0001308DF80E00D9E7CA
:10232000FFE79DF80F0004B080BD00BF80B501F04D
:102330006BFF80BD80B582B08DF807009DF8070067
:1023400020B9FFE7002000F03BFC0AE09DF8070001
:10235000012804D1FFE7012000F032FC00E0FFE794
:10236000FFE702B080BD00BF80B500F071FC80BD0A
:1023700080B582B08DF807009DF8070020B9FFE70F
:10238000002000F097FC0AE09DF80700012804D126
:10239000FFE7012000F08EFC00E0FFE7FFE702B05E
:1023A00080BD00BF80B500F0CDFC80BD80B584B09D
:1023B0008DF80F008DF80E108DF80D2000208DF88F
:1023C0000C00102102918DF80C00FFE79DF80C0025
:1023D000029988422CD2FFE79DF80C1044F69470C5
:1023E000C0F2020000EB410040789DF80F108842D7
:1023F00017D1FFE79DF80C1044F69470C0F202006C
:10240000019010F811009DF80D1001F0A5FF019842
:102410009DF80C1010F811009DF80E1001F0E2FF6D
:1024200006E0FFE79DF80C0001308DF80C00CDE7C9
:1024300004B080BD80B582B08DF807009DF807001C
:1024400001F0DCF802B080BD80B584B00390039841
:10245000002867D0FFE703980068029000200190F1
:10246000FFE70198029988425BD2FFE70398406832
:10247000019901EB410110F8110000F055F80398A3
:102480004068019901EB410200EB420110F8120093
:10249000497800F07DF803984068019901EB41020A
:1024A00000EB420110F81200897800F0F5F803986B
:1024B0004068019901EB410200EB420110F8120063
:1024C0000A79497900F044F903984068019901EBD1
:1024D000410100EB4100C078012813D1FFE70398C8
:1024E0004068019901EB410110F8110000F07AF900
:1024F00003984068019901EB410110F8110000F0C8
:10250000A3F909E003984068019901EB410110F833
:10251000110000F009F8FFE7FFE701980130019092
:102520009FE7FFE704B080BD83B08DF80B009DF8F6
:102530000B1044F6B470C0F2020050F82100019074
:102540009DF80B1045F28800C0F2020050F82100FF
:102550000090019801680020B0EBD17F05D0FFE723
:1025600000994FF0B640086000E0FFE70199086865
:1025700020F0030008600199086820F4001008604A
:102580000199086840F00040086003B0704700BF40
:1025900085B08DF813008DF812109DF8131044F6D5
:1025A000B470C0F2020050F8210003909DF813109F
:1025B00045F28800C0F2020050F82100029000208D
:1025C0008DF807008DF80600009003990968B0EBBC
:1025D000D17F05D0FFE702994FF0B640086000E0D8
:1025E000FFE79DF8130000EB400145F25C10C0F2DC
:1025F000020000EB810080680090FFE79DF8060074
:102600000099884234D2FFE79DF8130000EB4001A7
:1026100045F25C10C0F2020000EB8100406800B39C
:10262000FFE79DF812009DF8131001EB410245F2FF
:102630005C11C0F2020101EB820149689DF806209D
:10264000895C88420CD1FFE79DF812200399086845
:1026500002F0070220F0700040EA0210086007E074
:10266000FFE7FFE79DF8060001308DF80600C5E79B
:102670009DF806000099884204D1FFE701208DF8FB
:102680000700FFE70399086840F0004008609DF8E4
:10269000070005B0704700BF84B08DF80F008DF8BB
:1026A0000E109DF80F1044F6B470C0F2020050F8FE
:1026B000210002909DF80F1045F28800C0F2020040
:1026C00050F8210001909DF80F000138014600915B
:1026D0002F2800F239800099DFE801F01818181847
:1026E000181818181818181818181818181818186A
:1026F000181818181818181818181818361818361E
:1027000036363618363636181818181802980168F2
:102710000020B0EBD17F05D0FFE701994FF0B64024
:10272000086000E0FFE79DF80E200299086802F0BB
:102730000F0220F4706040EA0220086002990868E5
:1027400040F00040086000E0FFE704B0704700BFC1
:1027500083B08DF80B008DF80A108DF809209DF8D4
:102760000B1044F6B470C0F2020050F82100019042
:102770009DF80B1045F28800C0F2020050F82100CD
:102780000090019801680020B0EBD17F05D0FFE7F1
:1027900000994FF0B640086000E0FFE79DF80B009D
:1027A000282817D0FFE79DF80A200199086802F051
:1027B000010220F4803040EA024008609DF80920C0
:1027C0000199086802F0010220F4801040EA0250EA
:1027D0000860FFE70199086840F00040086003B016
:1027E000704700BF83B08DF80B009DF80B1044F6C6
:1027F000B470C0F2020050F8210001909DF80B1057
:1028000045F28800C0F2020050F8210000900198C3
:1028100001680020B0EBD17F05D0FFE700994FF0B1
:10282000B6400860FFE70199086820F400100860CE
:102830000199086840F4001008600199086840F0A8
:102840000040086003B0704783B08DF80B009DF81E
:102850000B1044F6B470C0F2020050F82100019051
:102860009DF80B1045F28800C0F2020050F82100DC
:102870000090019801680020B0EBD17F05D0FFE700
:1028800000994FF0B640086000E0FFE70199086842
:10289000012262F3010008600199086840F4001009
:1028A00008600199086840F00040086003B0704774
:1028B00080B584B003900398A0B3FFE70398017834
:1028C0000020019000F030F8039841780120029038
:1028D00000F02AF803988178032000F025F8039887
:1028E000C178042000F020F803980179082000F056
:1028F0001BF801980399097B00F08EF80298039960
:10290000096940F2F812C2F2000211600399497994
:1029100000F082F80398806840F2F411C2F20001DE
:102920000860FFE704B080BD82B08DF807008DF825
:1029300006104DF20000C4F2070001680020B0EB61
:10294000D17F09D0FFE74DF20001C4F2070100205A
:10295000C9F273400860FFE79DF807000146009147
:1029600008284ED80099DFE801F005104C1F2E4CC6
:102970004C4C3D009DF806204DF21001C4F20701B9
:10298000086862F3000008603CE09DF806204DF204
:102990001001C4F20701086802F0010220F00200F1
:1029A00040EA420008602DE09DF806204DF210013B
:1029B000C4F20701086802F0010220F0080040EAB2
:1029C000C20008601EE09DF806204DF21001C4F21E
:1029D0000701086802F0010220F0100040EA02102E
:1029E00008600FE09DF806204DF21001C4F20701C7
:1029F000086802F0010220F4807040EA02200860BA
:102A000000E0FFE74DF20001C4F20701086840F062
:102A10000040086002B0704781B08DF803008DF867
:102A200002104DF20000C4F2070001680020B0EB74
:102A3000D17F09D0FFE74DF20001C4F20701002069
:102A4000C9F273400860FFE79DF8020080B1FFE71C
:102A50004DF21001C4F2070108689DF8033045F2F9
:102A60003442C0F2020252F82320104308600FE003
:102A70004DF21001C4F2070108689DF8033045F2D9
:102A80003442C0F2020252F8232090430860FFE76C
:102A90004DF20001C4F20701086840F000400860F0
:102AA00001B070474DF20000C4F207000168002039
:102AB000B0EBD17F09D0FFE74DF20001C4F207016E
:102AC0000020C9F273400860FFE74DF20C01C4F228
:102AD0000701086840F0010008604DF20001C4F2EF
:102AE0000701086840F000400860704780B582B078
:102AF0004DF21000C4F20700006801904DF2000092
:102B0000C4F2070001680020B0EBD17F09D0FFE7D5
:102B10004DF20001C4F207010020C9F273400860C1
:102B2000FFE701994DF21000C4F2070001604DF279
:102B30000002C4F20702116841F000411160006810
:102B40004009C007C0B1FFE7019845F22C41C0F22F
:102B50000201096808420FD0FFE740F2F810C2F204
:102B60000000006838B1FFE740F2F810C2F2000040
:102B700000688047FFE7FFE74DF21000C4F207004E
:102B800000688008C007C0B1FFE7019845F22C41FA
:102B9000C0F20201496808420FD0FFE740F2F4108A
:102BA000C2F20000006838B1FFE740F2F410C2F250
:102BB000000000688047FFE7FFE702B080BD00002B
:102BC00081B08DF8030044F21400C4F206000168DD
:102BD0000020B0EBD17F08D0FFE744F21401C4F22B
:102BE00006014FF0B6400860FFE79DF8032044F26D
:102BF0001401C4F20601086802F0010220F48060AA
:102C000040EA82200860086840F4007008609DF87F
:102C1000030048B9FFE744F21401C4F20601086852
:102C200040F01000086008E044F21401C4F206010C
:102C3000086820F010000860FFE744F21401C4F2B5
:102C40000601086840F00040086001B0704700BF0E
:102C500044F21400C4F2060001680020B0EBD17FFA
:102C600008D0FFE744F21401C4F206014FF0B64069
:102C70000860FFE744F21400C4F20600016821F482
:102C80000071016000680009C00748B1FFE744F225
:102C90001401C4F20601086820F010000860FFE784
:102CA00044F21401C4F20601086840F000400860D4
:102CB000704700BF81B08DF8030044F21C00C4F2DD
:102CC000060001680020B0EBD17F08D0FFE744F296
:102CD0001C01C4F206014FF0B6400860FFE79DF802
:102CE000032044F21C01C4F20601086802F001024C
:102CF00020F4806040EA82200860086840F4007098
:102D000008609DF8030048B9FFE744F21C01C4F2D3
:102D10000601086840F01000086008E044F21C0159
:102D2000C4F20601086820F010000860FFE744F2D2
:102D30001C01C4F20601086840F00040086001B0C0
:102D4000704700BF44F21C00C4F206000168002076
:102D5000B0EBD17F08D0FFE744F21C01C4F20601BA
:102D60004FF0B6400860FFE744F21C00C4F20600D2
:102D7000016821F40071016000680009C00748B1D2
:102D8000FFE744F21C01C4F20601086820F01000BD
:102D90000860FFE744F21C01C4F20601086840F035
:102DA00000400860704700BF80B582B00190019874
:102DB000002869D0FFE70198C07D012806D1FFE710
:102DC0000199087D897D00F061F802E000F0B6F815
:102DD000FFE70198806900F0F1F80198407D00F06C
:102DE000F7F801981C3000F01BF9019890F82D00BD
:102DF000012803D1FFE700F06BF902E000F092F93F
:102E0000FFE7019890F82C0000F0B0F9019890F8D5
:102E10003100012806D1FFE7019890F8300000F05A
:102E2000CDF902E000F00AFAFFE70198406B0128B3
:102E300003D1FFE700F02CFA02E000F04DFAFFE7C3
:102E400001990878496800F06BFA0198017A8520A9
:102E500000F0C4FA0198417A862000F0BFFA019888
:102E6000817A872000F0BAFA0198407B18B9FFE711
:102E700000F036FBFFE70198007B00F051FB019862
:102E8000006900F075FBFFE702B080BD80B582B03D
:102E90008DF807008DF8061044F21800C4F2060001
:102EA00001680020B0EBD17F08D0FFE744F21801A1
:102EB000C4F206014FF0B6400860FFE79DF8072016
:102EC00044F21801C4F206010091086802F0010200
:102ED00020F0040040EA820008609DF8062008689F
:102EE00062F300000860086840F0020008600868AB
:102EF00040F00040086044F21400C4F2060001688B
:102F00000020B0EBD17F08D0FFE744F21401C4F2F7
:102F100006014FF0B6400860FFE744F21401C4F226
:102F20000601086840F001000860086840F00040B1
:102F30000860042000F062FB02B080BD44F214007F
:102F4000C4F2060001680020B0EBD17F08D0FFE793
:102F500044F21401C4F206014FF0B640086000E0EC
:102F6000FFE744F21800C4F2060001680020B0EB4D
:102F7000D17F08D0FFE744F21801C4F206014FF0F8
:102F8000B640086000E0FFE744F21402C4F2060213
:102F9000106820F00100106044F21801C4F206012C
:102FA000086820F002000860106840F000401060DF
:102FB000086840F000400860704700BF81B0009092
:102FC000009840F6A421C2F20001086001B07047E9
:102FD00081B0009044F21400C4F2060001680020A1
:102FE000B0EBD17F08D0FFE744F21401C4F2060130
:102FF0004FF0B6400860FFE7009A44F21401C4F2B3
:103000000601086802F0010220F0020040EA4200D6
:103010000860086840F00040086001B0704700BFD9
:1030200082B001900198002850D0FFE744F22C00B4
:10303000C4F2060001680020B0EBD17F08D0FFE7A2
:1030400044F22C01C4F206014FF0B640086000E0E3
:10305000FFE70198427844F22C01C4F20601009186
:10306000086802F0070220F4E02040EA024008600D
:1030700001980278086862F30100086001980279FB
:10308000086820F47F4040EA022008600198427AF4
:10309000086802F0010220F0100040EA0210086007
:1030A0000198027A086802F0010220F0200040EA4C
:1030B00042100860086840F0004008600198C0684D
:1030C00040F6A021C2F200010860FFE702B070479D
:1030D00080B500F0CDFC44F22800C4F2060001687F
:1030E0000020B0EBD17F08D0FFE744F22801C4F202
:1030F00006014FF0B6400860FFE744F22801C4F231
:103100000601086840F440500860086840F4007008
:103110000860086840F001000860086840F000405E
:10312000086080BD44F22800C4F206000168002057
:10313000B0EBD17F08D0FFE744F22801C4F20601CA
:103140004FF0B640086000E0FFE744F22801C4F207
:103150000601086820F001000860086820F000708F
:103160000860086840F000400860704781B0009037
:1031700044F22800C4F2060001680020B0EBD17FC1
:1031800008D0FFE744F22801C4F206014FF0B64030
:103190000860FFE7009A44F22801C4F206010868BB
:1031A00002F0010220F0020040EA420008600868D4
:1031B00040F00040086001B0704700BF81B08DF85A
:1031C000030049F21800C4F2070001680020B0EBC8
:1031D000D17F09D0FFE749F21801C4F207010020AE
:1031E000C9F66700086000E0FFE79DF8030068B9D2
:1031F000FFE749F20001C4F20701086820F480608B
:103200000860086840F0010008600CE049F2000125
:10321000C4F20701086840F480600860086820F084
:1032200001000860FFE749F21801C4F207010868CD
:1032300040F00040086001B0704700BF49F218003C
:10324000C4F2070001680020B0EBD17F09D0FFE78E
:1032500049F21801C4F207010020C9F667000860AE
:1032600000E0FFE749F20001C4F20701086820F41A
:1032700080600860086820F00100086049F21801C9
:10328000C4F20701086840F000400860704700BFC2
:103290004DF20000C4F2070001680020B0EBD17FBE
:1032A00009D0FFE74DF20001C4F207010020C9F286
:1032B00073400860FFE74DF20401C4F2070108689B
:1032C00020F0010008604DF20001C4F20701086817
:1032D00040F00040086070474DF20000C4F2070063
:1032E00001680020B0EBD17F09D0FFE74DF200016B
:1032F000C4F207010020C9F273400860FFE74DF2F5
:103300000401C4F20701086840F0010008604DF2B2
:103310000001C4F20701086840F0004008607047EF
:1033200080B584B08DF80F00029100208DF8070061
:103330009DF80F00012814D1FFE7032000F05EF98B
:10334000012804D0FFE700208DF8070008E002986C
:1033500000F086F900F098F901208DF80700FFE7EA
:1033600037E09DF80F00022814D1FFE7042000F099
:1033700045F9012804D0FFE700208DF8070008E098
:10338000029800F06DF900F09FF901208DF8070018
:10339000FFE71DE09DF80F00032814D1FFE705208B
:1033A00000F02CF9012804D0FFE700208DF8070079
:1033B00008E0029800F054F900F0A6F901208DF819
:1033C0000700FFE703E000208DF80700FFE7FFE7B5
:1033D000FFE79DF8070004B080BD00BF82B08DF804
:1033E00007008DF806109DF807000146009185281A
:1033F00008D0FFE70098862828D0FFE700988728A4
:1034000048D06AE044F20C00C4F2060001680020D3
:10341000B0EBD17F08D0FFE744F20C01C4F2060103
:103420004FF0B640086000E0FFE744F20C01C4F240
:103430000601086820F470609DF8062040EA02202A
:103440000860086840F00040086047E044F20C0063
:10345000C4F2060001680020B0EBD17F08D0FFE77E
:1034600044F20C01C4F206014FF0B640086000E0DF
:10347000FFE744F20C01C4F20601086820F0F000F6
:103480009DF8062040EA02100860086840F00040FD
:10349000086023E044F20C00C4F20600016800203A
:1034A000B0EBD17F08D0FFE744F20C01C4F2060173
:1034B0004FF0B640086000E0FFE744F20C01C4F2B0
:1034C0000601086820F00F009DF8062010430860F0
:1034D000086840F00040086000E0FFE702B0704775
:1034E00044F21C00C4F2060001680020B0EBD17F5A
:1034F00008D0FFE744F21C01C4F206014FF0B640C9
:10350000086000E0FFE744F21C01C4F2060108680D
:1035100020F001000860086840F000400860704733
:1035200081B0009044F21C00C4F206000168002043
:10353000B0EBD17F08D0FFE744F21C01C4F20601D2
:103540004FF0B640086000E0FFE7009A44F21C012B
:10355000C4F20601086802F0010220F0020040EA0D
:1035600042000860086840F00040086001B0704701
:1035700081B00090009840F6A821C2F200010860D6
:1035800001B0704782B000208DF8070044F2280097
:10359000C4F206000068C0F30040009000980128C3
:1035A00004D1FFE701208DF80700FFE79DF8070031
:1035B00002B0704781B000208DF8030044F228006B
:1035C000C4F206000068400CC00720B1FFE70120EC
:1035D0008DF80300FFE79DF8030001B0704700BFBE
:1035E00081B044F21C00C4F206000068C0F3004041
:1035F00000909DF8000001B0704700BF80B582B018
:103600008DF8070000208DF806009DF807000138AE
:103610000146009104281ED80099DFE801F0030854
:103620000D12170000F0E0F88DF8060014E000F02D
:10363000FFF88DF806000FE000F01EF98DF8060087
:103640000AE000F03DF98DF8060005E000F05CF9B5
:103650008DF8060000E0FFE79DF8060002B080BD8F
:1036600081B00090009801384DF68361C4F21B319F
:10367000A0FB0110C20D0821C4F20201086862F328
:103680000300086001B0704744F20C00C4F2060069
:1036900001680020B0EBD17F08D0FFE744F20C01B5
:1036A000C4F206014FF0B6400860FFE744F20C0197
:1036B000C4F206010868012262F31240086008683B
:1036C00040F000400860704744F20C00C4F206006D
:1036D00001680020B0EBD17F08D0FFE744F20C0175
:1036E000C4F206014FF0B6400860FFE744F20C0157
:1036F000C4F206010868022262F3124008600868FA
:1037000040F000400860704744F20C00C4F206002C
:1037100001680020B0EBD17F08D0FFE744F20C0134
:10372000C4F206014FF0B6400860FFE744F20C0116
:10373000C4F206010868032262F3124008600868B8
:1037400040F000400860704781B08DF8030044F2FB
:103750002C00C4F2060001680020B0EBD17F08D035
:10376000FFE744F22C01C4F206014FF0B6400860B6
:1037700000E0FFE79DF8032044F22C01C4F20601AB
:10378000086802F0010220F0200040EA42100860C0
:10379000086840F00040086001B0704740F6A02083
:1037A000C2F200000068704744F21C00C4F2060038
:1037B00001680020B0EBD17F08D0FFE744F21C0184
:1037C000C4F206014FF0B640086000E0FFE744F2A3
:1037D0001C01C4F20601086840F001000860086896
:1037E00040F000400860704782B000208DF807006C
:1037F0000090FFE7009848F29F61C0F20101884203
:1038000012D8FFE74DF20400C4F2070000688008F8
:10381000C00720B1FFE701208DF8070004E0FFE7B3
:10382000009801300090E5E79DF8070002B070476E
:1038300082B000208DF807000090FFE7009844F662
:103840003F31C0F24C01884212D8FFE749F2000034
:10385000C4F207000068400AC00720B1FFE701205A
:103860008DF8070004E0FFE7009801300090E5E7DD
:103870009DF8070002B0704782B000208DF8070065
:103880000090FFE7009848F29F61C0F20101884272
:1038900012D8FFE744F21C00C4F206000068000CD6
:1038A000C00720B1FFE701208DF8070004E0FFE723
:1038B000009801300090E5E79DF8070002B07047DE
:1038C00082B000208DF807000090FFE7009848F2D2
:1038D0009F61C0F20101884212D8FFE744F2140050
:1038E000C4F206000068000CC00720B1FFE7012009
:1038F0008DF8070004E0FFE7009801300090E5E74D
:103900009DF8070002B0704782B000208DF80700D4
:103910000090FFE7009848F29F61C0F201018842E1
:1039200034D8FFE744F22800C4F206000068000C17
:10393000C00730B3FFE744F22800C4F20600016874
:103940000020B0EBD17F08D0FFE744F22801C4F299
:1039500006014FF0B6400860FFE744F22801C4F2C8
:103960000601086840F000700860086820F40070E4
:103970000860086840F00040086001208DF80700EA
:1039800004E0FFE7009801300090C3E79DF80700CE
:1039900002B0704780B544F21400C4F2060000681B
:1039A000800CC00768B3FFE744F21400C4F20600BD
:1039B00001680020B0EBD17F08D0FFE744F214018A
:1039C000C4F206014FF0B6400860FFE744F214016C
:1039D000C4F20601086840F480200860086840F0DE
:1039E0000040086040F6A420C2F20000006838B130
:1039F000FFE740F6A420C2F2000000688047FFE71E
:103A0000FFE744F21C00C4F206000068800CC00707
:103A100068B3FFE744F21C00C4F20600016800200E
:103A2000B0EBD17F08D0FFE744F21C01C4F20601DD
:103A30004FF0B6400860FFE744F21C01C4F20601F3
:103A4000086840F480200860086840F00040086082
:103A500040F6A820C2F20000006838B1FFE740F647
:103A6000A820C2F2000000688047FFE7FFE780BDA2
:103A700044F23000C4F2060001680020B0EBD17FB0
:103A800008D0FFE744F23001C4F206014FF0B6401F
:103A90000860FFE744F23001C4F20601086840F014
:103AA00080700860086840F00040086070470000BF
:103AB00080B588B007900798002873D0FFE7079873
:103AC00001780020039000F06FF8079841780120FA
:103AD000049000F069F8079881780220059000F0C2
:103AE00063F80798C1780320069000F05DF8079806
:103AF00001790420009000F057F8079841790520DB
:103B0000019000F051F8079881790620029000F0AA
:103B10004BF803980799C97900F072F8049807994F
:103B2000097A00F06DF80798407A00F099F8079844
:103B3000807A00F0A9F80798C07A00F0B9F80698E2
:103B40000799897B00F0C8F800980799C97B00F0B5
:103B5000C3F801980799097C00F0BEF8029807990C
:103B6000497C00F0B9F80798017B072000F0B4F811
:103B70000798417B082000F0AFF803980799497D2A
:103B800000F01AF904980799097D00F015F90598D5
:103B90000799C97C00F010F906980799897C00F014
:103BA0000BF9FFE708B080BD81B08DF803008DF8F8
:103BB00002109DF8020080B9FFE79DF8031045F25E
:103BC0003C40C0F2020050F8212048F20401C4F247
:103BD00004010868904308600FE09DF8031045F267
:103BE0003C40C0F2020050F8212048F20401C4F227
:103BF0000401086810430860FFE701B0704700BF88
:103C000081B08DF803008DF802109DF8030078B99B
:103C1000FFE79DF8022048F20401C4F2040108689D
:103C200002F0010220F0100040EA0210086015E0E6
:103C30009DF8030001280FD1FFE79DF8022048F20C
:103C40000401C4F20401086802F0010220F020001F
:103C500040EA4210086000E0FFE7FFE701B070476C
:103C600081B08DF803009DF8033048F20401C4F2DE
:103C70000401086801229A4320F4804040EA82301F
:103C8000086001B0704700BF81B08DF803009DF857
:103C9000032048F20401C4F20401086802F00102A2
:103CA00020F4005040EA4230086001B0704700BF85
:103CB00081B08DF803009DF8032048F20401C4F29E
:103CC0000401086802F0010220F4805040EA02304A
:103CD000086001B0704700BF82B08DF807008DF812
:103CE00006109DF8070003380146009105285FD8AB
:103CF0000099DFE801F0031221303F4E9DF80620C5
:103D000048F22801C4F20401086802F0030220F41A
:103D1000405040EA023008604BE09DF8062048F22F
:103D20002801C4F20401086802F0030220F44040B4
:103D300040EA823008603CE09DF8062048F2280105
:103D4000C4F20401086802F0030220F4403040EAA3
:103D5000024008602DE09DF8062048F22801C4F2D8
:103D60000401086802F0030220F4402040EA824087
:103D700008601EE09DF8062048F22801C4F2040104
:103D8000086802F0030220F4407040EA0220086054
:103D90000FE09DF8062048F22801C4F204010868EB
:103DA00002F0030220F4406040EA8220086000E054
:103DB000FFE702B0704700BF82B08DF807008DF8B2
:103DC00006109DF8070001460091032840D800998D
:103DD000DFE801F00211202F9DF8062048F22801AB
:103DE000C4F20401086802F0010220F0006040EA19
:103DF000C26008602DE09DF8062048F22801C4F258
:103E00000401086802F0010220F0806040EA82604C
:103E100008601EE09DF8062048F22801C4F2040163
:103E2000086802F0010220F0007040EA4260086079
:103E30000FE09DF8062048F22801C4F2040108684A
:103E400002F0010220F0807040EA0260086000E0A9
:103E5000FFE702B0704700BF80B582B001900198C3
:103E600078B1FFE701988078012806D1FFE7019932
:103E70000878497800F008F802E000F067F8FFE7FA
:103E8000FFE702B080BD00BF82B08DF807008DF85B
:103E9000061048F20001C4F20401086820F4006032
:103EA00008609DF807000146009104280DD3FFE744
:103EB00000980838032808D3FFE700980B281BD088
:103EC000FFE700980C2821D02AE048F20001C4F254
:103ED0000401086820F0300008609DF8072044F2D3
:103EE0001001C4F20601086802F00F0220F47020ED
:103EF00040EA0240086014E048F20001C4F2040104
:103F00000868012262F3051008600AE048F2000127
:103F1000C4F204010868022262F30510086000E0A0
:103F2000FFE79DF8062048F20001C4F2040108688A
:103F300002F0070220F4E06040EA0220086008680E
:103F400040F40060086002B0704700BF48F2000112
:103F5000C4F20401086820F400600860704700BFE4
:103F600082B048F20000C4F204000168C1F30221EB
:103F7000019100680009800770BBFFE744F2100060
:103F8000C4F206000068C0F303400A2824D1FFE70A
:103F900048F20001C4F204010091086820F40060B6
:103FA0000860086820F03000086044F21002C4F293
:103FB000060210680A2363F313401060019A086830
:103FC00002F0070220F4E06040EA0220086008687E
:103FD00040F400600860FFE702B0704782B04EF224
:103FE0002800C4F20700006800F00F008DF80600FA
:103FF0009DF80600013801460091072816D800995F
:10400000DFE801F00408140C1414141000208DF8DB
:1040100007000FE001208DF807000BE002208DF86B
:10402000070007E003208DF8070003E000208DF86B
:104030000700FFE79DF8070002B0704780B582B027
:1040400001900198C8B1FFE70198007800F018F8D6
:104050000198407800F024F80198406800F030F8AA
:104060000198007A00F03EF80198407A00F04AF892
:104070000198C06800F056F8FFE702B080BD00BFAD
:1040800081B08DF803009DF803204EF20C01C4F2BC
:104090000701086862F30100086001B0704700BFC3
:1040A00081B08DF803009DF803204EF20C01C4F29C
:1040B00007010868520862F38200086001B0704787
:1040C00081B00090009800F01F024EF20C01C4F283
:1040D0000701086820F4F85040EA0220086001B0A7
:1040E000704700BF81B00090009A4EF20C01C4F2FC
:1040F0000701086820F0004040EAC270086001B083
:10410000704700BF81B08DF803009DF803204EF288
:104110001C01C4F20701086862F30100086001B0E5
:10412000704700BF82B001900020009001984BF2D0
:10413000646108400090009880B1FFE74EF21C01D6
:10414000C4F2070108684BF264629043009A10437E
:104150000860086840F0800008600DE04EF21C0125
:10416000C4F2070108684BF2646290430860086873
:1041700020F080000860FFE702B0704780B582B091
:104180000190019870B1FFE70198007800F00CF8F9
:104190000198406800F016F801998868C96800F035
:1041A00021F8FFE702B080BD81B00090009A4EF286
:1041B0002001C4F20701086862F30000086001B042
:1041C000704700BF81B000909DF800204EF224019E
:1041D000C4F20701086820F47F4040EA022008602A
:1041E00001B0704782B00190009101984EF22C010D
:1041F000C4F20701086000984EF23001C4F20701D2
:10420000086002B0704700BF81B04EF20800C4F2EF
:10421000070000684BF6E76108400090009850B135
:10422000FFE700984BF6E76108404EF21801C4F230
:104230000701086000E0FFE7009801B0704700BF89
:1042400081B04EF21C00C4F2070000684BF26461BA
:1042500008400090009801B0704700BF80B582B060
:1042600001900198FFF75EFF02B080BD80B582B07B
:104270008DF8070000208DF80600FFF7AFFE8DF8DF
:1042800006009DF8070001460091032820D80099F8
:10429000DFE801F002030C151BE09DF8060018B9D9
:1042A000FFE700F019F800E0FFE712E09DF80600D4
:1042B00018B9FFE700F020F800E0FFE709E09DF8FB
:1042C000060018B9FFE700F02FF800E0FFE700E074
:1042D000FFE702B080BD00BF80B54EF61051CEF2B0
:1042E0000001086820F004000860FDF75BFA30BFA9
:1042F000FDF746FA80BD00BF80B54EF22401C4F23E
:1043000007010868022262F3010008604EF61051AE
:10431000CEF20001086840F004000860FDF742FAA0
:1043200030BFFDF72DFA80BD80B54EF22401C4F2F6
:104330000701086840F0030008604EF61051CEF205
:104340000001086840F004000860FDF72BFA30BF58
:10435000FDF716FA80BD00BF81B08DF803008DF81F
:1043600002109DF803008DF801009DF80200D8B9F5
:10437000FFE79DF80300102809D1FFE74EF2300156
:10438000C4F20701086820F0010008600BE04EF25B
:104390002C01C4F2070108689DF8013001229A40FF
:1043A00090430860FFE71AE09DF80300102809D148
:1043B000FFE74EF23001C4F20701086840F0010047
:1043C00008600BE04EF22C01C4F2070108689DF86A
:1043D000013001229A4010430860FFE7FFE701B077
:1043E000704700BF81B08DF803008DF802109DF872
:1043F00003008DF801009DF803000E281FD8FFE789
:104400009DF8020068B9FFE74EF22C01C4F20701E3
:1044100008689DF801304FF480329A40904308605C
:104420000CE04EF22C01C4F2070108689DF801303F
:104430004FF480329A4010430860FFE7FFE701B075
:10444000704700BF81B08DF803009DF803008DF820
:1044500002004EF23400C4F2070000689DF802101A
:10446000C840C00720B9FFE700208DF8010003E035
:1044700001208DF80100FFE79DF8010001B07047B1
:1044800080B582B0019000208DF803008DF8020005
:104490009DF80300019900F01BF88DF802009DF8CB
:1044A0000200012812D0FFE79DF8031044F63010F7
:1044B000C0F2020050F8211040F6AC20C2F2000019
:1044C00001600068C06800F0F3FBFFE702B080BD48
:1044D00080B584B00390029100208DF80700029807
:1044E00048B9FFE7039944F63010C0F2020050F8D3
:1044F000210050B9FFE77C2000220C2311461DF05B
:1045000011F901208DF8070019E0039944F63010E5
:10451000C0F2020050F821000090009880680399D2
:10452000405C01280AD0FFE77C200022F0231146DE
:104530001DF0F8F801208DF80700FFE7FFE79DF870
:10454000070004B080BD00BF80B582B001908DF837
:10455000031000208DF80200019840F6AC21C2F251
:104560000001096800F016F88DF802009DF80200BD
:1045700001280CD0FFE701989DF8031040F6AC220B
:10458000C2F200021268D26800F048FCFFE702B0F5
:1045900080BD00BF80B588B00790069100208DF8DF
:1045A00017008DF81600069858B9FFE77C20002107
:1045B000012204920F231DF0B5F804988DF817001E
:1045C0003DE007980699098888420BD3FFE77C20D5
:1045D0000021012203920A231DF0A4F803988DF80C
:1045E00017002BE006984068079950F82100012831
:1045F0000BD0FFE77C20002101220292F0231DF066
:1046000091F802988DF8170017E007980699C96885
:1046100000F0D8FB8DF816009DF816000B280BD182
:10462000FFE77C200021012201920B231DF07AF884
:1046300001988DF81700FFE7FFE7FFE7FFE79DF818
:10464000170008B080BD00BF80B582B001908DF822
:10465000031000208DF8020001989DF8031040F629
:10466000AC22C2F20002126800F016F88DF80200C7
:104670009DF8020001280CD0FFE701989DF8031077
:1046800040F6AC22C2F200021268D26800F0F4FBDD
:10469000FFE702B080BD00BF80B584B003908DF805
:1046A0000B10019200208DF803008DF80200019894
:1046B00050B9FFE77C20002104220F231DF032F8BF
:1046C00001208DF803004AE0039801990988884287
:1046D0000AD3FFE77C20002104220A231DF022F8E0
:1046E00001208DF8030039E001984068039950F8E3
:1046F000210001280AD0FFE77C2000210422F023BA
:104700001DF010F801208DF8030026E09DF80B0045
:1047100008280ADBFFE77C20002104220D231DF07E
:1047200001F801208DF8030016E003980199C9688B
:1047300000F05EFB8DF802009DF802000E280AD101
:10474000FFE77C20002104220E231CF0EBFF012058
:104750008DF80300FFE7FFE7FFE7FFE7FFE79DF8BE
:10476000030004B080BD00BF80B582B000208DF88A
:1047700007008DF806009DF8070040F6AC21C2F254
:104780000001096800F012F88DF806009DF8060097
:10479000012809D0FFE740F6AC20C2F20000006813
:1047A000C06800F0A5FBFFE702B080BD80B584B013
:1047B0000390029100208DF80700029850B9FFE79E
:1047C0007C20002102220F231CF0ACFF01208DF879
:1047D000070012E0029880680399405C01280AD023
:1047E000FFE77C2000210222F0231CF09BFF012028
:1047F0008DF8070000E0FFE7FFE79DF8070004B031
:1048000080BD00BF80B582B0019000208DF803000C
:10481000019800F019F88DF803009DF803000128B5
:1048200010D0FFE70199B320088001997C204880CF
:104830000199012008710199022048710199002015
:104840008871FFE702B080BD80B582B00190002082
:104850008DF80300019850B9FFE77C200021032266
:1048600010231CF05FFF01208DF80300FFE79DF887
:10487000030002B080BD000082B08DF807008DF803
:1048800006109DF8071045F25840C0F2020050F89B
:10489000210000909DF80610012088400099486092
:1048A00002B0704782B08DF807008DF806109DF8B1
:1048B000071045F25840C0F2020050F82100009065
:1048C0009DF80610012088400099886002B070476A
:1048D00080B584B08DF80F008DF80E108DF80D2086
:1048E0009DF80F1045F25840C0F2020050F8210028
:1048F0000290FCF75FFA0298406901909DF80E1053
:10490000012000FA01F10198884301909DF80D0003
:104910009DF80E1000FA01F10198084301900198EA
:1049200002994861FCF74AFA04B080BD80B584B0B2
:104930000390029100200190FFE7019803998842BB
:104940000CD2FFE7029A01980B2100FB012000F036
:1049500007F8FFE7019801300190EEE704B080BD51
:1049600080B586B005900598017845F26C40C0F29C
:10497000020050F8210004900598017845F280402B
:10498000C0F2020050F8210003900598017845F22A
:104990005840C0F2020050F821000290029840698D
:1049A0000190FCF7FFF904980599497800EB810024
:1049B0000069C00BC00748B1FFE703980599497823
:1049C00000EB81014FF0B6400861FFE705984178A0
:1049D0008278049800EB8101086962F300000861A5
:1049E000059841788278049800EB810108695208A3
:1049F00062F34100086105984178C278049800EBA1
:104A00008101086902F0070220F4E06040EA022018
:104A10000861059841784279049800EB81010869A2
:104A200002F0010220F0080040EAC2000861059887
:104A30004178427A049800EB8101086902F0010292
:104A400020F0200040EA4210086105984178C279C0
:104A5000049800EB8101086920F0004040EAC27030
:104A6000086105984178027A049800EB8101086991
:104A700002F01F0220F0F85040EA0260086104983A
:104A80000599497800EB8101086940F4004008610C
:104A9000FCF78CF90598C078012807D1FFE7059845
:104AA0004178807A884002994860FFE7059841780C
:104AB000012000FA01F1019888430190059841789E
:104AC000007900FA01F101980843019001980299D8
:104AD000486106B080BD00BF80B584B08DF80F007E
:104AE0008DF80E108DF80D209DF80F1045F26C40DA
:104AF000C0F2020050F8210002909DF80F1045F21C
:104B00008040C0F2020050F821000190FCF74AF901
:104B100002989DF80E1000EB81000069C00BC007E1
:104B200048B1FFE701989DF80E1000EB81014FF0AE
:104B3000B6400861FFE79DF80D2002989DF80E1021
:104B400000EB8101086902F0070220F4E06040EA0E
:104B50000220086102989DF80E1000EB810108699F
:104B600040F400400861FCF721F904B080BD00BFAB
:104B700080B584B08DF80F008DF80E108DF80D20E3
:104B80009DF80F1045F26C40C0F2020050F8210071
:104B900002909DF80F1045F28040C0F2020050F8DC
:104BA00021000190FCF7FEF802989DF80E1000EB32
:104BB00081000069C00BC00748B1FFE701989DF86C
:104BC0000E1000EB81014FF0B6400861FFE79DF841
:104BD0000D2002989DF80E1000EB8101086902F08B
:104BE000010220F0080040EAC200086102989DF826
:104BF0000E1000EB8101086940F400400861FCF7E9
:104C0000D5F804B080BD00BF80B584B08DF80F002A
:104C10008DF80E108DF80D209DF80F1045F26C40A8
:104C2000C0F2020050F8210002909DF80F1045F2EA
:104C30008040C0F2020050F821000190FCF7B2F869
:104C400002989DF80E1000EB81000069C00BC007B0
:104C500048B1FFE701989DF80E1000EB81014FF07D
:104C6000B6400861FFE79DF80D2002989DF80E10F0
:104C700000EB8101086962F3000008619DF80D20D6
:104C800002989DF80E1000EB81010869520862F34A
:104C90004100086102989DF80E1000EB810108693F
:104CA00040F400400861FCF781F804B080BD0000CA
:104CB00080B582B00190019801694620FFF736FE69
:104CC000019800F003F802B080BD00BF80B584B049
:104CD000039003984088ADF80400039880684078FA
:104CE0008DF803000398806880788DF8020003989F
:104CF0008068C0788DF801000398806800788DF88E
:104D000000000020ADF80A00FFE7BDF80A00BDF87A
:104D10000410884254DAFFE703984068BDF80A108F
:104D200030F81100ADF80800BDF8080040098DF812
:104D30000700BDF8080000F01F008DF806009DF880
:104D400007009DF806109DF80220FFF711FF9DF85F
:104D500007009DF806109DF80120FFF755FF9DF80C
:104D6000000001281DD1FFE79DF80300012807D1AD
:104D7000FFE79DF807009DF80610FFF77DFD06E0B0
:104D80009DF807009DF80610FFF78CFDFFE79DF8E2
:104D900007009DF80610039A92681278FFF798FDB5
:104DA00007E09DF807009DF806100022FFF790FD30
:104DB000FFE7FFE7BDF80A000130ADF80A00A4E7FD
:104DC00004B080BD83B00290019100208DF80300F3
:104DD0000198C068029900EBC100407920B9FFE753
:104DE0000B208DF80300FFE79DF8030003B0704728
:104DF00083B00290019100208DF803000198C068F3
:104E0000029900EBC100807920B9FFE70E208DF8F0
:104E10000300FFE79DF8030003B0704780B584B03E
:104E200003908DF80B1001920198C068039930F837
:104E30003100ADF80200BDF8020040098DF8010014
:104E4000BDF8020000F01F008DF800009DF80B0077
:104E500028B1FFE79DF80B00012809D1FFE79DF875
:104E600001009DF800109DF80B20FFF731FD00E0D8
:104E7000FFE704B080BD00BF80B586B005908DF817
:104E8000131003920398C068059930F83100ADF80B
:104E90000A00BDF80A0040098DF80900BDF80A00B3
:104EA00000F01F008DF8080000208DF807009DF825
:104EB0001300012811D1FFE70398C068059900EBA2
:104EC000C100C0788DF807009DF809009DF8081012
:104ED0009DF80720FFF7FCFC00E0FFE79DF80900C4
:104EE0009DF808109DF81320FFF7F6FD06B080BD71
:104EF00080B584B0039003980088ADF80A000020C4
:104F0000ADF80800FFE7BDF80800BDF80A108842B8
:104F10003DDAFFE70398C068BDF8081000EBC10058
:104F2000407968BBFFE70398C068BDF8081000EB44
:104F3000C1000079012821D1FFE70398C068BDF8BE
:104F4000081030F83100ADF80600BDF80600400941
:104F50008DF80500BDF8060000F01F008DF8040074
:104F60009DF805009DF80410039AD268BDF808303A
:104F700002EBC302D278FFF7ABFC00E0FFE7FFE7EC
:104F8000FFE7BDF808000130ADF80800BBE704B04A
:104F900080BD000080B582B0019001208DF8030033
:104FA000019800F03DF88DF803009DF80300A0BBC8
:104FB000FFE744F62C70C0F20200016840F6303082
:104FC000C2F200000160006800680078002112222F
:104FD00000F054F88DF803009DF8030088B9FFE74E
:104FE00040F63030C2F200000068006800F08EF930
:104FF0008DF803009DF8030000F06AF88DF80300B7
:10500000FFE79DF8030038B9FFE740F24C11C2F208
:10501000000102200870FFE7FFE702B080BD00BF7B
:1050200080B582B0019000208DF8030040F24C1052
:10503000C2F20000007801280AD0FFE766200022B3
:10504000102311461CF06EFB01208DF80300FFE7D2
:105050009DF8030070B9FFE7019850B1FFE76620A3
:105060000022152311461CF05DFB01208DF8030082
:10507000FFE7FFE79DF8030002B080BD80B582B076
:105080008DF807008DF806108DF8052000208DF8AA
:1050900004009DF80700022815D0FFE79DF80700DF
:1050A00088B1FFE79DF8070001280CD0FFE79DF8C5
:1050B00006209DF80530662000211CF033FB0120FE
:1050C0008DF8040000E0FFE79DF8040002B080BD09
:1050D00080B582B08DF807009DF807008DF80600B6
:1050E0009DF8060070B1FFE76620002200921523AC
:1050F00011461CF017FB009840F63031C2F2000157
:10510000086000E0FFE79DF8060002B080BD00BF28
:1051100080B582B08DF8070001208DF806009DF85B
:10512000070000F025F88DF806009DF80600D8B9B4
:10513000FFE79DF8070040F63031C2F20001096830
:10514000096800F0AFF88DF806009DF807009DF89B
:10515000061000F027F88DF8060040F24C11C2F25C
:10516000000102200870FFE79DF8060002B080BD34
:1051700080B582B08DF807009DF80700012111224B
:10518000FFF77CFF8DF806009DF8060030B9FFE7B9
:10519000012000F05DF88DF80600FFE79DF806009D
:1051A00002B080BD80B582B08DF807008DF8061082
:1051B0009DF806008DF805009DF80500B0B1FFE7E9
:1051C00066200021012211231CF0ACFA9DF8050095
:1051D000022807D1FFE766200021012216231CF0D8
:1051E000ADFAFFE701208DF8050003E000208DF8FF
:1051F0000500FFE79DF8050002B080BD80B540F6D0
:105200003030C2F200000068006800F0A5F880BDF0
:1052100080B582B00190019838B9FFE7662000217F
:10522000042214231CF07EFA0FE00199B3200880B9
:105230000199662048800199012008710199022096
:105240004871019900208871FFE702B080BD00BF5E
:1052500080B582B0019000208DF80300FBF7DAFEE4
:1052600040F24C10C2F20000007802280DD0FFE797
:10527000FBF7D4FE9DF804206620002110231CF0CB
:1052800051FA01208DF8030008E040F24C11C2F2FF
:10529000000103200870FBF7C1FEFFE79DF8030043
:1052A00002B080BD80B584B08DF80F00029100205F
:1052B0008DF807008DF806009DF80F00C0B1FFE7DC
:1052C00002989DF80F1000EB8100C068406800F064
:1052D0004DF88DF806009DF8060020B9FFE7002084
:1052E0008DF8070003E001208DF80700FFE708E0D4
:1052F00000F074F98DF806009DF806008DF807009F
:10530000FFE79DF8070004B080BD00BF80B582B004
:10531000019001208DF8030000208DF80200019813
:10532000007848B9FFE700F059F98DF802009DF8C0
:1053300002008DF803000AE00198017800EB81007B
:10534000C068406800F012F88DF80300FFE79DF890
:10535000030002B080BD00BF80B582B0019001990A
:105360004868896800F086F902B080BD80B584B0D5
:10537000039042F20000C4F20500029000208DF874
:10538000070000F06DF88DF80600FFE7039848B9B4
:10539000FFE745F2D360C0F2020040F21F1100F0B7
:1053A0006BF858E09DF8060020B9FFE701208DF862
:1053B000070006E00398694600F064F88DF80700DE
:1053C000FFE79DF80700002844D1FFE7FBF72AFE1E
:1053D00000F0D6F80398C0680299C86000F0D8F8C9
:1053E0008DF807009DF8070080B9FFE703988079E2
:1053F00058B1FFE700F0C4F803988068029908618B
:1054000000F0C6F88DF80700FFE7FFE79DF80700FA
:1054100050B9FFE700F0B4F800980299886000F0F6
:10542000B7F88DF80700FFE7FBF700FE0398407917
:1054300040B1FFE70398006940F63431C2F2000141
:10544000086006E040F63431C2F200010020086036
:10545000FFE7FFE7FFE79DF8070004B080BD00BF4E
:1054600081B042F20000C4F205000090009880680C
:10547000C0F3801001B0704782B001900091FFE747
:10548000FEE700BF80B584B00390029142F20000B5
:10549000C4F20500019000208DF80300FFE7039897
:1054A00040B9FFE745F2D360C0F20200E721FFF701
:1054B000E3FF61E0019880680299086003988079B1
:1054C00030B1FFE703998868C968884204D2FFE7D2
:1054D0000398C06820B9FFE701208DF803004AE077
:1054E0000299086840F27E32904308600398007881
:1054F00000F003020299086840EA0220086003985D
:10550000807900F001020299086840EA42100860C0
:105510000398807800F001020299086840EAC2000E
:1055200008600398407800F001020299086840EA98
:10553000820008600398C07800F0010202990868B0
:1055400040EA420008600398407900F001020299A5
:10555000086840EA021008600398007900F0010230
:105560000299086840EA821008600299086840F0D1
:1055700001000860FFE7FFE79DF8030004B080BD6D
:1055800007B47A487A497B4A0160026007BC7047D9
:1055900083B00020029042F20001C4F205010191A3
:1055A0008DF80300FFE701988068000EC00780B9FE
:1055B000FFE7029849F69A11C0F20101884204D32C
:1055C000FFE702208DF8030003E00298013002900B
:1055D000E9E79DF8030003B0704700BF80B582B0D3
:1055E00042F20000C4F20500019000208DF8030093
:1055F000FFF736FFA8B3FFE7FBF714FDFFF7C0FF87
:1056000001994020C0F204108860FFF7C1FF8DF8B7
:1056100003009DF80300D8B9FFE7FFF7B1FF019938
:105620004FF6FF70C0F20100C860FFF7B1FF8DF8C0
:1056300003009DF8030050B9FFE7FFF7A1FF0199B0
:1056400000200861FFF7A4FF8DF80300FFE7FFE7E4
:10565000FBF7ECFC40F63431C2F200010020086098
:1056600003E001208DF80300FFE79DF8030002B07E
:1056700080BD00BF80B582B001900091019818B143
:10568000FFE701988047FFE7FBF7CCFC07B43748FA
:1056900039493A4A0160026007BCFBF7C7FC009831
:1056A00018B1FFE700988047FFE702B080BD00BF58
:1056B00080B584B00390029142F20000C4F205006C
:1056C000019000208DF80300FFF7CAFE012820D1C9
:1056D000FFE7FBF7A7FCFFF753FF03980199CA68A0
:1056E000C860029870B1FFE7FFF74AFF029801997E
:1056F0000A690861FFF744FF0199886840F02000BB
:105700008860FFE7FBF792FCFFF742FF8DF803008C
:1057100003E001208DF80300FFE79DF8030004B0CB
:1057200080BD00BF80B582B042F20000C4F2050027
:10573000019001988068800EC007A0B1FFE7019931
:10574000886840F08060886040F63430C2F2000023
:10575000006838B1FFE740F63430C2F2000000685C
:105760008047FFE7FFE702B080BD0000142005403E
:10577000C4A1D9B00F3B1E1AD6B1C4A07B0C0D1E1C
:1057800080B586B00590002103910291059800F044
:10579000F1F88DF806009DF80600002840F0E8803A
:1057A000FFE700208DF81300FFE79DF81300039A30
:1057B00040F2FC11C2F2000151F82210097888422F
:1057C00035DAFFE7039940F2FC10C2F2000050F80E
:1057D000211049689DF8132001EB021149680291DC
:1057E000039950F8210040689DF8131000EB011058
:1057F000007A8DF807009DF8070028B9FFE70299A5
:10580000002002F06FFC0BE09DF80700012805D195
:10581000FFE70299012002F065FC00E0FFE7FFE7E7
:10582000FFE79DF8130001308DF81300BDE700205D
:105830008DF81300FFE79DF81300039A40F2FC1166
:10584000C2F2000151F82210097A884217DAFFE704
:10585000039940F2FC10C2F2000050F82100C06829
:105860009DF8131001EB410100EB810001F01CFBDE
:10587000FFE79DF8130001308DF81300DBE70020EF
:105880008DF81300FFE79DF81300039A40F2FC1116
:10589000C2F2000151F822100978884219DAFFE7B4
:1058A000039940F2FC10C2F2000050F82100406859
:1058B0009DF8131000EB011040680290029948888F
:1058C00001F020FBFFE79DF8130001308DF8130075
:1058D000D9E700208DF81300FFE79DF81300039A25
:1058E00040F2FC11C2F2000151F82210097A8842FC
:1058F00028DAFFE7039940F2FC10C2F200000090A2
:1059000050F82100C0689DF8131001EB410200EB34
:10591000820110F82200497801F08CFB009803996D
:1059200050F82100C0689DF8131001EB410100EB15
:10593000810001F09DFBFFE79DF8130001308DF819
:105940001300CAE7039800EB400040F63831C2F27A
:1059500000010A1800205070039800EB40000A185C
:1059600002209070039800EB400201208854FFE76A
:1059700006B080BD80B584B003908DF80B10002078
:105980008DF80A000190019800EB400140F6383094
:10599000C2F20000405C58B1FFE701208DF80A0018
:1059A0009DF80B207920002114231BF0BBFE22E080
:1059B000039858B1FFE701208DF80A009DF80B20ED
:1059C0007920002110231BF0ADFE13E0019A44F66C
:1059D0002C30C0F2020050F8220040F2FC11C2F25A
:1059E000000141F822009DF80B0000F09BF88DF8B3
:1059F0000A00FFE7FFE79DF80A0004B080BD00BF82
:105A000080B584B00020029001908DF803000298C8
:105A100000EB400140F63830C2F20000405C38B97B
:105A2000FFE779200021012211231BF07BFE77E0A4
:105A3000012000F077F88DF803009DF8030000289E
:105A40006DD1FFE700208DF80F00FFE79DF80F00F4
:105A5000029A40F2FC11C2F2000151F822100978BA
:105A6000884218DAFFE7029940F2FC10C2F2000007
:105A700050F8210040689DF80F1000EB01104068BD
:105A80000190019801F026FCFFE79DF80F0001301E
:105A90008DF80F00DAE700208DF80F00FFE79DF882
:105AA0000F00029A40F2FC11C2F2000151F82210DC
:105AB000097A884217DAFFE7029940F2FC10C2F235
:105AC000000050F82100C0689DF80F1001EB410163
:105AD00000EB810001F0FCFAFFE79DF80F000130B8
:105AE0008DF80F00DBE7029A40F2FC11C2F20001D0
:105AF000002041F82200029901EB410240F63831C2
:105B0000C2F200018B1802225A70029B03EB43037E
:105B10000B449A70029A02EB42028854FFE7FFE7B7
:105B200004B080BD80B584B08DF80F0000208DF8E2
:105B30000E0002908DF80700FFE79DF80700029A1B
:105B400040F2FC11C2F2000151F82210097888429B
:105B500015DAFFE79DF807009DF80F1001F0EAF84D
:105B60008DF80E009DF80E00012801D1FFE706E038
:105B7000FFE79DF8070001308DF80700DDE79DF88D
:105B80000E0038BBFFE700208DF80700FFE79DF807
:105B90000700029A40F2FC11C2F2000151F82210F3
:105BA000097A884215DAFFE79DF807009DF80F1083
:105BB00000F070FC8DF80E009DF80E00012801D158
:105BC000FFE706E0FFE79DF8070001308DF80700CA
:105BD000DDE7FFE79DF80E0004B080BD80B584B01E
:105BE0008DF80F00ADF80C1000208DF80B0001901F
:105BF00000909DF80F00022100F038F88DF80B009E
:105C00009DF80B0078BBFFE7BDF80C00B0F5004F26
:105C100021DCFFE7019940F2FC10C2F2000050F8CD
:105C2000210040689DF80F1000EB011040680090C3
:105C3000BDF80C00009901F06BFA8DF80B009DF88F
:105C40000B0038B1FFE779200021022232231BF03C
:105C500069FDFFE706E079200021022232231BF0D4
:105C600061FDFFE7FFE704B080BD00BF80B582B0F3
:105C70008DF807008DF806100020009000989DF820
:105C8000061001F0A9F88DF805009DF8050018BB75
:105C9000FFE79DF807009DF8061001F0BFF88DF8AA
:105CA00005009DF80500B0B9FFE79DF807009DF8D5
:105CB000061001F0D1F88DF805009DF8050048B9EF
:105CC000FFE79DF807009DF8061001F033F88DF806
:105CD0000500FFE7FFE7FFE79DF8050002B080BD84
:105CE00080B584B08DF80F00ADF80C10ADF80A2027
:105CF00000208DF80900019000909DF80F0003210D
:105D0000FFF7B4FF8DF809009DF80900002846D17F
:105D1000FFE79DF80F00019A40F2FC11C2F200016A
:105D200051F82210496801EB00114978BDF80C20A8
:105D3000032300F037F888BBFFE7BDF80A00B0F591
:105D4000004F23DCFFE7019940F2FC10C2F2000093
:105D500050F8210040689DF80F1000EB01104068DA
:105D60000090BDF80C00BDF80A10009A01F044FA4A
:105D70008DF809009DF8090038B1FFE7792000216E
:105D8000032232231BF0CEFCFFE706E0792000213E
:105D9000032232231BF0C6FCFFE7FFE7FFE704B056
:105DA00080BD00BF80B586B08DF817008DF8161045
:105DB000ADF814208DF8133000208DF812000390F8
:105DC0000290029940F2FC10C2F2000050F821004B
:105DD00040689DF8171000EB0110406801909DF895
:105DE0001600B8B9FFE7019802F094F80390BDF8E7
:105DF0001400039988420BD9FFE79DF813207920FE
:105E000000211A231BF08EFC01208DF8120000E007
:105E1000FFE70AE09DF813207920002113231BF0EF
:105E200081FC01208DF81200FFE79DF8120006B0FA
:105E300080BD00BF80B584B08DF80F0000208DF8C4
:105E40000E00029001909DF80F000421FFF70EFF55
:105E50008DF80E009DF80E0090B9FFE7029940F210
:105E6000FC10C2F2000050F8210040689DF80F10AD
:105E700000EB011040680190019801F02BFAFFE758
:105E800004B080BD80B584B08DF80F0000208DF87F
:105E90000E008DF80D000290029940F2FC10C2F243
:105EA000000050F8210040689DF80F1000EB011031
:105EB000406801909DF80F000521FFF7D7FE8DF88F
:105EC0000E009DF80E0078B9FFE7019801F068FA1E
:105ED000012804D1FFE701208DF80D0003E0002028
:105EE0008DF80D00FFE7FFE79DF80D0004B080BDC1
:105EF00080B584B08DF80F0000208DF80E00029060
:105F0000029940F2FC10C2F2000050F821004068F3
:105F10009DF80F1000EB0110406801909DF80F00F4
:105F20000621FFF7A3FE8DF80E009DF80E0020B9A4
:105F3000FFE7019801F084FAFFE704B080BD00BFDD
:105F400080B584B08DF80F008DF80E1000208DF80C
:105F50000D008DF80C000290029940F2FC10C2F284
:105F6000000050F8210040689DF80F1000EB011070
:105F7000406801909DF80E0020B9FFE700208DF8E1
:105F80000C000DE09DF80E00012804D1FFE7012070
:105F90008DF80C0003E002208DF80C00FFE7FFE70E
:105FA0009DF80F000721FFF761FE8DF80D009DF8A9
:105FB0000D0080BBFFE7029940F2FC10C2F2000026
:105FC00050F8210040689DF80F1000EB0110C068E8
:105FD000072100F023F88DF80D009DF80D00C8B9D9
:105FE000FFE79DF80C00019901F0A0FA8DF80D0073
:105FF0009DF80D0038B1FFE77920002107223023FA
:106000001BF090FB05E09DF80C00019901F050FA9F
:10601000FFE7FFE7FFE704B080BD00BF80B582B0B7
:1060200001908DF80310019858B9FFE701208DF811
:1060300002009DF803207920002131231BF072FB20
:1060400003E000208DF80200FFE79DF8020002B097
:1060500080BD00BF80B582B00190019838B9FFE7DC
:1060600079200021082215231BF05CFB0FE0019929
:10607000B320088001997920488001990120087196
:10608000019902204871019900208871FFE702B050
:1060900080BD00BF80B584B08DF80F0000208DF862
:1060A0000E00ADF80C00029001909DF80F00202129
:1060B000FFF7DCFD8DF80E009DF80E00A0B9FFE79C
:1060C000029940F2FC10C2F2000050F82100406832
:1060D0009DF80F1000EB011040680190019801F04D
:1060E00089FAADF80C00FFE7BDF80C00B0F5004FE1
:1060F00007DDFFE779200021202232231BF012FB6D
:10610000FFE7BDF80C0004B080BD00BF80B584B0CF
:106110008DF80F008DF80E1000208DF80D00029004
:10612000029940F2FC10C2F2000050F821004068D1
:106130009DF80F1000EB0110406801909DF80F00D2
:106140002121FFF793FD8DF80D009DF80D0030B96A
:10615000FFE79DF80E00019901F082FAFFE704B015
:1061600080BD00BF80B584B08DF80F00ADF80C1075
:1061700000208DF80B000190019940F2FC10C2F252
:10618000000050F8210040689DF80F1000EB01104E
:10619000406800909DF80F002B21FFF767FD8DF8F8
:1061A0000B009DF80B0080BBFFE7009801F0D2FECA
:1061B0008DF80B009DF80B0038B1FFE77920002126
:1061C0002B2212231BF0AEFA1EE0BDF80C00019A40
:1061D00040F2FC11C2F2000151F8221049689DF80A
:1061E0000F2001EB0211496801F022FB8DF80B0032
:1061F0009DF80B0038B1FFE7792000212B224123C5
:106200001BF09CFAFFE7FFE7FFE704B080BD00BF8B
:1062100080B584B08DF80F00ADF80C1000208DF81B
:106220000B00019000909DF80F002A21FFF71EFD42
:106230008DF80B009DF80B0078BBFFE7019940F249
:10624000FC10C2F2000050F8210040689DF80F10C9
:1062500000EB011040680090BDF80C00B0F5004F55
:1062600013DCFFE7BDF80C00009901F02FFB8DF85F
:106270000B009DF80B0038B1FFE7792000212A229E
:1062800032231BF04FFAFFE706E0792000212A2293
:1062900032231BF047FAFFE7FFE704B080BD00BFE1
:1062A00080B584B08DF80F00ADF80C10ADF80A2061
:1062B00000208DF80900019000909DF80F00292121
:1062C000FFF7D4FC8DF809009DF80900002842D1A1
:1062D000FFE7019840F2FC11C2F2000151F82000E2
:1062E00040689DF80F2000EB0210406800909DF878
:1062F0000F00019A51F82210496801EB001149780A
:10630000BDF80C202923FFF74DFD18BBFFE7BDF8B2
:106310000A00B0F5004F07DDFFE7792000212922B0
:1063200032231BF0FFF914E0BDF80C00BDF80A1091
:10633000009A01F031FB8DF809009DF8090038B191
:10634000FFE779200021292232231BF0EBF9FFE738
:10635000FFE7FFE7FFE704B080BD00BF80B584B072
:106360008DF80F00ADF80C10ADF80A2000208DF864
:10637000090001909DF80F002D21FFF777FC8DF8A3
:1063800009009DF80900E8BBFFE79DF80F00019A9E
:1063900040F2FC11C2F2000151F82210496801EBF1
:1063A00000114978BDF80C202D23FFF7FBFC40BB02
:1063B000FFE7BDF80A00BDF80C10B0EB510F04D890
:1063C000FFE7BDF80A0038B9FFE7792000212D2248
:1063D0003A231BF0A7F913E0BDF80C00BDF80A1032
:1063E000019B40F2FC12C2F2000252F823205268D4
:1063F0009DF80F3002EB0312526801F031FBFFE70A
:10640000FFE7FFE704B080BD80B582B08DF80700DC
:1064100000208DF806000090009800EB400140F647
:106420003830C2F20000405C38B9FFE77920002123
:10643000282211231BF076F929E09DF80700032894
:106440001DD8FFE79DF80700282100F023F88DF8FC
:1064500006009DF8060088B9FFE7009940F2FC109D
:10646000C2F2000050F82100C0689DF8071001EB4F
:10647000410100EB810001F037FBFFE706E07920E6
:106480000021282236231BF04DF9FFE7FFE702B079
:1064900080BD00BF80B584B08DF80F008DF80E1060
:1064A00000208DF80D000290029940F2FC10C2F21B
:1064B000000050F82100C0689DF80F1001EB410169
:1064C00000EB8100019001984078012810D1FFE78E
:1064D0000198406858B9FFE701208DF80D009DF83C
:1064E0000E207920002135231BF01CF9FFE720E066
:1064F00001984078022810D1FFE70198806858B9C8
:10650000FFE701208DF80D009DF80E207920002175
:1065100035231BF007F9FFE70AE001208DF80D0095
:106520009DF80E207920002135231BF0FBF8FFE7B2
:10653000FFE79DF80D0004B080BD00BF80B584B0BA
:106540008DF80F00ADF80C10ADF80A2000208DF882
:10655000090001909DF80F002C21FFF787FB8DF8B3
:1065600009009DF80900E8BBFFE79DF80F00019ABC
:1065700040F2FC11C2F2000151F82210496801EB0F
:1065800000114978BDF80C202C23FFF70BFC40BB11
:10659000FFE7BDF80A00BDF80C10B0EB510F04D8AE
:1065A000FFE7BDF80A0038B9FFE7792000212C2267
:1065B0003A231BF0B7F813E0BDF80C00BDF80A1041
:1065C000019B40F2FC12C2F2000252F823205268F2
:1065D0009DF80F3002EB0312526801F0A9FAFFE7B1
:1065E000FFE7FFE704B080BD80B584B08DF80F00F1
:1065F000ADF80C10ADF80A208DF8093000208DF8A8
:106600000800019000909DF80F003721FFF72EFB46
:106610008DF808009DF80800D8BBFFE7019940F20B
:10662000FC10C2F2000050F8210040689DF80F10E5
:1066300000EB011040680090BDF80C00B0F5004F71
:106640001FDCFFE7BDF80A00BDF80C10009A01F04E
:10665000BBFC8DF808009DF8080038B1FFE77920F1
:10666000002137223A231BF05DF809E0BDF80C0049
:10667000BDF80A10009A9DF8093001F09DFAFFE775
:1066800006E079200021372232231BF04BF8FFE788
:10669000FFE704B080BD00BF80B584B08DF80F0067
:1066A000ADF80C1000208DF80B000190019800EB64
:1066B000400140F63830C2F20000405C38B9FFE7D4
:1066C000792000212E2211231BF02CF838E09DF8B0
:1066D0000F0003282CD8FFE79DF80F002E21FFF7AD
:1066E000D9FE8DF80B009DF80B0000BBFFE7BDF84D
:1066F0000C00C00598B1FFE7BDF80C00019A40F20C
:10670000FC11C2F2000151F82210C9689DF80F2057
:1067100002EB420201EB820101F0B4FA06E07920BB
:1067200000212E223D231AF0FDFFFFE7FFE706E0E0
:10673000792000212E2236231AF0F4FFFFE7FFE72D
:1067400004B080BD80B584B08DF80F00ADF80C109A
:1067500000208DF80B000190019800EB400140F6FD
:106760003830C2F20000405C38B9FFE779200021E0
:106770002F2211231AF0D6FF38E09DF80F000328CE
:106780002CD8FFE79DF80F002F21FFF783FE8DF82F
:106790000B009DF80B0000BBFFE7BDF80C00C00527
:1067A00098B1FFE7BDF80C00019A40F2FC11C2F26B
:1067B000000151F82210C9689DF80F2002EB420237
:1067C00001EB820101F084FA06E0792000212F22FA
:1067D0003D231AF0A7FFFFE7FFE706E0792000213D
:1067E0002F2236231AF09EFFFFE7FFE704B080BD9B
:1067F00080B582B08DF807008DF8061000208DF866
:1068000005000090009800EB400140F63830C2F2DD
:106810000000405C38B9FFE77920002132221123C3
:106820001AF080FF2BE09DF8070003281FD8FFE730
:106830009DF807003221FFF72DFE8DF805009DF829
:10684000050098B9FFE79DF80600009A40F2FC1198
:10685000C2F2000151F82210C9689DF8072002EB2E
:10686000420201EB820101F059FAFFE706E07920CC
:106870000021322236231AF055FFFFE7FFE702B06E
:1068800080BD00BF80B582B08DF807008DF806107E
:1068900000208DF805000090009800EB400140F6C4
:1068A0003830C2F20000405C38B9FFE7792000219F
:1068B000332211231AF036FF2BE09DF8070003283E
:1068C0001FD8FFE79DF807003321FFF7E3FD8DF8A0
:1068D00005009DF8050098B9FFE79DF80600009AAD
:1068E00040F2FC11C2F2000151F82210C9689DF873
:1068F000072002EB420201EB820101F035FAFFE7CB
:1069000006E079200021332236231AF00BFFFFE73F
:10691000FFE702B080BD00BF80B586B005900020C3
:106920008DF813000390039800EB400140F63830D7
:10693000C2F20000084480788DF80A00059800280B
:1069400000F0CB80FFE70598092100F0D5F88DF81D
:1069500013009DF81300002840F0BE80FFE7039865
:1069600000EB400140F63830C2F2000001444878A4
:106970008978884204D1FFE7059900200870AAE0D1
:10698000039800EB400140F63830C2F200000844A2
:10699000807801460191022812D3FFE7019802286E
:1069A00040F08B80FFE705990220087001208DF8E8
:1069B000130079200021092219231AF0B3FE89E07F
:1069C00000208DF80B00FFE79DF80B00039A40F2C2
:1069D000FC11C2F2000151F82210097888421EDA37
:1069E000FFE7039940F2FC10C2F2000050F82100CA
:1069F00040689DF80B1000EB0110406801F0DAF9D7
:106A00008DF813009DF81300012801D1FFE706E07F
:106A1000FFE79DF80B0001308DF80B00D4E79DF8DF
:106A2000130000283ED1FFE700208DF80B00FFE7A0
:106A30009DF80B00039A40F2FC11C2F2000151F8DC
:106A40002210097A884219DAFFE7039940F2FC1014
:106A5000C2F2000050F82100C0689DF80B1001EB55
:106A6000410100EB81009DF80A1001F00FFAFFE7E9
:106A70009DF80B0001308DF80B00D9E70599002037
:106A80000870039800EB400140F63830C2F2000075
:106A9000421891785170039901EB410101440220A1
:106AA000887009E0059903200870792000210922E7
:106AB00016231AF043FEFFE70CE005990420087046
:106AC00001208DF8130079200021092217231AF0E4
:106AD00029FEFFE7FFE7FFE709E07920002109220F
:106AE00015231AF01FFE01208DF81300FFE79DF813
:106AF000130006B080BD00BF80B584B003908DF850
:106B00000B1000208DF80A000190019800EB400165
:106B100040F63830C2F20000405C68B9FFE70399E4
:106B2000012008708DF80A009DF80B2079200021C3
:106B300011231AF0F7FD06E09DF80B00FEF7F2FFB7
:106B40008DF80A00FFE79DF80A0004B080BD00BF81
:106B500080B584B00390029100208DF8070000906A
:106B6000029848B3FFE7039830B3FFE7009800EBC3
:106B7000400140F63830C2F20000405C60B9FFE7E7
:106B8000792000210A2211231AF0CCFD029901205C
:106B900008708DF807000EE0009800EB400140F609
:106BA0003830C2F200000844407803990870029916
:106BB00000200870FFE709E001208DF80700792028
:106BC00000210A2215231AF0ADFDFFE79DF807000A
:106BD00004B080BD80B584B00390029100208DF890
:106BE00007000090029848B3FFE7039830B3FFE72F
:106BF000009800EB400140F63830C2F20000405CE3
:106C000060B9FFE7792000210B2211231AF08AFDD9
:106C10000299012008708DF807000EE0009800EB43
:106C2000400140F63830C2F20000084480780399F1
:106C30000870029900200870FFE709E001208DF834
:106C40000700792000210B2215231AF06BFDFFE7C6
:106C50009DF8070004B080BD80B584B08DF80F00AA
:106C6000029100208DF8070000900298002853D070
:106C7000FFE7009800EB400140F63830C2F2000018
:106C8000405C60B9FFE7792000210C2211231AF043
:106C900049FD0299012008708DF807003BE000983B
:106CA00000EB400140F63830C2F200000844407862
:106CB0009DF80F10884226D0FFE79DF80F000128AD
:106CC00011D0FFE79DF80F0068B1FFE779200021A0
:106CD0000C2217231AF026FD0299042008700120C7
:106CE0008DF807000EE00299002008709DF80F0053
:106CF000009901EB410240F63831C2F20001114423
:106D00008870FFE706E002990220087001208DF8E4
:106D10000700FFE7FFE709E001208DF80700792071
:106D200000210C2215231AF0FDFCFFE79DF8070057
:106D300004B080BD80B584B08DF80F008DF80E10C2
:106D400000208DF80D000290029940F2FC10C2F272
:106D5000000050F8210040689DF80F1000EB011072
:106D60004068019001984078012810D1FFE7019810
:106D7000406858B9FFE701208DF80D009DF80E20FE
:106D80007920002134231AF0CDFCFFE720E00198A0
:106D90004078022810D1FFE70198806858B9FFE7D2
:106DA00001208DF80D009DF80E207920002134235C
:106DB0001AF0B8FCFFE70AE001208DF80D009DF8FD
:106DC0000E207920002134231AF0ACFCFFE7FFE706
:106DD0009DF80D0004B080BD80B582B001908DF8A3
:106DE0000310019800EB400140F63830C2F2000079
:106DF000405C58B9FFE79DF803207920002111235A
:106E00001AF090FC01208DF8020003E000208DF8BC
:106E10000200FFE79DF8020002B080BD80B582B09D
:106E20008DF807008DF806109DF807000D280BD38C
:106E3000FFE79DF806207920002112231AF072FC4A
:106E400001208DF8050003E000208DF80500FFE724
:106E50009DF8050002B080BD80B582B08DF80700B6
:106E60008DF80610002000909DF80700009A40F26F
:106E7000FC11C2F2000151F82210097888420BDBA4
:106E8000FFE701208DF805009DF8062079200021FC
:106E900040231AF047FC03E000208DF80500FFE7CF
:106EA0009DF8050002B080BD80B582B001900198C8
:106EB00000788DF803000198407801280CD1FFE795
:106EC0000198406838B1FFE79DF8030001994968CF
:106ED00004F010FAFFE712E00198407802280CD184
:106EE000FFE70198806838B1FFE79DF8030001993A
:106EF000896801F097FAFFE700E0FFE7FFE702B0DB
:106F000080BD00BF80B584B0ADF80E0002910020B6
:106F10000190029800788DF80300BDF80E000299E8
:106F200000F04CF88DF801009DF80100002843D1D5
:106F3000FFE70298407801281CD1FFE702984068DB
:106F400000788DF802009DF803009DF8021007F00C
:106F500067F9BDF80E10484301900198C00B0190ED
:106F60009DF803009DF80210BDF80420002304F0F2
:106F70001BFD20E00298407802281AD1FFE7029812
:106F8000806800788DF802009DF8030003F0AEFBE6
:106F9000BDF80E10484301900198C00B01909DF878
:106FA00003009DF80210BDF80420002301F05AFCF4
:106FB00000E0FFE7FFE7FFE704B080BD80B584B0E5
:106FC000ADF80E00029100208DF80700BDF80E000C
:106FD000B0F5004F04D9FFE701208DF8070025E048
:106FE000BDF80E00C0F50040ADF8040002984078EE
:106FF00001460091012804D0FFE70098022808D03C
:107000000FE0BDF80400029901F004F98DF80700C3
:107010000BE0BDF80400029901F05CF98DF807005F
:1070200003E001208DF80700FFE7FFE79DF8070068
:1070300004B080BD80B582B08DF807008DF80610D1
:107040009DF80600012805D1FFE79DF8070007F02D
:10705000FBF80BE09DF80600022805D1FFE79DF83C
:10706000070003F051FB00E0FFE7FFE702B080BD3F
:1070700080B582B00190019800788DF803000198E6
:10708000407801280DD1FFE70198406840B1FFE743
:107090009DF8030001994968096804F0A9F8FFE721
:1070A00013E00198407802280DD1FFE7019880682D
:1070B00040B1FFE79DF8030001998968096801F074
:1070C00067F9FFE700E0FFE7FFE702B080BD00BF20
:1070D00080B582B00190019800788DF80300019886
:1070E0004078012805D1FFE79DF8030004F0A6FBD6
:1070F0000BE001984078022805D1FFE79DF80300D6
:1071000001F03EFB00E0FFE7FFE702B080BD00BFFB
:1071100080B586B0ADF816000491049800788DF81B
:107120000F0000208DF80E0002908DF807000498E3
:107130004078012822D1FFE704984068E8B1FFE7D2
:107140000498406800788DF80E009DF80F009DF8B7
:107150000E1007F065F802900298BDF8161048432B
:10716000C0F3CF3002909DF80F009DF80E10BDF8CF
:107170000820012304F018FCFFE739E00498407868
:10718000022833D1FFE70498806870B3FFE70498C2
:10719000806800788DF80E009DF80F0003F0A6FAC5
:1071A00002900298BDF816104843C0F3CF30029009
:1071B0009DF80F009DF80E1003F048FA022809D13F
:1071C000FFE70298B0F5004F04D3FFE701208DF8E8
:1071D000070009E09DF80F009DF80E10BDF808208B
:1071E000012301F03FFBFFE7FFE700E0FFE7FFE7D8
:1071F0009DF8070006B080BD80B586B0ADF81600DA
:10720000ADF814100492049800788DF80F00002057
:107210008DF80D00BDF81600BDF814104843C00BE2
:10722000ADF80A000498407801281AD1FFE70498C5
:107230004068A8B1FFE70498406800788DF80E0018
:107240009DF80F009DF80E10BDF81620BDF80A300D
:10725000EE464FF0010CCEF800C004F0E7FEFFE769
:1072600034E00498407802282ED1FFE70498806823
:1072700048B3FFE70498806800788DF80E009DF809
:107280000F009DF80E1003F0E1F902280AD1FFE784
:10729000BDF90A00B0F1FF3F04DCFFE701208DF8E3
:1072A0000D000FE09DF80F009DF80E10BDF81620A0
:1072B000BDF80A30EE464FF0010CCEF800C001F0E8
:1072C000B7FDFFE7FFE700E0FFE7FFE79DF80D00F0
:1072D00006B080BD80B582B00190019800788DF82D
:1072E000030001984078012828D1FFE70198406801
:1072F00000788DF802009DF803009DF8021006F05A
:1073000027FF012819D1FFE79DF803009DF802101F
:1073100007F066F88DF801009DF803009DF8021053
:10732000022206F027FF9DF803009DF802109DF849
:107330000120012304F0A2FFFFE72EE0019840782E
:10734000022828D1FFE70198806800788DF80200B4
:107350009DF803009DF8021003F08AF9012819D165
:10736000FFE79DF803009DF8021003F073FA8DF813
:1073700000009DF803009DF80210022203F03CF982
:107380009DF803009DF802109DF80020012301F0F4
:1073900025FEFFE700E0FFE7FFE702B080BD00BF8A
:1073A00080B584B0039000208DF80B000399097814
:1073B0008DF80A108DF809000398407801281AD139
:1073C000FFE703984068A8B1FFE70398406800789A
:1073D0008DF809009DF80A009DF8091005F0EEF8F7
:1073E0008DF808009DF80800002818BF01208DF8CE
:1073F0000B00FFE720E00398407802281AD1FFE74E
:1074000003988068A8B1FFE70398806800788DF83A
:1074100009009DF80A009DF8091001F049FF8DF858
:1074200007009DF80700002818BF01208DF80B0009
:10743000FFE700E0FFE7FFE79DF80B0004B080BD29
:1074400080B582B00190019800788DF80300019812
:107450004078012811D1FFE70198406860B1FFE74B
:107460000198406800788DF802009DF803009DF8AF
:10747000021005F0BFFBFFE717E0019840780228F3
:1074800011D1FFE70198806860B1FFE7019880683B
:1074900000788DF802009DF803009DF8021002F0BC
:1074A0001FF9FFE700E0FFE7FFE702B080BD00BF84
:1074B00080B584B08DF80F000291029800788DF8A5
:1074C000070002984078012813D1FFE7029840682E
:1074D00070B1FFE70298406800788DF806009DF8CB
:1074E00007009DF806109DF80F2005F009FCFFE746
:1074F00019E002984078022813D1FFE702988068CB
:1075000070B1FFE70298806800788DF806009DF85A
:1075100007009DF806109DF80F2002F067F9FFE7BD
:1075200000E0FFE7FFE704B080BD00BF80B584B096
:107530008DF80F00029101208DF807000298007865
:107540008DF8060002984078012826D1FFE70298BE
:10755000406808B3FFE70298406800788DF805009E
:107560009DF806009DF8051006F0E0FD8DF804007A
:107570009DF80400022805D0FFE79DF804000428C8
:1075800005D1FFE79DF80F00022804D1FFE7002096
:107590008DF80700FFE7FFE727E002984078022810
:1075A00021D1FFE702988068E0B1FFE70298806888
:1075B00000788DF805009DF806009DF8051003F091
:1075C00045F88DF803009DF80300022805D1FFE778
:1075D0009DF80F00022804D1FFE700208DF8070076
:1075E000FFE7FFE700E0FFE7FFE79DF8070004B0D3
:1075F00080BD00BF80B582B001900020ADF80200D0
:10760000019800788DF801000198407801280ED18A
:10761000FFE70198406800788DF800009DF80100B0
:107620009DF8001006F09AFAADF8020014E00198F7
:10763000407802280ED1FFE70198806800788DF825
:1076400000009DF801009DF8001002F093FDADF8D8
:10765000020000E0FFE7FFE7BDF8020002B080BDD6
:1076600080B582B08DF8070000910098407801281D
:1076700006D1FFE79DF80700009900F011F80CE033
:1076800000984078022806D1FFE79DF8070000998E
:1076900000F06AF800E0FFE7FFE702B080BD00BF3E
:1076A00080B584B08DF80F0002919DF80F008DF821
:1076B000070002984068407A8DF806009DF80600A1
:1076C0000138B0FA80F040098DF805000298007882
:1076D0008DF804000298406800788DF803009DF84A
:1076E00004009DF8031006F033FD03280ED0FFE7D9
:1076F0009DF80700012808D1FFE79DF804009DF8D8
:107700000310032206F036FDFFE720E09DF8070096
:10771000E0B9FFE79DF804009DF8031006F054FD62
:107720009DF804009DF8031006F012FD02280CD10C
:10773000FFE79DF804009DF8031006F051FE8DF858
:10774000050001208DF80700FFE7FFE7FFE79DF840
:1077500004009DF803109DF805209DF8073004F003
:107760008DFD04B080BD00BF80B584B08DF80F00E2
:1077700002919DF80F008DF8070002988068407A0A
:107780008DF806009DF806000138B0FA80F0400937
:107790008DF80500029800788DF804000298806842
:1077A00000788DF803009DF804009DF8031002F0A6
:1077B0005FFF03280ED0FFE79DF80700012808D1DE
:1077C000FFE79DF804009DF80310032202F014FF68
:1077D000FFE720E09DF80700E0B9FFE79DF804000F
:1077E0009DF8031002F056FF9DF804009DF8031069
:1077F00002F03EFF02280CD1FFE79DF804009DF83F
:10780000031003F027F88DF8050001208DF807001C
:10781000FFE7FFE7FFE79DF804009DF803109DF8E0
:1078200005209DF8073001F0D9FB04B080BD00BFF2
:1078300080B584B0ADF80E00029101208DF80700EC
:10784000029800788DF806000298407801281DD132
:10785000FFE7BDF80E00C0B1FFE7BDF80E10002035
:10786000B0EB113F11D1FFE700208DF8070002981F
:10787000406800788DF805009DF806009DF8051019
:10788000BDF80E2006F078FAFFE71AE0029840787B
:10789000022814D1FFE7BDF80E0078B1FFE7BDF86C
:1078A0000E003F280AD8FFE700208DF807009DF85A
:1078B0000600BDF80E1002F013FDFFE700E0FFE741
:1078C000FFE79DF8070004B080BD00BF80B586B01B
:1078D000ADF81600049100208DF80F000290049876
:1078E00000788DF807000498407801281CD1FFE744
:1078F0000498406800788DF806009DF807009DF810
:10790000061006F08DFCBDF8161048430290029850
:10791000C00B02909DF807009DF80610BDF80820E6
:10792000002304F041F833E00498407802282DD178
:10793000FFE70498806800788DF806009DF807003E
:1079400002F0D4FEBDF81610484302900298C00B16
:1079500002909DF807009DF8061002F077FE0228BD
:1079600009D1FFE70298B0F5004F04D3FFE70120EB
:107970008DF80F0009E09DF807009DF80610BDF88E
:107980000820002300F06EFFFFE700E0FFE7FFE7BD
:107990009DF80F0006B080BD80B586B0ADF816002A
:1079A000ADF814100492049800788DF80F000020B0
:1079B0008DF80D00BDF81600BDF814104843C00B3B
:1079C000ADF80A0004984078012815D1FFE7049823
:1079D000406800788DF80E009DF80F009DF80E109D
:1079E000BDF81620BDF80A30EE464FF0000CCEF878
:1079F00000C004F01BFB2FE004984078022829D136
:107A0000FFE70498806800788DF80E009DF80F005D
:107A10009DF80E1002F01AFE02280AD1FFE7BDF908
:107A20000A00B0F1FF3F04DCFFE701208DF80D00F4
:107A30000FE09DF80F009DF80E10BDF81620BDF860
:107A40000A30EE464FF0000CCEF800C001F0F0F91D
:107A5000FFE700E0FFE7FFE79DF80D0006B080BDFF
:107A600080B584B0ADF80E00ADF80C10029202980B
:107A700000788DF8070002984078012815D1FFE7BB
:107A80000298406800788DF806009DF807009DF880
:107A90000610BDF80E20BDF80C30EE464FF0000C7D
:107AA000CEF800C005F01AFD1BE0029840780228CD
:107AB00015D1FFE70298806800788DF806009DF8E0
:107AC00007009DF80610BDF80E20BDF80C30EE46FC
:107AD0004FF0000CCEF800C002F02EF900E0FFE7F6
:107AE000FFE704B080BD00BF80B582B0019001986F
:107AF00000788DF80300019840788DF802009DF819
:107B00000200012805D1FFE79DF8030006F052FAB4
:107B10000BE09DF80200022805D1FFE79DF8030065
:107B200002F092FC00E0FFE7FFE702B080BD00BF7B
:107B300080B584B0ADF80E00ADF80C10029202983A
:107B400000788DF8070002984078012815D1FFE7EA
:107B50000298406800788DF806009DF807009DF8AF
:107B60000610BDF80E20BDF80C30EE464FF0010CAB
:107B7000CEF800C005F0B2FC1BE002984078022865
:107B800015D1FFE70298806800788DF806009DF80F
:107B900007009DF80610BDF80E20BDF80C30EE462B
:107BA0004FF0010CCEF800C002F0C6F800E0FFE78D
:107BB000FFE704B080BD00BF80B586B0ADF8160009
:107BC000ADF8141004928DF80F300020ADF80C00C1
:107BD000049800788DF80B0004984078012825D18E
:107BE000FFE70498406800788DF80A009DF80B00C4
:107BF0009DF80A1006F014FBADF80C00BDF80C005F
:107C0000BDF816104843C00BADF80C009DF80B00F2
:107C10009DF80A10BDF80C20BDF814309DF80FC077
:107C2000EE46CEF800C005F05DFE29E004984078ED
:107C3000022823D1FFE70498806800788DF80A00B5
:107C40009DF80B0002F052FDADF80C00BDF80C00E1
:107C5000BDF816104843C00BADF80C009DF80B00A2
:107C60009DF80A10BDF80C20BDF814309DF80FC027
:107C7000EE46CEF800C002F057F900E0FFE7FFE75C
:107C800006B080BD80B584B0ADF80E0002910298B8
:107C9000407801460191B0B1FFE70198012804D076
:107CA000FFE70198022807D00EE002980078BDF89F
:107CB0000E1006F01FF908E002980078BDF80E10CB
:107CC00002F05AFB01E000E0FFE704B080BD00BF16
:107CD00080B584B0ADF80E0002910298407801465C
:107CE0000191B0B1FFE70198012804D0FFE70198A6
:107CF000022807D00EE002980078BDF80E1006F0BA
:107D000029F908E002980078BDF80E1002F068FB2F
:107D100001E000E0FFE704B080BD00BF80B584B0A3
:107D20008DF80F0002910298407801460191B0B1A0
:107D3000FFE70198012804D0FFE70198022807D047
:107D40000EE0029800789DF80F1006F04DF908E05B
:107D5000029800789DF80F1002F08EFB01E000E021
:107D6000FFE704B080BD00BF80B584B08DF80F0080
:107D700002910298407801460191B0B1FFE7019865
:107D8000012804D0FFE70198022807D00EE00298EE
:107D900000789DF80F1006F043F908E0029800788B
:107DA0009DF80F1002F084FB01E000E0FFE704B053
:107DB00080BD00BF80B584B00390039800788DF833
:107DC0000B0000208DF8090003984078012827D186
:107DD000FFE70398406800788DF80A009DF80B00D3
:107DE0009DF80A1006F0B4F98DF808009DF8080017
:107DF000012804D1FFE701208DF80900FFE79DF875
:107E00000B009DF80A1006F0F9F98DF807009DF8AF
:107E1000070020B1FFE701208DF80900FFE730E0FF
:107E200003984078022827D1FFE7039880680078FC
:107E30008DF80A009DF80B009DF80A1002F018FC5E
:107E40008DF806009DF80600012804D1FFE7012007
:107E50008DF80900FFE79DF80B009DF80A1002F06D
:107E600033FC8DF805009DF8050020B1FFE70120E7
:107E70008DF80900FFE703E001208DF80900FFE716
:107E8000FFE79DF8090004B080BD00BF80B584B055
:107E900003908DF80B100398407801460191A0B330
:107EA000FFE70198012804D0FFE70198022816D0C7
:107EB0002CE00398406888B1FFE79DF80B0030B9CB
:107EC000FFE703980078002106F0C6F805E0039864
:107ED0000078012106F0C0F8FFE7FFE717E00398FC
:107EE000806888B1FFE79DF80B0030B9FFE7039881
:107EF0000078002102F0F8FA05E0039800780121EB
:107F000002F0F2FAFFE7FFE701E0FFE7FFE704B066
:107F100080BD00BF83B00290029840780146009176
:107F200080B1FFE70098012804D0FFE700980228FD
:107F300004D008E04FF6FE70019008E04FF6FE70A6
:107F4000019004E0FFE74FF6FF700190FFE7019812
:107F500003B0704784B0039001208DF80B000398A4
:107F60004078012812D1FFE703984068006901902A
:107F7000019850B1FFE701980078012804D1FFE78C
:107F800000208DF80B00FFE7FFE718E0039840782A
:107F9000022812D1FFE703988068006900900098DA
:107FA00050B1FFE700980078012804D1FFE70020D6
:107FB0008DF80B00FFE7FFE700E0FFE7FFE79DF824
:107FC0000B0004B0704700BF80B586B0ADF8160056
:107FD000ADF81410049201208DF80F000498007879
:107FE0008DF80E000020ADF80C00BDF81400C0F5AF
:107FF0000040ADF806000498407801283AD1FFE728
:108000000498406800788DF805009DF80E009DF8F2
:10801000051006F005F9ADF80A00BDF80A00BDF834
:1080200006104843C00BADF80800BDF81400B0F5C9
:10803000004F1ED0FFE7BDF81400D0B1FFE7BDF838
:108040001600BDF808100844ADF80C00BDF80C008F
:10805000BDF8161088420BDDFFE7BDF80A00BDF839
:108060000C10884204DDFFE700208DF80F00FFE7C9
:10807000FFE732E09DF80E0002F038FBADF80A0091
:10808000BDF80A00BDF806104843C00BADF8080063
:10809000BDF81400B0F5004F1ED0FFE7BDF8140086
:1080A000D0B1FFE7BDF81600BDF808100844ADF8E0
:1080B0000C00BDF80C00BDF8161088420BDDFFE780
:1080C000BDF80A00BDF80C10884204DDFFE700206F
:1080D0008DF80F00FFE7FFE7FFE79DF80F0006B000
:1080E00080BD00BF80B582B08DF807000091009878
:1080F0004078012806D1FFE79DF80700009900F0BD
:1081000011F80CE000984078022806D1FFE79DF8AE
:108110000700009900F046F800E0FFE7FFE702B033
:1081200080BD00BF80B584B08DF80F000291029829
:10813000406800788DF80700029800788DF80600F6
:1081400002984068407A8DF805009DF806009DF879
:1081500007109DF80F2006F02DF99DF8050048B98D
:10816000FFE79DF806009DF807109DF80F2006F028
:108170000BF914E09DF80F0040B9FFE79DF80600E9
:108180009DF80710012206F0FFF807E09DF80600B1
:108190009DF80710002206F0F7F8FFE7FFE704B0AC
:1081A00080BD00BF80B584B08DF80F0002910298A9
:1081B000806800788DF80700029800788DF8060036
:1081C00002988068407A8DF805009DF8050048B94E
:1081D000FFE79DF806009DF807109DF80F2002F0BC
:1081E00023FB14E09DF80F0040B9FFE79DF806005F
:1081F0009DF80710012202F017FB07E09DF806002A
:108200009DF80710002202F00FFBFFE7FFE704B024
:1082100080BD00BF80B586B0ADF816000491002087
:108220008DF80F00049909788DF80E10ADF80C0048
:108230000498406800788DF805009DF80500C00797
:10824000002842D1FFE704984068807A06283BD195
:10825000FFE70498406800694088ADF806009DF883
:108260000E009DF8051005F0DBFFADF80A00BDF823
:108270000A00BDF816104843C00BADF80800BDF861
:108280001600B0F5004F1ED0FFE7BDF81600D0B1C4
:10829000FFE7BDF80600BDF808100844ADF80C0073
:1082A000BDF80C00BDF80610884207DDFFE7BDF8F9
:1082B0000A00BDF80C10884204DCFFE701208DF8AD
:1082C0000F00FFE7FFE7FFE7FFE79DF80F0006B0AD
:1082D00080BD00BF80B586B0ADF8160004910020C7
:1082E0008DF80F00049909788DF80E10ADF80C0088
:1082F0000498806800788DF805009DF80500C00797
:10830000002840D1FFE704988068807A032839D19B
:10831000FFE70498806800694088ADF806009DF882
:108320000E0002F0E3F9ADF80A00BDF80A00BDF84E
:1083300016104843C00BADF80800BDF81600B0F5A4
:10834000004F1ED0FFE7BDF81600D0B1FFE7BDF823
:108350000600BDF808100844ADF80C00BDF80C008C
:10836000BDF80610884207DDFFE7BDF80A00BDF83A
:108370000C10884204DCFFE701208DF80F00FFE7B6
:10838000FFE7FFE7FFE79DF80F0006B080BD0000A4
:1083900080B584B08DF80F000291FFE79DF80F00C3
:1083A000042809D3FFE745F2FD60C0F2020040F265
:1083B0004E6100F031F82CE0029848B9FFE745F231
:1083C000FD60C0F2020040F24F6100F025F820E0AD
:1083D0009DF80F1045F29440C0F2020050F82100C1
:1083E00001900199486920F4007048610298427830
:1083F0000199086802F0070220F01C0040EA8200A0
:108400000860029802780199086862F30100086028
:10841000FFE704B080BD00BF82B001900091FFE78C
:10842000FEE700BF80B584B08DF80F000291FFE732
:108430009DF80F00042809D3FFE745F2FD60C0F264
:10844000020040F2C461FFF7E7FF2EE0029848B94E
:10845000FFE745F2FD60C0F2020040F2C561FFF7A0
:10846000DBFF22E09DF80F000299096800F020F878
:1084700000208DF80700FFE79DF807000299097AB0
:10848000884211DAFFE79DF80F00029949689DF8CC
:10849000072051F8221000F045F8FFE79DF807008B
:1084A00001308DF80700E7E7FFE704B080BD00BFAB
:1084B00080B582B08DF807000091FFE79DF80700B6
:1084C000042809D3FFE745F2FD60C0F2020040F244
:1084D0003361FFF7A1FF23E0009848B9FFE745F2B9
:1084E000FD60C0F2020040F23461FFF795FF17E033
:1084F0009DF80700009902F0FDFA009800789DF8B9
:10850000072040F62841C2F20001885400984078C4
:108510009DF8072040F62441C2F200018854FFE78D
:1085200002B080BD80B586B08DF817000491FFE7DA
:108530009DF81700042809D3FFE745F2FD60C0F25B
:1085400002004FF4BC61FFF767FF16E1049848B9D9
:10855000FFE745F2FD60C0F2020040F2E151FFF793
:108560005BFF0AE19DF8171045F2A440C0F202003B
:1085700050F8210002909DF8171045F29440C0F287
:10858000020050F821000190049800788DF80F0047
:108590009DF80F0040088DF80E000498807A02F0D4
:1085A00017FB8DF803009DF8171040F65C30C2F2FF
:1085B000000000EB01119DF80F20002021F81200AF
:1085C0000498407A9DF8172040F64C51C2F2000101
:1085D00001EBC2019DF80F20885401989DF80F10FF
:1085E000049A527A02F00EFB9DF8032001989DF840
:1085F0000F1000EB8101886962F301008861019826
:108600009DF80F1000EB81018869022262F383005C
:10861000886101989DF80F10049AD27A02F068FBE5
:108620009DF817009DF80F10049A927A02F0D6FB7D
:1086300001989DF80F1000EB8101886B4FF6FF72D7
:10864000104388639DF80F00C00730BBFFE7049814
:10865000006908B3FFE701989DF80E10049A1269AB
:10866000127802F003FC01989DF80F1002F042FC12
:10867000012810D1FFE70498006940889DF8172071
:1086800040F60441C2F2000101EBC2019DF80E2048
:1086900021F81200FFE7FFE7FFE70498027B01984B
:1086A0009DF80F1000EB8101886902F0010220F0B3
:1086B000400040EA821088619DF817009DF80F1075
:1086C00040F6DC32C2F2000202EBC002525C00F063
:1086D00003FA9DF8171040F6BC30C2F2000000EB20
:1086E000C1019DF80F200120885401989DF80F10BA
:1086F00000EB8101886920F01000886104984068CF
:108700009DF8172040F6CC41C2F2000101EB421166
:108710009DF80F2041F82200049840689DF817202A
:1087200040F64C41C2F2000101EB42119DF80F20CE
:1087300041F822000498007A01280AD1FFE79DF849
:108740000F10012000FA01F2029908691043086134
:1087500009E09DF80F10012000FA01F20299086962
:1087600090430861FFE701989DF80F1000EB81012D
:10877000886920F020008861FFE706B080BD00BF57
:1087800085B08DF813009DF8131045F29440C0F2A7
:10879000020050F8210003909DF8131045F2A44008
:1087A000C0F2020050F8210002900399086820F0FE
:1087B0000300086002990020009008600299486058
:1087C000029988600299C86002990969029A116940
:1087D000C9B2116102994969029948610299896D8A
:1087E0000299886502990866029948660299886626
:1087F0000299C96E0299C86602990867029948678A
:10880000029988678DF80700FFE79DF807000728A1
:1088100025D8FFE702989DF8071000EB81008069DA
:1088200002989DF8071000EB8101002088610299F1
:108830009DF8072001EB820188639DF8132040F624
:108840003C31C2F2000101EBC2019DF807208854BF
:10885000FFE79DF8070001308DF80700D5E705B068
:10886000704700BF80B584B08DF80F008DF80E10F2
:10887000ADF80C208DF80B300020ADF808009DF805
:108880000E0040088DF80700BDF80C009DF80F2081
:1088900040F65C31C2F2000101EB02119DF80E209E
:1088A00021F812009DF80F1040F69C30C2F2000033
:1088B00000EBC1009DF80E10405C8DF806009DF89D
:1088C0000F009DF80E1000F0CDF8F8F743FB9DF86F
:1088D0000F1040F6BC30C2F2000000EBC1009DF862
:1088E0000E10405C022823D1FFE79DF80F1040F6E0
:1088F000BC30C2F2000000EBC1019DF80E20012047
:108900008854F8F72BFB9DF80F009DF80E1040F6E9
:10891000DC32C2F2000202EBC002525C00F0DCF872
:108920009DF80F009DF80E10002200F05BF902E0A8
:10893000F8F714FBFFE79DF8060001280FD1FFE7C9
:108940009DF80F009DF80E10BDF80C309DF80B201F
:10895000EC46CCF800201A4600F0C6F97FE09DF8FE
:108960000600022810D1FFE79DF80F009DF80E10B9
:10897000BDF80C2053089DF80B20EC46CCF80020E5
:108980001A4600F0B1F969E09DF80600032863D1AA
:10899000FFE7BDF80C00A8B9FFE79DF80F009DF8B0
:1089A0000E1040F6FC32C2F2000232F81020013202
:1089B0009DF80B30EC46CCF8003093B2002200F06A
:1089C00093F948E0BDF80C009DF80F2040F6FC310B
:1089D000C2F2000131F8121088420FD1FFE79DF872
:1089E0000F009DF80E10BDF80C209DF80B30EC46E2
:1089F000CCF80030002300F077F92BE09DF80F1041
:108A000040F6FC30C2F2000030F8110040F604429B
:108A1000C2F2000202EBC1019DF8073031F81310D9
:108A20000844BDF80C10401AADF808009DF80F007E
:108A30009DF80E1002EBC0029DF8073032F81320AB
:108A4000BDF808309DF80BC0EE46CEF800C000F02F
:108A50004BF9FFE7FFE700E0FFE7FFE7FFE704B0C0
:108A600080BD00BF80B582B08DF807008DF806107C
:108A70009DF8071040F65C30C2F2000000EB0110D8
:108A80009DF8061030F81100A8B1FFE79DF8072007
:108A900040F6FC30C2F2000030F8120040F65C31C3
:108AA000C2F2000101EB02119DF8062031F812100C
:108AB000884207D1FFE79DF807009DF8061002F0F5
:108AC00091FA06E09DF807009DF8061002F0BAFA48
:108AD000FFE702B080BD00BF80B584B08DF80F0005
:108AE0008DF80E108DF80D209DF80F1045F2944072
:108AF000C0F2020050F821000290F8F7E3F99DF867
:108B00000E0001460191072866D80199DFE801F0BF
:108B100004101C2834404C589DF80D200299C86D53
:108B200002F0010220F4807040EA0220C86554E09F
:108B30009DF80D200299C86D02F0010220F400702A
:108B400040EA4220C86548E09DF80D200299C86DB2
:108B500002F0010220F4806040EA8220C8653CE017
:108B60009DF80D200299C86D02F0010220F400600A
:108B700040EAC220C86530E09DF80D200299C86D1A
:108B800002F0010220F4805040EA0230C86524E07F
:108B90009DF80D200299C86D02F0010220F40050EA
:108BA00040EA4230C86518E09DF80D200299C86D72
:108BB00002F0010220F4804040EA8230C8650CE0F7
:108BC0009DF80D200299C86D02F0010220F40040CA
:108BD00040EAC230C86500E0FFE7F8F777F904B073
:108BE00080BD00BF80B584B08DF80F008DF80E10E9
:108BF0008DF80D209DF80F1045F29440C0F2020050
:108C000050F821000290F8F75DF99DF80E0001463A
:108C10000191072862D80199DFE801F0040C1824BB
:108C2000303C48549DF80D200299C86D62F3000055
:108C3000C86554E09DF80D200299C86D02F001024C
:108C400020F0020040EA4200C86548E09DF80D208F
:108C50000299C86D02F0010220F0040040EA82008F
:108C6000C8653CE09DF80D200299C86D02F0010234
:108C700020F0080040EAC200C86530E09DF80D20F1
:108C80000299C86D02F0010220F0100040EA0210C3
:108C9000C86524E09DF80D200299C86D02F001021C
:108CA00020F0200040EA4210C86518E09DF80D2031
:108CB0000299C86D02F0010220F0400040EA8210E3
:108CC000C8650CE09DF80D200299C86D02F0010204
:108CD00020F0800040EAC210C86500E0FFE7F8F726
:108CE000F5F804B080BD00BF80B586B08446089812
:108CF0008DF817C08DF81610ADF81420ADF81230AD
:108D00008DF8110000208DF80B009DF8160040082A
:108D10008DF80A00FFE79DF81700042809D3FFE744
:108D200045F2FD60C0F202004FF40861FFF774FBEA
:108D300079E09DF81600082809D3FFE745F2FD60A9
:108D4000C0F2020040F68101FFF766FB6BE09DF880
:108D5000171045F29440C0F2020050F82100039031
:108D600003989DF80A1002F00FFA012832D1FFE7AC
:108D7000F8F7E8F8BDF8142003989DF80A1000EB06
:108D8000C101886B4FF6FF73984310448863BDF8A8
:108D9000122003989DF80A1000EBC101C86B6FF315
:108DA0000F001044C863F8F7D1F89DF817009DF83C
:108DB0000A104900C9B200220192FFF713FF019A7D
:108DC0009DF817009DF80A1049000131C9B2FFF75C
:108DD00009FF18E0F8F7B6F8BDF8142003989DF8DD
:108DE000161000EB8101886B4FF6FF739843104417
:108DF0008863F8F7ABF89DF817009DF8161000226D
:108E0000FFF7F0FEFFE7F8F76DF89DF811200399E2
:108E1000486F02F0010220F4807040EA02204867A7
:108E2000F8F764F8FFE79DF80B0006B080BD00BFBF
:108E300080B584B0844606988DF80FC08DF80E106A
:108E4000ADF80C20ADF80A308DF809000020ADF81F
:108E50000600FFE79DF80F00042809D3FFE745F25D
:108E6000FD60C0F2020040F25E71FFF7D5FA63E0E8
:108E70009DF80E00082809D3FFE745F2FD60C0F217
:108E8000020040F25F71FFF7C7FA55E0F8F762F8A9
:108E90009DF80F1040F6BC30C2F2000000EBC1009C
:108EA0009DF80E10405C022823D1FFE79DF80F10BB
:108EB00040F6BC30C2F2000000EBC1019DF80E206C
:108EC00001208854F8F74AF89DF80F009DF80E101D
:108ED00040F6DC32C2F2000202EBC002525CFFF745
:108EE000FBFD9DF80F009DF80E100022FFF77AFEA3
:108EF00002E0F8F733F8FFE7BDF80C0020B9FFE710
:108F00000020ADF806000CE0BDF80A00ADF8060040
:108F10009DF80F00BDF80C109DF8092000F00EF828
:108F2000FFE79DF80F009DF80E10BDF806209DF894
:108F30000930FFF797FCFFE704B080BD80B584B02F
:108F40008DF80F0002918DF80720FFE79DF80F00C4
:108F5000042809D3FFE745F2FD60C0F2020040F2A9
:108F60009661FFF759FA36E09DF80F1045F29440EC
:108F7000C0F2020050F82100009002989DF80F20E6
:108F800040F6FC31C2F2000121F81200F7F7D2FFDF
:108F900000980069800AC00738B1FFE7029A00997B
:108FA000C868C0EA6200C86007E00298013800990A
:108FB000CA68C0EA0200C860FFE79DF80720009970
:108FC000486F02F0010220F4807040EA02204867F6
:108FD000F7F7B4FFFFE704B080BD00BF80B582B0F3
:108FE0008DF807008DF806108DF805208DF80430F7
:108FF000FFE79DF80700042809D3FFE745F2FD606D
:10900000C0F2020040F29171FFF706FA7BE09DF892
:109010000600082809D3FFE745F2FD60C0F2020010
:1090200040F29271FFF7F8F96DE09DF8071040F6F5
:10903000BC30C2F2000000EBC1009DF80610405C9D
:10904000022836D1FFE79DF8071040F65C30C2F2E7
:10905000000000EB01119DF80620002021F812000D
:10906000F7F718FF9DF8071040F63C30C2F20000F9
:1090700000EBC1009DF80610405C800700280FD56A
:10908000FFE79DF8071040F63C30C2F2000000EB0D
:10909000C1019DF80620885C40F004008854FFE779
:1090A000F7F7FCFE9DF807009DF8061000F02EF87B
:1090B00018E09DF8071040F6BC30C2F2000000EB4B
:1090C000C1009DF80610405C032809D1FFE79DF818
:1090D00007009DF806109DF8042000F093F800E0CA
:1090E000FFE7FFE79DF807009DF806109DF80520B3
:1090F000FFF7F2FC9DF807009DF806109DF804208C
:10910000FFF770FDFFE702B080BD00BF80B584B0FF
:109110008DF80F008DF80E109DF80F1045F2944059
:10912000C0F2020050F82100029000208DF80600E5
:10913000F7F7F0FE9DF80F1040F63C30C2F2000049
:1091400000EBC1009DF80E10405C00F009008DF8A6
:1091500007009DF8070050B9FFE702989DF80E1030
:1091600000EB8101886920F010008861FFE7029818
:109170009DF80E1000EB8101886920F020008861C5
:10918000F7F7CCFE00208DF80500FFE79DF80500FD
:1091900007281EDCFFE79DF80F1040F63C30C2F2B6
:1091A000000000EBC1009DF80510405C00F00200DB
:1091B0008DF807009DF8070020B1FFE701208DF82A
:1091C000060006E0FFE79DF8050001308DF8050078
:1091D000DCE79DF8060050B9FFE7F7F76BFE029950
:1091E000086920F400700861F7F768FEFFE7F7F7F9
:1091F00099FE0299486920F400704861F7F796FEDD
:1092000004B080BD80B582B08DF807008DF80610DF
:109210008DF805209DF8071045F29440C0F2020039
:1092200050F8210000909DF80500012807D1FFE7C4
:109230009DF807009DF80610FFF768FF36E09DF8DF
:10924000071040F63C30C2F2000000EBC1009DF870
:109250000610405C800700280AD5FFE7F7F72AFED2
:109260000099086940F400700861F7F727FEFFE7EE
:109270009DF8071040F63C30C2F2000000EBC10040
:109280009DF80610405C10F0090F0ED0FFE7F7F7CD
:1092900041FE00989DF8061000EB8101886940F0BE
:1092A00010008861F7F73AFEFFE7FFE702B080BDE4
:1092B00080B584B08DF80F008DF80E1001208DF868
:1092C0000500FFE79DF80F00042809D3FFE745F2EA
:1092D000FD60C0F2020040F2CC71FFF79DF855E04E
:1092E0009DF80E00082809D3FFE745F2FD60C0F2A3
:1092F000020040F2CD71FFF78FF847E09DF80F10A4
:1093000045F29440C0F2020050F821000290029809
:1093100000688007F0B1FFE702989DF80E1000F09A
:1093200039F88DF807009DF80700012808D1FFE7FC
:1093300002989DF80E1000F07FF88DF8050008E007
:109340009DF80F009DF80E1000F0C8F88DF805008C
:10935000FFE707E002989DF80E1000F06DF88DF819
:109360000500FFE702989DF80E1000F067F98DF8F0
:1093700006009DF80600012807D1FFE79DF80510BB
:10938000012088438DF80500FFE7FFE79DF8050001
:1093900004B080BD83B002908DF8071000208DF8D6
:1093A00006009DF807000146009107283ED8009965
:1093B000DFE801F0040B121920272E350298C06D4A
:1093C00000F001008DF8060031E00298C06DC0F396
:1093D00040008DF806002AE00298C06DC0F38000BE
:1093E0008DF8060023E00298C06DC0F3C0008DF830
:1093F00006001CE00298C06DC0F300108DF8060056
:1094000015E00298C06DC0F340108DF806000EE024
:109410000298C06DC0F380108DF8060007E0029836
:10942000C06DC0F3C0108DF8060000E0FFE79DF8A6
:10943000060003B0704700BF83B002908DF807109C
:1094400000208DF806009DF80700014600910728CE
:109450003ED80099DFE801F0040B121920272E35C1
:109460000298C06DC0F300208DF8060031E002982C
:10947000C06DC0F340208DF806002AE00298C06D50
:10948000C0F380208DF8060023E00298C06DC0F381
:10949000C0208DF806001CE00298C06DC0F30030BB
:1094A0008DF8060015E00298C06DC0F340308DF8CD
:1094B00006000EE00298C06DC0F380308DF8060003
:1094C00007E00298C06DC0F3C0308DF8060000E0E0
:1094D000FFE79DF8060003B0704700BF88B08DF825
:1094E0001F008DF81E109DF81F1045F29440C0F229
:1094F000020050F8210006900020ADF81400ADF8ED
:1095000012009DF81E1049088DF81110ADF80E00DC
:109510008DF80D009DF81F1040F69C30C2F200003F
:1095200000EBC1009DF81E10405C8DF817000698F6
:109530004068ADF814009DF817000146029101281B
:1095400008D0FFE70298022817D0FFE70298032807
:1095500026D06DE006989DF81E1000EB8100806B10
:10956000ADF81200BDF81410BDF812200020914291
:10957000B8BF01208DF80D005BE006989DF81E1025
:1095800000EB8100806BADF81200BDF81410BDF83F
:10959000122000209142B8BF01208DF80D0048E054
:1095A00006989DF8111000EBC100806BADF8120019
:1095B00006989DF8111000EBC100C06BADF80E00CD
:1095C0009DF81E00C007C8B9FFE7BDF81410BDF82C
:1095D00012200120914201900ADBFFE7BDF8141030
:1095E000BDF80E2000209142C8BF01200190FFE786
:1095F000019800F001008DF80D0018E0BDF814107E
:10960000BDF812200020914200900ADBFFE7BDF870
:109610001410BDF80E2000209142D8BF0120009008
:10962000FFE7009800F001008DF80D00FFE700E073
:10963000FFE79DF80D0008B0704700BF83B00290AF
:109640008DF8071000208DF806009DF807000146F0
:10965000009107283ED80099DFE801F0040B1219A9
:1096600020272E350298806DC0F300208DF806006B
:1096700031E00298806DC0F340208DF806002AE0AA
:109680000298806DC0F380208DF8060023E00298D8
:10969000806DC0F3C0208DF806001CE00298806D3C
:1096A000C0F300308DF8060015E00298806DC0F31D
:1096B00040308DF806000EE00298806DC0F38030D7
:1096C0008DF8060007E00298806DC0F3C0308DF879
:1096D000060000E0FFE79DF8060003B0704700BFFA
:1096E00080B582B08DF807008DF80610FFE79DF871
:1096F0000700042809D3FFE745F2FD60C0F202002D
:1097000040F60101FEF788FE6DE09DF8060008288E
:1097100009D3FFE745F2FD60C0F2020040F6020106
:10972000FEF77AFE5FE09DF80600C00730B9FFE75C
:109730009DF8060001308DF8050005E09DF8060053
:1097400001388DF80500FFE79DF8071040F69C30C2
:10975000C2F2000000EBC1009DF80610405C8DF8DD
:1097600004009DF80400032829D1FFE7F7F792FBD6
:109770009DF8071040F63C30C2F2000000EBC10239
:109780009DF80630D15C01F00801D1549DF8071016
:1097900000EBC1019DF80520885C00F0F7008854BB
:1097A000F7F77CFB9DF807009DF80610FFF7AEFC6D
:1097B0009DF807009DF80510FFF7A8FC12E09DF842
:1097C000071040F63C30C2F2000000EBC1019DF8EA
:1097D0000620002088549DF807009DF80610FFF72A
:1097E00095FCFFE7FFE702B080BD00BF80B582B007
:1097F0008DF807008DF806108DF80520FFE79DF81D
:109800000700042809D3FFE745F2FD60C0F202001B
:1098100040F63401FEF700FEB5E09DF8060008288A
:1098200009D3FFE745F2FD60C0F2020040F63501C2
:10983000FEF7F2FDA7E09DF8071045F29440C0F254
:10984000020050F821000090F7F724FB9DF8071064
:1098500040F63C30C2F2000000EBC1019DF806204A
:10986000885C00F0FC008854F7F718FBF7F752FB10
:1098700000989DF8061000EB8101886920F0200017
:109880008861F7F74BFBF7F74DFB0099486920F427
:1098900000704861F7F74AFB9DF8071040F69C30CE
:1098A000C2F2000000EBC1009DF80610405C8DF88C
:1098B00004009DF80400012809D1FFE79DF8070086
:1098C0009DF806109DF8052000F060F817E09DF85F
:1098D0000400022809D1FFE79DF807009DF8061053
:1098E0009DF8052000F0D8F808E09DF807009DF8E5
:1098F00006109DF8052000F0F3F8FFE7FFE79DF85C
:10990000071040F65C30C2F2000000EB01109DF839
:10991000061030F81100E0B1FFE79DF8072040F68F
:10992000FC30C2F2000030F8120040F65C31C2F2A6
:10993000000101EB02119DF8062031F81210884257
:1099400007D0FFE79DF807009DF8061000F068F9C2
:1099500018E0F7F79FFA9DF8071040F63C30C2F286
:10996000000000EBC1019DF80620885C40F0040077
:109970008854F7F793FA9DF807009DF80610FFF753
:10998000C5FBFFE7FFE702B080BD00BF80B582B036
:109990008DF807008DF806108DF80520F7F77AFA94
:1099A0009DF8050001460091B8B1FFE70098012835
:1099B0003FD0FFE70098022868D1FFE79DF8071025
:1099C00040F63C30C2F2000000EBC1019DF80620D9
:1099D000885C40F00300885459E09DF8071040F679
:1099E0004C50C2F2000000EBC1009DF80610405C34
:1099F00078B9FFE79DF8071040F63C30C2F200004E
:109A000000EBC1019DF80620885C40F002008854FC
:109A10000EE09DF8071040F63C30C2F2000000EB6B
:109A2000C1019DF80620885C40F001008854FFE7E2
:109A30002DE09DF8071040F64C50C2F2000000EBFC
:109A4000C1009DF80610405C01280FD1FFE79DF88A
:109A5000071040F63C30C2F2000000EBC1019DF857
:109A60000620885C40F0020088540EE09DF8071044
:109A700040F63C30C2F2000000EBC1019DF8062028
:109A8000885C40F001008854FFE700E0FFE7F7F74B
:109A900005FA02B080BD00BF80B582B08DF8070026
:109AA0008DF806108DF80520F7F7F4F99DF80500FC
:109AB00002280FD1FFE79DF8071040F63C30C2F2B4
:109AC000000000EBC1019DF80620885C40F0010019
:109AD000885400E0FFE7F7F7E1F902B080BD00BF6E
:109AE00080B582B08DF807008DF806108DF805203E
:109AF0009DF80600C00730B9FFE79DF80600013069
:109B00008DF8040005E09DF8060001388DF804008A
:109B1000FFE7F7F7BFF99DF805000146009108B38C
:109B2000FFE7009801284AD0FFE70098022872D189
:109B3000FFE79DF8071040F63C30C2F2000000EB52
:109B4000C1029DF80630D15C41F00101D1549DF86D
:109B5000071000EBC1019DF80420885C40F008006C
:109B6000885459E09DF8071040F64C50C2F20000AE
:109B700000EBC1009DF80610405C01280FD1FFE703
:109B80009DF8071040F63C30C2F2000000EBC10126
:109B90009DF80620885C40F0010088540EE09DF896
:109BA000071040F63C30C2F2000000EBC1019DF806
:109BB0000420885C40F008008854FFE72CE09DF802
:109BC000071040F64C50C2F2000000EBC1009DF8B7
:109BD0000610405C78B9FFE79DF8071040F63C306E
:109BE000C2F2000000EBC1019DF80620885C40F045
:109BF000010088540EE09DF8071040F63C30C2F298
:109C0000000000EBC1019DF80420885C40F00800D2
:109C10008854FFE700E0FFE7F7F740F902B080BDA6
:109C200080B584B08DF80F008DF80E109DF80F10E0
:109C300045F29440C0F2020050F8210002909DF8D5
:109C40000F1040F69C30C2F2000000EBC1009DF8FE
:109C50000E10405C8DF807009DF80E00C00730B96B
:109C6000FFE79DF80E0001308DF8060005E09DF835
:109C70000E0001388DF80600FFE79DF80F1040F642
:109C80003C30C2F2000000EBC1009DF80E10405CB9
:109C9000800700280AD5FFE7F7F70CF90299086951
:109CA00040F400700861F7F709F9FFE7F7F732F9B8
:109CB0009DF80F1040F63C30C2F2000000EBC100EE
:109CC0009DF80E10405CC00750B1FFE702989DF868
:109CD0000E1000EB8101886940F010008861FFE7F9
:109CE0009DF80700032823D1FFE702989DF806108E
:109CF00000EB8101886920F0200088619DF80F1039
:109D000040F63C30C2F2000000EBC1009DF80610A6
:109D1000405C000700280AD5FFE702989DF806106E
:109D200000EB8101886940F010008861FFE7FFE7E0
:109D3000F7F7F4F804B080BD80B586B08446089883
:109D40008DF817C08DF81610ADF81420ADF812304C
:109D50008DF811000020ADF8040001208DF80300FB
:109D60008DF80200FFE79DF81700042809D3FFE7EC
:109D700045F2FD60C0F2020040F6BD01FEF74CFB6B
:109D8000CFE09DF81600082809D3FFE745F2FD60F3
:109D9000C0F2020040F6BE01FEF73EFBC1E09DF8B6
:109DA000171040F69C30C2F2000000EBC1009DF895
:109DB0001610405C8DF807009DF80700032804D0BA
:109DC000FFE700208DF80300FFE79DF8030048B986
:109DD000FFE745F2FD60C0F2020040F6C701FEF762
:109DE0001BFB9EE0BDF81200BDF8141000EB510003
:109DF000ADF80400BDF80400BDF81210884207DD7C
:109E0000FFE7BDF81400BDF80410884204DCFFE74A
:109E100000208DF80200FFE79DF8020048B9FFE737
:109E200045F2FD60C0F2020040F6CF01FEF7F4FA01
:109E300077E09DF8160040088DF810009DF8171087
:109E400045F29440C0F2020050F821000290BDF8A3
:109E500014009DF8172040F6FC31C2F2000121F8F1
:109E60001200F7F767F802980069800AC00758B136
:109E7000FFE7BDF814200299C8684FF6FF739843B6
:109E800040EA5200C86008E0BDF8140001380299A9
:109E9000CA68C0EA0200C860FFE7F7F74FF8BDF8EC
:109EA00014004008ADF80E00BDF80E009DF8172014
:109EB00040F65C31C2F2000101EB02119DF8162060
:109EC00021F81200F7F73EF8BDF8122002989DF82D
:109ED000101000EBC101886B4FF6FF7398431044DC
:109EE0008863BDF81200BDF80E10084402999DF871
:109EF000102001EBC201CA6BC0EA0200C863F7F789
:109F000025F8F6F7EFFF9DF811200299486F02F04F
:109F1000010220F4807040EA02204867F6F7E6FF6D
:109F2000FFE706B080BD00BF80B586B084460898C4
:109F30008DF817C08DF81610ADF81420ADF812305A
:109F40008DF811000020ADF80E00ADF80C009DF862
:109F5000161049088DF80B10ADF8080001208DF897
:109F600007008DF80600FFE79DF81700042809D3C5
:109F7000FFE745F2FD60C0F2020040F60E11FEF769
:109F80004BFAF5E09DF81600082809D3FFE745F2E3
:109F9000FD60C0F2020040F60F11FEF73DFAE7E067
:109FA0009DF8171040F69C30C2F2000000EBC10093
:109FB0009DF81610405C8DF80A009DF80A000328F1
:109FC00004D0FFE700208DF80700FFE79DF80700A9
:109FD00048B9FFE745F2FD60C0F2020040F61811F3
:109FE000FEF71AFAC4E09DF8171040F6FC30C2F2F2
:109FF000000030F81100BDF8141088422DD0FFE7A2
:10A00000BDF8140048B3FFE7BDF812009DF8172013
:10A0100040F6FC31C2F2000131F812100844BDF8DC
:10A020001410401AADF80800BDF80800BDF8121071
:10A0300088420DDDFFE79DF8171040F6FC30C2F2B4
:10A04000000030F81100BDF80810884204DCFFE77A
:10A0500000208DF80600FFE7FFE79DF8060048B9ED
:10A06000FFE745F2FD60C0F2020040F62211FEF764
:10A07000D3F97DE0BDF812009DF8172040F60441A9
:10A08000C2F2000101EBC2019DF80B2021F8120081
:10A09000BDF814009DF8172040F65C31C2F20001B3
:10A0A00001EB02119DF8162021F81200BDF81200F4
:10A0B00020B9FFE70120ADF80E0004E0BDF8120062
:10A0C000ADF80E00FFE79DF8171040F6FC30C2F225
:10A0D000000030F81100BDF8141088420FD1FFE7DE
:10A0E0009DF8171040F60440C2F2000000EBC100DA
:10A0F0009DF80B1030F81100ADF80C0028E0BDF809
:10A10000140058B9FFE79DF8171040F6FC30C2F272
:10A11000000030F81100ADF80C0018E09DF8172091
:10A1200040F60440C2F2000000EBC2009DF80B10A4
:10A1300030F8110040F6FC31C2F2000131F8121083
:10A140000844BDF81410401AADF80C00FFE7FFE713
:10A150009DF817009DF81610BDF80E20BDF80C30C4
:10A160009DF811C0EE46CEF800C0FEF7BDFDFFE73A
:10A1700006B080BD80B586B08DF817008DF816103A
:10A1800000200490FFE79DF81700042809D3FFE79B
:10A1900045F2FD60C0F2020040F65411FEF73CF9B2
:10A1A00099E09DF81600082809D3FFE745F2FD6005
:10A1B000C0F2020040F65511FEF72EF98BE09DF833
:10A1C000171045F29440C0F2020050F821000390AD
:10A1D0009DF8171040F69C30C2F2000000EBC10061
:10A1E0009DF81610405C8DF80B009DF81600400895
:10A1F0008DF80A0003989DF81610FFF7CBF8002899
:10A2000068D1FFE79DF80B0003283AD1FFE70398D8
:10A21000C168012010FA81F0019003989DF80A109E
:10A2200000EBC100C06B80B20090009803999DF8CC
:10A230000A2001EBC201896B89B288420BD9FFE782
:10A24000009803999DF80A2001EBC201896B89B23D
:10A25000401A009002E000200090FFE7009801996A
:10A26000884203D9FFE701980090FFE79DF81600A8
:10A27000C00728B9FFE701980099401A0090FFE74E
:10A2800021E09DF80B0001280FD1FFE70398C1687A
:10A29000012010FA81F0019003989DF8161000EB50
:10A2A0008100806B80B200900CE00398C06880B29F
:10A2B000019003989DF8161000EB8100806B80B22E
:10A2C0000090FFE7FFE70098C0030199B0FBF1F0B1
:10A2D0000490FFE7FFE7BDF8100006B080BD00BFA7
:10A2E00080B584B08DF80F00ADF80C10FFE79DF835
:10A2F0000F00042809D3FFE745F2FD60C0F2020019
:10A3000040F69911FEF788F833E0BDF80C100020F4
:10A310003F29019007D8FFE7BDF80C00002818BFBF
:10A3200001200190FFE70198C00748B9FFE745F217
:10A33000FD60C0F2020040F69A11FEF76DF818E0D9
:10A340009DF80F1045F29440C0F2020050F8210031
:10A350000290F6F7D7FDBDF80C200299486E02F086
:10A360003F0220F47C0040EA82404866F6F7CEFDCA
:10A37000FFE704B080BD00BF80B586B08DF8170040
:10A380000491FFE79DF81700042809D3FFE745F281
:10A39000FD60C0F2020040F6B711FEF73DF81CE088
:10A3A0009DF8171045F2A440C0F2020050F82100B9
:10A3B0000390F6F777FD04986FF35F200190039800
:10A3C000806D02900199029840EA01400290029843
:10A3D00003998865F6F76AFDFFE706B080BD00BF08
:10A3E00080B586B08DF817000491FFE79DF817003F
:10A3F000042809D3FFE745F2FD60C0F2020040F6F1
:10A40000D911FEF709F81CE09DF8171045F2A44099
:10A41000C0F2020050F821000390F6F743FD0498C3
:10A420006FF35F2001900398806D0290019902986C
:10A4300020EA01400290029803998865F6F736FDFC
:10A44000FFE706B080BD00BF80B582B08DF8070081
:10A450009DF8071045F29440C0F2020050F8210028
:10A460000090F6F73FFD0099486F40F48070486710
:10A47000F6F73CFD02B080BD80B584B08DF80F00CA
:10A4800002919DF80F1045F2A440C0F2020050F86E
:10A4900021000190F6F70EFD9DF808000290029A47
:10A4A0000199086990430861F6F708FD04B080BD82
:10A4B00080B584B08DF80F0002919DF80F1045F221
:10A4C000A440C0F2020050F821000190F6F7F2FC1F
:10A4D0009DF808000290029A0199086910430861EA
:10A4E000F6F7ECFC04B080BD80B584B08DF80F00A9
:10A4F0008DF80E10FFE79DF80F00042809D3FFE741
:10A5000045F2FD60C0F2020040F63321FDF784FF02
:10A5100070E09DF80F1045F29440C0F2020050F830
:10A52000210002909DF80E00012841D1FFE7002094
:10A530008DF80700FFE79DF80700072824D8FFE7FC
:10A540009DF80F1040F6DC30C2F2000000EBC100B5
:10A550009DF80710405C8DF806009DF80F009DF8EF
:10A560000710022200F048F89DF80F009DF8071030
:10A570009DF806200123FEF731FDFFE79DF8070057
:10A5800001308DF80700D6E7F6F7A4FC02990868B9
:10A5900020F003000860F6F7A1FCF6F7E3FC02994F
:10A5A00048684FF6FF7290434860F6F7DFFC20E002
:10A5B000F6F790FC9DF80F1040F62440C2F2000020
:10A5C000425C0299086802F0070220F01C0040EA91
:10A5D000820008609DF80F1040F62840C2F200008B
:10A5E000425C0299086862F301000860F6F776FCA5
:10A5F000FFE7FFE704B080BD80B582B08DF80700AB
:10A600008DF806108DF80520F6F7A4FC9DF807C01C
:10A6100040F6BC31C2F2000101EBCC009DF80630DF
:10A62000C05C40F62C42C2F2000202EBCC02D054D5
:10A630009DF805009DF8072001EBC2019DF806205A
:10A640008854F6F78BFC02B080BD00BF81B08DF856
:10A6500003008DF802109DF8031040F69C30C2F202
:10A66000000000EBC1009DF80210405C01B0704793
:10A6700081B08DF803008DF802109DF8031040F6AC
:10A68000BC30C2F2000000EBC1009DF80210405C3B
:10A6900001B0704781B08DF803008DF802109DF86D
:10A6A000033040F62C40C2F2000000EBC3009DF8DE
:10A6B0000220805C40F6BC31C2F2000101EBC30114
:10A6C000885401B0704700BF81B08DF803008DF849
:10A6D00002109DF8031040F63C30C2F2000000EB7F
:10A6E000C1009DF80210405C01B0704781B08DF848
:10A6F00003009DF8031040F6FC30C2F2000030F871
:10A70000110001B0704700BF80B584B08DF80F0014
:10A710009DF80F1045F29440C0F2020050F821005D
:10A7200002900299086F40F4802008670299086F30
:10A7300040F400200867029800210122019200F0F5
:10A7400017F8019A0298114600F012F8019A02983F
:10A75000022100F00DF8019A0298032100F008F898
:10A760000299086F40F00100086704B080BD00BF87
:10A7700083B002908DF807108DF806209DF8070031
:10A7800001460091032834D80099DFE801F0020E59
:10A790001A269DF806200299086E02F0010220F0A8
:10A7A000080040EAC200086624E09DF806200299ED
:10A7B000086E02F0010220F4006040EAC220086640
:10A7C00018E09DF806200299086E02F0010220F4BC
:10A7D000002040EAC24008660CE09DF8062002997D
:10A7E000086E02F0010220F0006040EAC2600866D4
:10A7F00000E0FFE703B0704780B582B08DF8070036
:10A800009DF8071045F29440C0F2020050F8210074
:10A810000090F6F76FFB0099086F40F001000867A1
:10A82000F6F76CFB02B080BD81B08DF803008DF8A7
:10A8300002108DF801209DF801009DF8032040F6DC
:10A84000DC31C2F2000101EBC2019DF80220885404
:10A8500001B0704781B08DF803008DF802109DF8AB
:10A86000031040F6DC30C2F2000000EBC1009DF89E
:10A870000210405C01B0704780B584B08DF80F00C5
:10A880009DF80F1045F29440C0F2020050F82100EC
:10A89000029002980069C0F340208DF807000298EA
:10A8A0004069C0F340208DF806009DF8070000289D
:10A8B00051D0FFE79DF8060000284CD0FFE7029931
:10A8C000486920F40070486100208DF80500FFE71A
:10A8D0009DF8050007283DD8FFE79DF80F1040F6CA
:10A8E0003C30C2F2000000EBC1009DF80510405C56
:10A8F0008DF804009DF804008007002823D5FFE7A9
:10A900009DF80400400700281DD4FFE79DF80F10B4
:10A9100040F64C40C2F2000000EB41109DF80510DB
:10A9200050F8210070B1FFE79DF80F1040F64C4041
:10A93000C2F2000000EB41109DF8051050F8210014
:10A940008047FFE7FFE7FFE79DF8050001308DF83E
:10A950000500BDE7FFE704B080BD00BF80B586B04D
:10A960008DF817009DF8171045F29440C0F20200D0
:10A9700050F82100049000208DF80D00FFE79DF8AD
:10A980000D00072800F2B380FFE704989DF80D1032
:10A9900000EB81008069C0F300108DF80F0004986F
:10A9A0009DF80D1000EB81008069C0F340108DF818
:10A9B0000E009DF80F00002800F09280FFE79DF840
:10A9C0000E00002800F08C80FFE704989DF80D1021
:10A9D00000EB8101886920F0200088619DF8171044
:10A9E00040F63C30C2F2000000EBC1009DF80D10B3
:10A9F000405C00F001008DF80C009DF80C00E8B1FF
:10AA0000FFE79DF8171040F6CC40C2F2000000EBC3
:10AA100041109DF80D1050F8210070B1FFE79DF82E
:10AA2000171040F6CC40C2F2000000EB41109DF838
:10AA30000D1050F821008047FFE7FFE79DF8171041
:10AA400040F69C30C2F2000000EBC1009DF80D10F2
:10AA5000405C032843D1FFE79DF80D00C00728B9EB
:10AA6000FFE79DF80D000130019004E09DF80D0016
:10AA700001380190FFE701988DF80B009DF8171041
:10AA800040F63C30C2F2000000EBC1009DF80D1012
:10AA9000405C00F008008DF80C009DF80C00E8B157
:10AAA000FFE79DF8171040F6CC40C2F2000000EB23
:10AAB00041109DF80B1050F8210070B1FFE79DF890
:10AAC000171040F6CC40C2F2000000EB41109DF898
:10AAD0000B1050F821008047FFE7FFE7FFE7FFE793
:10AAE000FFE79DF80D0001308DF80D0047E706B037
:10AAF00080BD00BF83B08DF80B0001919DF80B1055
:10AB000045F29440C0F2020050F8210000900198F4
:10AB100002790099086902F0010220F4806040EA9D
:10AB20008220086101980079012815D1FFE701987A
:10AB300040889DF80B2040F6FC31C2F2000121F85C
:10AB40001200019842880099C8684FF6FF73984335
:10AB500040EA5200C86012E0019840889DF80B203E
:10AB600040F6FC31C2F2000121F812000198408841
:10AB700001380099CA68C0EA0200C860FFE701987E
:10AB800042790099486E02F0030220F4403040EA16
:10AB9000024048660198C2880099486E02F03F0260
:10ABA00020F47C0040EA824048660198027A0099CD
:10ABB000886D02F0010220F0807040EA0260886532
:10ABC0000099086920F40070086103B0704700BF65
:10ABD00081B08DF803009DF80300012805D0FFE740
:10ABE0009DF80300022804D1FFE702208DF802003F
:10ABF00003E001208DF80200FFE79DF8020001B09C
:10AC0000704700BF83B002908DF807108DF80620C2
:10AC10009DF8070001460091072866D80099DFE8F3
:10AC200001F004101C2834404C589DF8062002996D
:10AC3000886D02F0010220F4807040EA02208865ED
:10AC400054E09DF806200299886D02F0010220F47C
:10AC5000007040EA4220886548E09DF8062002998D
:10AC6000886D02F0010220F4806040EA822088654D
:10AC70003CE09DF806200299886D02F0010220F464
:10AC8000006040EAC220886530E09DF80620029905
:10AC9000886D02F0010220F4805040EA023088659D
:10ACA00024E09DF806200299886D02F0010220F44C
:10ACB000005040EA4230886518E09DF8062002996D
:10ACC000886D02F0010220F4804040EA82308865FD
:10ACD0000CE09DF806200299886D02F0010220F434
:10ACE000004040EAC230886500E0FFE703B07047EB
:10ACF00083B002908DF807108DF806209DF80700AC
:10AD000001460091072866D80099DFE801F0041099
:10AD10001C2834404C589DF806200299886D02F09A
:10AD2000010220F4803040EA0240886554E09DF83A
:10AD300006200299886D02F0010220F4003040EAFA
:10AD40004240886548E09DF806200299886D02F02F
:10AD5000010220F4802040EA824088653CE09DF8B2
:10AD600006200299886D02F0010220F4002040EADA
:10AD7000C240886530E09DF806200299886D02F097
:10AD8000010220F4801040EA0250886524E09DF81A
:10AD900006200299886D02F0010220F4001040EABA
:10ADA0004250886518E09DF806200299886D02F0EF
:10ADB000010220F4800040EA825088650CE09DF892
:10ADC00006200299886D02F0010220F4000040EA9A
:10ADD000C250886500E0FFE703B0704780B584B0DB
:10ADE0008DF80F008DF80E108DF80D209DF80F10C6
:10ADF00045F29440C0F2020050F8210002909DF804
:10AE00000D0001460191012808D0FFE701980228B2
:10AE10000CD0FFE70198032810D017E002989DF8A6
:10AE20000E104908002200F099F810E002989DF8F1
:10AE30000E104908002200F091F808E002989DF8F1
:10AE40000E104908012200F089F800E0FFE79DF8A4
:10AE50000D009DF80F2040F69C31C2F2000101EB7D
:10AE6000C2019DF80E20885404B080BD83B00290CA
:10AE70008DF807108DF806209DF807000146009117
:10AE8000032834D80099DFE801F0020E1A269DF855
:10AE900006200299086E02F0010220F0020040EA4A
:10AEA0004200086624E09DF806200299086E02F030
:10AEB000010220F4007040EA4220086618E09DF884
:10AEC00006200299086E02F0010220F4003040EAE8
:10AED000424008660CE09DF806200299086E02F0D8
:10AEE000010220F0007040EA4260086600E0FFE7DF
:10AEF00003B0704784B003908DF80B109DF80B00E1
:10AF000040088DF80A00002001909DF80A000146D3
:10AF1000009103281CD80099DFE801F002080E1404
:10AF20000398006EC0F38000019012E00398006E59
:10AF3000C0F3802001900CE00398006EC0F38040C5
:10AF4000019006E00398006EC0F38060019000E07D
:10AF5000FFE79DF8040004B0704700BF83B0029083
:10AF60008DF807108DF806209DF807000146009126
:10AF7000032834D80099DFE801F0020E1A269DF864
:10AF800006200299086E02F0010220F0040040EA57
:10AF90008200086624E09DF806200299086E02F0FF
:10AFA000010220F4806040EA8220086618E09DF8E3
:10AFB00006200299086E02F0010220F4802040EA87
:10AFC000824008660CE09DF806200299086E02F0A7
:10AFD000010220F0806040EA8260086600E0FFE73E
:10AFE00003B0704780B582B08DF807008DF8061069
:10AFF000F5F750FF9DF8071040F63C30C2F2000014
:10B0000000EBC1009DF80610405C800700280FD5BA
:10B01000FFE79DF8071040F63C30C2F2000000EB5D
:10B02000C1019DF80620885C40F004008854FFE7C9
:10B03000F5F734FF9DF807009DF80610FEF766F857
:10B0400002B080BD80B584B08DF80F008DF80E1071
:10B050009DF80F1045F29440C0F2020050F8210014
:10B0600002909DF80F1040F69C30C2F2000000EBF9
:10B07000C1009DF80E10405C8DF807009DF80E0091
:10B08000C00730B9FFE79DF80E0001308DF80600CB
:10B0900005E09DF80E0001388DF80600FFE7F5F792
:10B0A000F9FE9DF80F1040F63C30C2F2000000EBB4
:10B0B000C1009DF80E10405C800700281AD5FFE7FC
:10B0C0009DF80F1040F63C30C2F2000000EBC101C9
:10B0D0009DF80E20885C00F0FB008854F5F7DEFE3A
:10B0E000F5F7E8FE0299086940F400700861F5F789
:10B0F000E5FE02E0F5F7D2FEFFE7F5F70BFF9DF85E
:10B100000F1040F63C30C2F2000000EBC1009DF889
:10B110000E10405CC00750B1FFE702989DF80E107A
:10B1200000EB8101886940F010008861FFE79DF81D
:10B130000700032823D1FFE702989DF8061000EBD3
:10B140008101886920F0200088619DF80F1040F689
:10B150003C30C2F2000000EBC1009DF80610405CDC
:10B16000000700280AD5FFE702989DF8061000EBBB
:10B170008101886940F010008861FFE7FFE7F5F77B
:10B18000CDFE04B080BD00BF83B002908DF80710E3
:10B1900000208DF806009DF8070001460091032865
:10B1A00020D80099DFE801F0020910170298006E1C
:10B1B000C0F380008DF8060015E00298006EC0F321
:10B1C00080208DF806000EE00298006EC0F38040EB
:10B1D0008DF8060007E00298006EC0F380608DF8DD
:10B1E000060000E0FFE79DF8060003B0704700008E
:10B1F00080B586B08DF81700049100200090FFE71D
:10B200009DF81700022809D3FFE745F22A70C0F223
:10B21000020040F60F1100F067F862E0049848B9A8
:10B22000FFE745F22A70C0F202004FF4116100F00E
:10B230005BF856E09DF8171045F2B440C0F20200EA
:10B2400050F8210002909DF8171045F2BC40C0F262
:10B25000020050F82100039004988078A8BBFFE713
:10B2600000208DF80700FFE79DF807000499097991
:10B27000884224DAFFE7049880689DF8071050F8A8
:10B280002100007800F10C01012000FA01F3029A7C
:10B29000916B99439163049989689DF8072051F84F
:10B2A000221009780C3100FA01F10098084300904F
:10B2B000FFE79DF8070001308DF80700D4E7009AFA
:10B2C0000299486B104348630AE00299886B20F4A6
:10B2D000805088630399486B40F000404863FFE763
:10B2E000FFE706B080BD00BF82B001900091FFE78C
:10B2F000FEE700BF80B584B08DF80F000291FFE734
:10B300009DF80F00022809D3FFE745F22A70C0F22A
:10B31000020040F6A511FFF7E7FFB4E0029848B934
:10B32000FFE745F22A70C0F2020040F6A611FFF7CF
:10B33000DBFFA8E0029800688078002843D1FFE78F
:10B3400000208DF80700FFE79DF807000299097AB1
:10B35000884237DAFFE7029840689DF8071050F8F6
:10B36000210000900098807A01280AD0FFE7009819
:10B37000807A032805D0FFE70098807A06280DD14F
:10B38000FFE79DF80F1040F66C50C2F2000000EB92
:10B39000C10100980278002088540CE09DF80F103D
:10B3A00040F66C50C2F2000000EBC1010098027838
:10B3B00001208854FFE7FFE79DF8070001308DF872
:10B3C0000700C1E73CE000208DF80700FFE79DF88B
:10B3D00007000299097A884231DAFFE7029840684B
:10B3E0009DF8071050F8210000900098807A0128FD
:10B3F0000AD0FFE70098807A032805D0FFE700987D
:10B40000807A06280AD1FFE79DF80F2040F66C519C
:10B41000C2F20001002001F8320009E09DF80F207F
:10B4200040F66C51C2F20001012001F83200FFE742
:10B43000FFE79DF8070001308DF80700C7E7FFE739
:10B440009DF80F000299096800F020F800208DF89F
:10B450000700FFE79DF807000299097A884211DA90
:10B46000FFE79DF80F00029949689DF8072051F801
:10B47000221000F093F8FFE79DF8070001308DF8E7
:10B480000700E7E7FFE704B080BD00BF80B584B0E8
:10B490008DF80F000291FFE79DF80F00022809D3F5
:10B4A000FFE745F22A70C0F2020040F6DE01FFF726
:10B4B0001BFF70E0029848B9FFE745F22A70C0F21E
:10B4C000020040F6DF01FFF70FFF64E09DF80F0078
:10B4D000029903F09BF90298807828BBFFE70020CF
:10B4E000ADF80600FFE7BDF8060002990979884229
:10B4F00019DAFFE702988068BDF8061050F821209D
:10B5000050889DF80F3040F6DC51C2F2000101EB8B
:10B51000C301127821F81200FFE7BDF806000130E0
:10B52000ADF80600DFE723E00020ADF80600FFE7F6
:10B53000BDF8060003281AD8FFE702988268106851
:10B5400040889DF80F3040F6DC51C2F2000101EB5B
:10B55000C301BDF8063052F82320127821F81200FA
:10B56000FFE7BDF806000130ADF80600E0E7FFE7B1
:10B57000029800789DF80F2040F61C61C2F200018D
:10B580008854029840789DF80F2040F61E61C2F260
:10B5900000018854FFE704B080BD00BF80B586B0CD
:10B5A0008DF817000491FFE79DF81700022809D3D2
:10B5B000FFE745F22A70C0F2020040F68601FFF76D
:10B5C00093FE38E1049848B9FFE745F22A70C0F2CB
:10B5D000020040F68701FFF787FE2CE19DF8171067
:10B5E00045F2B440C0F2020050F8210002909DF8EC
:10B5F000171045F2BC40C0F2020050F82100019043
:10B60000049800788DF80F009DF80F0040088DF821
:10B610000E009DF80E008DF80D009DF8171040F6F5
:10B620008C50C2F2000000EB01119DF80F200020A9
:10B6300021F812000498407A9DF8172040F6D06156
:10B64000C2F2000101EBC2019DF80F20885401985D
:10B650009DF80F10049A527A03F0F4F90498C07A16
:10B660009DF8172040F6FC51C2F20001009101EB59
:10B6700002119DF80F2021F8120001989DF80F107B
:10B680009DF8173040F63062C2F2000202EBC302AE
:10B69000525C03F049FA01989DF80F1000EB81010C
:10B6A000C86B20F00100C86301989DF80F10049A40
:10B6B000127B03F0AFFA9DF817009DF80F10049A63
:10B6C000927A03F02BFB009801999DF80F2001EB73
:10B6D0008202D16D4FF6FF731943D1659DF81710A3
:10B6E00000EB01109DF80F1030F81120019800EBCD
:10B6F0008101D1F8100162F30400C1F810019DF836
:10B700000F00C00730BBFFE70498006908B3FFE7EC
:10B7100001989DF80D10049A1269127803F0D2FB7B
:10B7200001989DF80F1003F019FC012810D1FFE7D4
:10B730000498006940889DF8172040F6EC51C2F249
:10B74000000101EBC2019DF80D2021F81200FFE776
:10B75000FFE7FFE70498427B01989DF80F1000EB8C
:10B760008101C86B02F0010220F0400040EA821023
:10B77000C86301989DF80F109DF8173040F6CC5221
:10B78000C2F2000202EBC302525C00F065FA9DF8BF
:10B79000171040F6BC50C2F2000000EBC1019DF84A
:10B7A0000F200120885401989DF80F1000EB8101B3
:10B7B000C86B20F01000C863049840689DF81720FB
:10B7C00040F68061C2F2000101EB42119DF80F20AA
:10B7D00041F82200049840689DF8172040F6406127
:10B7E000C2F2000101EB42119DF80F2041F8220046
:10B7F0000498007A01280AD1FFE79DF80F10012074
:10B8000000FA01F20299486B1043486309E09DF881
:10B810000F10012000FA01F20299486B904348632F
:10B82000FFE701989DF80F1000EB8101C86B20F035
:10B830002000C863FFE706B080BD00BF85B08DF86B
:10B8400013009DF8131045F2B440C0F2020050F806
:10B85000210003900399486B20F4704048630399DA
:10B86000002001900860039A516BC9B2516303999B
:10B87000896B03998863039AD16F01F47F41D16783
:10B880000399D1F880100399C1F880000399C1F899
:10B8900084000399C1F888000399C1F88C000399CA
:10B8A000C1F890000399C1F894000399C1F8980079
:10B8B0000399C1F89C000399C1F8A0000399C1F84D
:10B8C000A4008DF80B00FFE79DF80B00032869D852
:10B8D000FFE703989DF80B1000EB8101002000901A
:10B8E000486003999DF80B2001EB820148610399A0
:10B8F0009DF80B2001EB8201486203999DF80B2013
:10B9000001EBC201C96B03999DF80B2001EBC20149
:10B91000C86303999DF80B2001EBC201096C0399E0
:10B920009DF80B2001EBC201086403999DF80B20E0
:10B9300001EBC201C86503999DF80B2001EBC20120
:10B94000086603999DF80B2001EB8201C1F8000104
:10B9500003999DF80B2001EBC201C1F81001039976
:10B960009DF80B2001EBC201C1F814019DF81320D2
:10B9700040F67C51C2F2000101EBC2029DF80B308F
:10B9800002F813009DF8132001EBC2019DF80B2073
:10B9900001EB42014870FFE79DF80B0001308DF884
:10B9A0000B0091E705B0704780B586B08DF81700A1
:10B9B0008DF81610ADF814208DF813309DF817107F
:10B9C00045F2BC40C0F2020050F821000390002074
:10B9D000ADF80A009DF8160040088DF80900BDF882
:10B9E00014009DF8172040F68C51C2F2000101EBC3
:10B9F00002119DF8162021F812009DF8171040F64C
:10BA0000AC50C2F2000000EBC1009DF81610405C83
:10BA10008DF808009DF817009DF8161000F0E0F86A
:10BA2000F5F728FA9DF8171040F6BC50C2F2000056
:10BA300000EBC1009DF81610405C022823D1FFE7FF
:10BA40009DF8171040F6BC50C2F2000000EBC10197
:10BA50009DF8162001208854F5F710FA03989DF8F8
:10BA600016109DF8173040F6CC52C2F2000202EBDD
:10BA7000C302525C00F0F0F803989DF81610002203
:10BA800000F076F902E0F5F7F9F9FFE79DF8080014
:10BA9000012805D0FFE79DF8080003280FD1FFE734
:10BAA0009DF817009DF81610BDF814309DF813206E
:10BAB000EC46CCF800201A4600F0E2F98EE09DF842
:10BAC0000800022805D0FFE79DF80800042810D1DF
:10BAD000FFE79DF817009DF81610BDF814205308D5
:10BAE0009DF81320EC46CCF800201A4600F0C8F967
:10BAF00073E09DF8080006286DD1FFE7BDF814003B
:10BB0000C8B9FFE79DF817009DF8161040F6DC5203
:10BB1000C2F2000202EBC0029DF8093032F8132095
:10BB200001329DF81330EC46CCF8003093B200227D
:10BB300000F0A6F94EE0BDF814009DF8172040F67D
:10BB4000DC51C2F2000101EBC2019DF8092031F87D
:10BB5000121088420FD1FFE79DF817009DF81610CC
:10BB6000BDF814209DF81330EC46CCF800300023CB
:10BB700000F086F92DE09DF8171040F6DC50C2F277
:10BB8000000000EBC1009DF8093030F8130040F6CA
:10BB9000EC52C2F2000202EBC10131F8131008446A
:10BBA000BDF81410401AADF80A009DF817009DF872
:10BBB000161002EBC0029DF8093032F81320BDF8D0
:10BBC0000A309DF813C0EE46CEF800C000F058F9D8
:10BBD000FFE7FFE700E0FFE7FFE7FFE706B080BD14
:10BBE00080B582B08DF807008DF806109DF807101B
:10BBF00040F68C50C2F2000000EB01109DF80610D8
:10BC000030F81100C0B1FFE79DF8073040F6DC5076
:10BC1000C2F2000000EBC3009DF8062002F0FE0116
:10BC2000405A40F68C51C2F2000101EB031131F889
:10BC30001210884207D1FFE79DF807009DF8061013
:10BC400003F0AAFA06E09DF807009DF8061003F03D
:10BC5000D3FAFFE702B080BD80B584B003908DF8C1
:10BC60000B108DF80A20F5F7C5F89DF80B0001467A
:10BC70000191072800F277800199DFE801F00412B2
:10BC8000202E3C4A58669DF80A200399D1F884007A
:10BC900002F0010220F4807040EA0220C1F8840022
:10BCA00062E09DF80A200399D1F8840002F00102B5
:10BCB00020F4007040EA4220C1F8840054E09DF86E
:10BCC0000A200399D1F8840002F0010220F4806078
:10BCD00040EA8220C1F8840046E09DF80A200399DA
:10BCE000D1F8840002F0010220F4006040EAC22092
:10BCF000C1F8840038E09DF80A200399D1F8840047
:10BD000002F0010220F4805040EA0230C1F88400C1
:10BD10002AE09DF80A200399D1F8840002F001027C
:10BD200020F4005040EA4230C1F884001CE09DF845
:10BD30000A200399D1F8840002F0010220F4804027
:10BD400040EA8230C1F884000EE09DF80A20039991
:10BD5000D1F8840002F0010220F4004040EAC23031
:10BD6000C1F8840000E0FFE7F5F748F804B080BDB3
:10BD700080B584B003908DF80B108DF80A20F5F78C
:10BD800039F89DF80B0001460191072800F27380F5
:10BD90000199DFE801F0040E1C2A384654629DF830
:10BDA0000A200399D1F8840062F30000C1F88400EE
:10BDB00062E09DF80A200399D1F8840002F00102A4
:10BDC00020F0020040EA4200C1F8840054E09DF8EF
:10BDD0000A200399D1F8840002F0010220F0040047
:10BDE00040EA8200C1F8840046E09DF80A200399E9
:10BDF000D1F8840002F0010220F0080040EAC200FD
:10BE0000C1F8840038E09DF80A200399D1F8840035
:10BE100002F0010220F0100040EA0210C1F8840094
:10BE20002AE09DF80A200399D1F8840002F001026B
:10BE300020F0200040EA4210C1F884001CE09DF888
:10BE40000A200399D1F8840002F0010220F040009A
:10BE500040EA8210C1F884000EE09DF80A200399A0
:10BE6000D1F8840002F0010220F0800040EAC21004
:10BE7000C1F8840000E0FFE7F4F7C0FF04B080BD24
:10BE800080B586B0844608988DF817C08DF81610D6
:10BE9000ADF81420ADF812308DF8110000208DF8A7
:10BEA0000B009DF8160040088DF80A00FFE79DF88A
:10BEB0001700022809D3FFE745F22A70C0F20200FA
:10BEC00040F6AF31FFF710FAABE09DF816000828F6
:10BED00009D3FFE745F22A70C0F202004FF43B613C
:10BEE000FFF702FA9DE09DF8171045F2BC40C0F242
:10BEF000020050F82100039003989DF80A1001F009
:10BF000003FF012858D1FFE7F4F794FFBDF8142090
:10BF100003989DF80A1000EBC101C86D4FF6FF733E
:10BF200098431044C865BDF8122003989DF80A1084
:10BF300000EBC101086E6FF30F00104408669DF816
:10BF4000171040F6FC50C2F2000000EB01119DF802
:10BF50000A2031F82230039901EBC202D2F8101105
:10BF600063F30401C2F810119DF8171000EB0110E3
:10BF70009DF80A104900013130F81120039800EBB8
:10BF80008101D1F8100162F30400C1F81001F4F747
:10BF900055FF03989DF80A104900C9B2002201928A
:10BFA000FFF7E6FE019A03989DF80A104900013157
:10BFB000C9B2FFF7DDFE2CE0F4F73CFFBDF814201A
:10BFC00003989DF8161000EB8101C86D4FF6FF73C2
:10BFD00098431044C8659DF8171040F6FC50C2F213
:10BFE000000000EB01109DF8161030F811200398A6
:10BFF00000EB8101D1F8100162F30400C1F81001D7
:10C00000F4F71CFF03989DF816100022FFF7B0FE0E
:10C01000FFE703989DF80A109DF8112001F010FC2D
:10C02000FFE79DF80B0006B080BD00BF80B584B06F
:10C03000844606988DF80FC08DF80E10ADF80C20D0
:10C04000ADF80A308DF809000020ADF802009DF827
:10C050000E0040088DF80100FFE79DF80F00022850
:10C0600009D3FFE745F22A70C0F2020040F66D21C5
:10C07000FFF73AF980E09DF80E00082809D3FFE7A2
:10C0800045F22A70C0F2020040F66E21FFF72CF94B
:10C0900072E09DF80F1045F2BC40C0F2020050F86B
:10C0A00021000190F4F7E6FE9DF80F1040F6BC5019
:10C0B000C2F2000000EBC1009DF80E10405C0228A7
:10C0C00023D1FFE79DF80F1040F6BC50C2F20000EC
:10C0D00000EBC1019DF80E2001208854F4F7CEFE3C
:10C0E00001989DF80E109DF80F3040F6CC52C2F228
:10C0F000000202EBC302525CFFF7AEFD01989DF80F
:10C100000E100022FFF734FE02E0F4F7B7FEFFE75F
:10C11000BDF80C0020B9FFE70020ADF8020020E0D8
:10C12000BDF80A00ADF802000198416B0120B0EBA8
:10C13000D17F0AD1FFE79DF80F00BDF80C209DF8D4
:10C140000930002100F01AF80AE09DF80F009DF870
:10C150000110BDF80C209DF8093000F00FF8FFE742
:10C16000FFE79DF80F009DF80E10BDF802209DF826
:10C170000930FFF719FCFFE704B080BD80B586B039
:10C180008DF817008DF8161004928DF80F30FFE728
:10C190009DF81700022809D3FFE745F22A70C0F284
:10C1A000020040F66C11FFF79FF864E09DF817104D
:10C1B00045F2BC40C0F2020050F821000290029803
:10C1C000416B0120B0EBD17F1FD1FFE700208DF83C
:10C1D000070004989DF8172040F6DC51C2F20001D8
:10C1E00021F8320004989DF8172001EBC20250801C
:10C1F00004989DF8172001EBC202908004989DF8E6
:10C20000172001EBC201C88011E09DF816008DF8DF
:10C21000070004989DF8172040F6DC51C2F2000197
:10C2200001EBC2019DF8162021F81200FFE70298E9
:10C230009DF8071001F06CFA01280AD1FFE79DF87C
:10C2400017009DF80710049AC2F34F0201F09EFAFE
:10C2500009E09DF817009DF80710049A013A92B280
:10C2600001F094FAFFE702989DF807109DF80F205F
:10C2700001F0E6FAFFE706B080BD00BF80B582B0EE
:10C280008DF807008DF806108DF805208DF8043024
:10C29000FFE79DF80700022809D3FFE745F22A705F
:10C2A000C0F2020040F6AB21FFF71EF882E09DF8D5
:10C2B0000600082809D3FFE745F22A70C0F2020001
:10C2C00040F6AC21FFF710F874E09DF8071045F236
:10C2D000BC40C0F2020050F8210000909DF8071009
:10C2E00040F6BC50C2F2000000EBC1009DF8061001
:10C2F000405C022836D1FFE79DF8071040F68C50CD
:10C30000C2F2000000EB01119DF80620002021F888
:10C310001200F4F757FD9DF8071040F67C50C2F26A
:10C32000000000EBC1009DF80610405C800700286B
:10C330000FD5FFE79DF8071040F67C50C2F20000D1
:10C3400000EBC1019DF80620885C40F00400885491
:10C35000FFE7F4F73BFD9DF807009DF8061000F09D
:10C360002BF818E09DF8071040F6BC50C2F2000010
:10C3700000EBC1009DF80610405C032809D1FFE7DF
:10C380009DF807009DF806109DF8042000F0C2F803
:10C3900000E0FFE7FFE700989DF806109DF80520F4
:10C3A000FFF75AFC00989DF806109DF80420FFF74F
:10C3B000DFFCFFE702B080BD80B584B08DF80F00D0
:10C3C0008DF80E109DF80F1045F2BC40C0F202002F
:10C3D00050F82100029000208DF806009DF80E0014
:10C3E00040088DF80400F4F70DFD9DF80F1040F69D
:10C3F0007C50C2F2000000EBC1009DF80E10405CC2
:10C4000000F009008DF807009DF8070050B9FFE71C
:10C4100002989DF80E1000EB8101C86B20F010000F
:10C42000C863FFE702989DF80E1000EB8101C86B0E
:10C4300020F02000C863F4F7E9FC0298416B01206A
:10C44000B0EBD17F28D1FFE700208DF80500FFE792
:10C450009DF8050007281EDCFFE79DF80F1040F649
:10C460007C50C2F2000000EBC1009DF80510405C5A
:10C4700000F002008DF807009DF8070020B1FFE7EB
:10C4800001208DF8060006E0FFE79DF80500013069
:10C490008DF80500DCE728E09DF80F1040F67C5091
:10C4A000C2F2000000EBC1019DF8042011F8121047
:10C4B00001F002018DF807109DF80F1000EBC1008C
:10C4C0009DF8041000EB4100407800F002019DF857
:10C4D000070008438DF807009DF8070020B1FFE72B
:10C4E00001208DF80600FFE7FFE79DF8060040B940
:10C4F000FFE79DF80F009DF80E10002202F036FABB
:10C50000FFE79DF80F009DF8041000F0DDFC04B07B
:10C5100080BD00BF80B582B08DF807008DF8061091
:10C520008DF805209DF8071045F2BC40C0F20200CE
:10C5300050F8210000909DF80500012807D1FFE781
:10C540009DF807009DF80610FFF736FF34E09DF8D0
:10C55000071040F67C50C2F2000000EBC1009DF8CD
:10C560000610405C8007002808D5FFE79DF807000B
:10C570009DF80610012202F0F9F9FFE79DF8071077
:10C5800040F67C50C2F2000000EBC1009DF806109E
:10C59000405C10F0090F0ED0FFE7F4F733FC009871
:10C5A0009DF8061000EB8101C86B40F01000C863D5
:10C5B000F4F72CFCFFE7FFE702B080BD80B584B044
:10C5C0008DF80F008DF80E1001208DF80400FFE7A4
:10C5D0009DF80F00022809D3FFE745F22A70C0F248
:10C5E000020040F6EB21FEF77FFE69E09DF80E00A9
:10C5F000082809D3FFE745F22A70C0F2020040F68E
:10C60000EC21FEF771FE5BE09DF80F1045F2BC4097
:10C61000C0F2020050F8210002900298416B012004
:10C62000B0EBD17F04D1FFE701208DF8070008E0CF
:10C6300002989DF80E10490800F046F88DF80700A2
:10C64000FFE79DF80700012831D1FFE702989DF828
:10C650000E1000F06DF88DF806009DF80600012818
:10C6600008D1FFE702989DF80E1000F0BBF88DF896
:10C67000040008E09DF80F009DF80E1000F00CF982
:10C680008DF80400FFE702989DF80E1000F00EFAF6
:10C690008DF805009DF80500012807D1FFE79DF8FA
:10C6A0000410012088438DF80400FFE707E002989A
:10C6B0009DF80E1000F04CFA8DF80400FFE7FFE73C
:10C6C0009DF8040004B080BD83B002908DF807107F
:10C6D00000208DF806009DF8070001460091032810
:10C6E00020D80099DFE801F0020910170298406B8A
:10C6F000C0F300308DF8060015E00298406BC0F3DF
:10C7000040308DF806000EE00298406BC0F3803098
:10C710008DF8060007E00298406BC0F3C0308DF83A
:10C72000060000E0FFE79DF8060003B0704700BF79
:10C7300083B002908DF8071000208DF806009DF858
:10C74000070001460091072846D80099DFE801F06C
:10C75000040C141C242C343C0298D0F8840000F003
:10C7600001008DF8060038E00298D0F88400C0F38C
:10C7700040008DF8060030E00298D0F88400C0F345
:10C7800080008DF8060028E00298D0F88400C0F3FD
:10C79000C0008DF8060020E00298D0F88400C0F3B5
:10C7A00000108DF8060018E00298D0F88400C0F35D
:10C7B00040108DF8060010E00298D0F88400C0F315
:10C7C00080108DF8060008E00298D0F88400C0F3CD
:10C7D000C0108DF8060000E0FFE79DF8060003B0EA
:10C7E000704700BF83B002908DF8071000208DF8CD
:10C7F00006009DF8070001460091072846D80099D9
:10C80000DFE801F0040C141C242C343C0298D0F80E
:10C810008400C0F300208DF8060038E00298D0F8BC
:10C820008400C0F340208DF8060030E00298D0F874
:10C830008400C0F380208DF8060028E00298D0F82C
:10C840008400C0F3C0208DF8060020E00298D0F8E4
:10C850008400C0F300308DF8060018E00298D0F88C
:10C860008400C0F340308DF8060010E00298D0F844
:10C870008400C0F380308DF8060008E00298D0F8FC
:10C880008400C0F3C0308DF8060000E0FFE79DF89B
:10C89000060003B0704700BF88B08DF81F008DF808
:10C8A0001E109DF81F1045F2BC40C0F2020050F867
:10C8B000210006909DF81E0040088DF8160000200B
:10C8C000ADF81400ADF81200ADF810008DF80F00AF
:10C8D0009DF81F1040F6AC50C2F2000000EBC10002
:10C8E0009DF81E10405C8DF817000698416B0120E2
:10C8F000B0EBD17F05D1FFE706984068ADF8140092
:10C900000AE006989DF81E1001F0FE0100EB4100C0
:10C910004068ADF81400FFE79DF8170001380146A4
:10C920000291052800F2BC800299DFE801F00316AD
:10C93000294DB97106989DF81E1000EB8100C06D5D
:10C94000ADF81200BDF81410BDF81220002091427D
:10C95000B8BF01208DF80F00A3E006989DF81E10C7
:10C9600000EB8100C06DADF81200BDF81410BDF8E9
:10C97000122000209142B8BF01208DF80F0090E0F6
:10C9800006989DF8161000EBC100C06DADF81200BE
:10C990009DF81E00C00758B9FFE7BDF81410BDF898
:10C9A000122000209142B8BF01208DF80F000AE04C
:10C9B000BDF81410BDF8122000209142C8BF01201C
:10C9C0008DF80F00FFE76CE006989DF8161000EB5D
:10C9D000C100C06DADF812009DF81E00C00758B927
:10C9E000FFE7BDF81410BDF8122000209142B8BF37
:10C9F00001208DF80F000AE0BDF81410BDF81220D8
:10CA000000209142C8BF01208DF80F00FFE748E0E9
:10CA100006989DF8161000EBC100C06DADF812002D
:10CA200006989DF8161000EBC100006EADF81000DE
:10CA30009DF81E00C007C8B9FFE7BDF81410BDF887
:10CA400012200120914201900ADBFFE7BDF814108B
:10CA5000BDF8102000209142C8BF01200190FFE7DF
:10CA6000019800F001008DF80F0018E0BDF81410D7
:10CA7000BDF812200020914200900ADBFFE7BDF8CC
:10CA80001410BDF8102000209142D8BF0120009062
:10CA9000FFE7009800F001008DF80F00FFE700E0CD
:10CAA000FFE79DF80F0008B0704700BF83B0029009
:10CAB0008DF8071000208DF806009DF8070001464C
:10CAC000009107283ED80099DFE801F0040B121905
:10CAD00020272E350298C06F00F001008DF8060067
:10CAE00031E00298C06FC0F340008DF806002AE0E4
:10CAF0000298C06FC0F380008DF8060023E0029812
:10CB0000C06FC0F3C0008DF806001CE00298C06F33
:10CB1000C0F300108DF8060015E00298C06FC0F356
:10CB200040108DF806000EE00298C06FC0F3801030
:10CB30008DF8060007E00298C06FC0F3C0108DF8B2
:10CB4000060000E0FFE79DF8060003B0704700BF55
:10CB500083B002908DF8071000208DF806009DF834
:10CB600007000146009107283ED80099DFE801F050
:10CB7000040B121920272E350298C06FC0F3002035
:10CB80008DF8060031E00298C06FC0F340208DF8A8
:10CB900006002AE00298C06FC0F380208DF80600DE
:10CBA00023E00298C06FC0F3C0208DF806001CE09F
:10CBB0000298C06FC0F300308DF8060015E00298AF
:10CBC000C06FC0F340308DF806000EE00298C06FD1
:10CBD000C0F380308DF8060007E00298C06FC0F304
:10CBE000C0308DF8060000E0FFE79DF8060003B0B6
:10CBF000704700BF80B582B08DF807008DF8061031
:10CC0000FFE79DF80700022809D3FFE745F22A70E5
:10CC1000C0F2020040F62831FEF766FB6DE09DF899
:10CC20000600082809D3FFE745F22A70C0F2020087
:10CC300040F62931FEF758FB5FE09DF80600C0077B
:10CC400030B9FFE79DF8060001308DF8050005E0DA
:10CC50009DF8060001388DF80500FFE79DF80710E4
:10CC600040F6AC50C2F2000000EBC1009DF8061087
:10CC7000405C8DF804009DF80400062829D1FFE7E8
:10CC8000F4F7A0F89DF8071040F67C50C2F20000BF
:10CC900000EBC1029DF80630D15C01F00801D154CF
:10CCA0009DF8071000EBC1019DF80520885C00F09D
:10CCB000F7008854F4F78AF89DF807009DF80610ED
:10CCC000FFF77AFB9DF807009DF80510FFF774FB4E
:10CCD00012E09DF8071040F67C50C2F2000000EB15
:10CCE000C1019DF80620002088549DF807009DF89A
:10CCF0000610FFF761FBFFE7FFE702B080BD00BF52
:10CD000080B584B08DF80F008DF80E108DF80D20D1
:10CD1000FFE79DF80F00022809D3FFE745F22A70CC
:10CD2000C0F2020040F65D31FEF7DEFAC9E09DF880
:10CD30000E00082809D3FFE745F22A70C0F202006E
:10CD400040F65E31FEF7D0FABBE09DF80F1045F2D9
:10CD5000BC40C0F2020050F821000290F4F732F813
:10CD60009DF80F1040F67C50C2F2000000EBC101AC
:10CD70009DF80E20885C00F0FC008854F4F726F83B
:10CD8000F4F740F802989DF80E1000EB8101C86B93
:10CD900020F02000C863F4F739F89DF80F009DF8E3
:10CDA0000E1000F091F89DF80F1040F6AC50C2F252
:10CDB000000000EBC1009DF80E10405C8DF80700EC
:10CDC0009DF80700012809D1FFE79DF80F009DF8A5
:10CDD0000E109DF80D2000F0BBF82BE09DF8070029
:10CDE000032809D1FFE79DF80F009DF80E109DF86C
:10CDF0000D2000F033F91CE09DF80700022805D053
:10CE0000FFE79DF80700042809D1FFE79DF80F0010
:10CE10009DF80E109DF80D2000F012FA08E09DF824
:10CE20000F009DF80E109DF80D2000F02DFAFFE781
:10CE3000FFE7FFE79DF80F1040F68C50C2F20000AC
:10CE400000EB01109DF80E1030F81100F8B1FFE76B
:10CE50009DF80F3040F6DC50C2F2000000EBC3003A
:10CE60009DF80E2002F0FE01405A40F68C51C2F2AD
:10CE7000000101EB031131F81210884207D0FFE7DF
:10CE80009DF80F009DF80E1000F09EFA18E0F3F7E1
:10CE900099FF9DF80F1040F67C50C2F2000000EBA5
:10CEA000C1019DF80E20885C40F004008854F3F71F
:10CEB0008DFF9DF80F009DF80E10FFF77DFAFFE73C
:10CEC000FFE704B080BD00BF80B584B08DF80F00CF
:10CED0008DF80E109DF80F1045F2BC40C0F2020014
:10CEE00050F8210002900298416B0120B0EBD17FF5
:10CEF00004D1FFE700208DF80E00FFE7F3F78AFF6B
:10CF00009DF80E000146019103281CD80199DFE825
:10CF100001F002080E140299886B20F48050886397
:10CF200012E00299886B20F4005088630CE00299AB
:10CF3000886B20F48040886306E00299886B20F4B7
:10CF40000040886300E0FFE7F3F768FF04B080BDAE
:10CF500080B582B08DF807008DF806108DF8052099
:10CF6000F3F730FF9DF8050001460091B8B1FFE7E7
:10CF7000009801283FD0FFE70098022868D1FFE71A
:10CF80009DF8071040F67C50C2F2000000EBC10192
:10CF90009DF80620885C40F00300885459E09DF815
:10CFA000071040F6D060C2F2000000EBC1009DF80F
:10CFB0000610405C78B9FFE79DF8071040F67C50FA
:10CFC000C2F2000000EBC1019DF80620885C40F031
:10CFD000020088540EE09DF8071040F67C50C2F223
:10CFE000000000EBC1019DF80620885C40F00100C4
:10CFF0008854FFE72DE09DF8071040F6D060C2F29C
:10D00000000000EBC1009DF80610405C01280FD124
:10D01000FFE79DF8071040F67C50C2F2000000EBDD
:10D02000C1019DF80620885C40F0020088540EE0A3
:10D030009DF8071040F67C50C2F2000000EBC101E1
:10D040009DF80620885C40F001008854FFE700E06E
:10D05000FFE7F3F7BBFE02B080BD00BF80B582B032
:10D060008DF807008DF806108DF805209DF8061044
:10D07000012088438DF80400F3F7A4FE9DF8050015
:10D0800001460091C0B1FFE70098012873D0FFE787
:10D090000098022840F0CE80FFE79DF8071040F688
:10D0A0007C50C2F2000000EBC1019DF80620885CB4
:10D0B00040F003008854BEE09DF8040001282CD104
:10D0C000FFE79DF8071040F6D060C2F2000000EBC9
:10D0D000C1009DF80610405C78B9FFE79DF8071085
:10D0E00040F67C50C2F2000000EBC1019DF8062022
:10D0F000885C40F0020088540EE09DF8071040F66E
:10D100007C50C2F2000000EBC1019DF80620885C53
:10D1100040F001008854FFE72CE09DF8071040F62E
:10D12000D060C2F2000000EBC1009DF80610405C28
:10D1300001280FD1FFE79DF8071040F67C50C2F29E
:10D14000000000EBC1019DF80620885C40F0020061
:10D1500088540EE09DF8071040F67C50C2F20000A3
:10D1600000EBC1019DF80620885C40F00100885466
:10D17000FFE7FFE75FE09DF8040001282DD1FFE7FE
:10D180009DF8071040F6D060C2F2000000EBC1002D
:10D190009DF80610405C01280FD1FFE79DF80710AD
:10D1A00040F67C50C2F2000000EBC1019DF8062061
:10D1B000885C40F0020088540EE09DF8071040F6AD
:10D1C0007C50C2F2000000EBC1019DF80620885C93
:10D1D00040F001008854FFE72BE09DF8071040F66F
:10D1E000D060C2F2000000EBC1009DF80610405C68
:10D1F00078B9FFE79DF8071040F67C50C2F20000B6
:10D2000000EBC1019DF80620885C40F002008854C4
:10D210000EE09DF8071040F67C50C2F2000000EBD3
:10D22000C1019DF80620885C40F001008854FFE7AA
:10D23000FFE700E0FFE7F3F7C9FD02B080BD00BFE4
:10D2400080B582B08DF807008DF806108DF80520A6
:10D25000F3F7B8FD9DF8050002280FD1FFE79DF810
:10D26000071040F67C50C2F2000000EBC1019DF8AF
:10D270000620885C40F00100885400E0FFE7F3F7E7
:10D28000A5FD02B080BD00BF80B582B08DF807005B
:10D290008DF806108DF805209DF80600C00730B9FE
:10D2A000FFE79DF8060001308DF8040005E09DF8C9
:10D2B000060001388DF80400FFE7F3F783FD9DF8C1
:10D2C00005000146009108B3FFE7009801284AD005
:10D2D000FFE70098022872D1FFE79DF8071040F69B
:10D2E0007C50C2F2000000EBC1029DF80630D15C18
:10D2F00041F00101D1549DF8071000EBC1019DF8E8
:10D300000420885C40F00800885459E09DF807101C
:10D3100040F6D060C2F2000000EBC1009DF806109C
:10D32000405C01280FD1FFE79DF8071040F67C50C4
:10D33000C2F2000000EBC1019DF80620885C40F0BD
:10D34000010088540EE09DF8071040F67C50C2F2B0
:10D35000000000EBC1019DF80420885C40F008004B
:10D360008854FFE72CE09DF8071040F6D060C2F229
:10D37000000000EBC1009DF80610405C78B9FFE7A3
:10D380009DF8071040F67C50C2F2000000EBC1018E
:10D390009DF80620885C40F0010088540EE09DF85E
:10D3A000071040F67C50C2F2000000EBC1019DF86E
:10D3B0000420885C40F008008854FFE700E0FFE7A5
:10D3C000F3F704FD02B080BD80B584B08DF80F0086
:10D3D0008DF80E109DF80F1045F2BC40C0F202000F
:10D3E00050F8210002909DF80F1040F6AC50C2F2A8
:10D3F000000000EBC1009DF80E10405C8DF80700A6
:10D400009DF80E00C00730B9FFE79DF80E0001300F
:10D410008DF8060005E09DF80E0001388DF8060035
:10D42000FFE79DF80F1040F67C50C2F2000000EBC1
:10D43000C1009DF80E10405C8007002808D5FFE76A
:10D440009DF80F009DF80E10012201F08FFAFFE702
:10D45000F3F7D8FC9DF80F1040F67C50C2F20000A4
:10D4600000EBC1009DF80E10405CC00750B1FFE713
:10D4700002989DF80E1000EB8101C86B40F010007F
:10D48000C863FFE79DF80700062823D1FFE702984D
:10D490009DF8061000EB8101C86B20F02000C863E6
:10D4A0009DF80F1040F67C50C2F2000000EBC10066
:10D4B0009DF80610405C000700280AD5FFE7029897
:10D4C0009DF8061000EB8101C86B40F01000C863A6
:10D4D000FFE7FFE7F3F79AFC04B080BD80B586B0A4
:10D4E000844608988DF817C08DF81610ADF81420F2
:10D4F000ADF812308DF811000020ADF804000120C5
:10D500008DF803008DF80200FFE79DF81700022850
:10D5100009D3FFE745F22A70C0F2020040F6F1316C
:10D52000FDF7E2FEF2E09DF81600082809D3FFE7B8
:10D5300045F22A70C0F2020040F6F231FDF7D4FE47
:10D54000E4E09DF8171040F6AC50C2F2000000EB8A
:10D55000C1009DF81610405C8DF807009DF807008B
:10D56000062804D0FFE700208DF80300FFE79DF8B0
:10D57000030048B9FFE745F22A70C0F2020040F606
:10D58000FB31FDF7B1FEC1E0BDF81200BDF814108B
:10D5900000EB5100ADF80400BDF80400BDF8121016
:10D5A000884207DDFFE7BDF81400BDF8041088428B
:10D5B00004DCFFE700208DF80200FFE79DF8020081
:10D5C00048B9FFE745F22A70C0F2020040F6034175
:10D5D000FDF78AFE9AE09DF8160040088DF81000CD
:10D5E0009DF8171045F2BC40C0F2020050F821002F
:10D5F0000290BDF814009DF8172040F6DC51C2F2ED
:10D60000000101EBC2019DF8102021F812000298E0
:10D610009DF8101000F07CF801280AD1FFE79DF872
:10D6200017009DF81010BDF81420520800F0AEF855
:10D630000AE09DF817009DF81010BDF81420013A7B
:10D6400092B200F0A3F8FFE7BDF814004008ADF86F
:10D650000E00BDF80E009DF8172040F68C51C2F266
:10D66000000101EB02119DF8162021F81200F3F7DA
:10D67000E1FBBDF8122002989DF8101000EBC101EB
:10D68000C86D4FF6FF7398431044C865BDF812008B
:10D69000BDF80E10084402999DF8102001EBC2015C
:10D6A0000A6EC0EA020008669DF8171040F6FC50AA
:10D6B000C2F2000000EB01119DF8102031F8223079
:10D6C000029901EBC202D2F8101163F30401C2F80F
:10D6D00010119DF8171000EB01109DF81010490073
:10D6E000013130F81120029800EB8101D1F81001CE
:10D6F00062F30400C1F81001F3F7A0FB02989DF853
:10D7000010109DF8112000F09BF8FFE706B080BDD7
:10D7100083B002908DF8071000208DF80600029863
:10D72000416B0120B0EBD17F04D1FFE700208DF8E1
:10D730000700FFE79DF8070001460091032820D865
:10D740000099DFE801F0020910170298406BC0F35E
:10D7500000208DF8060015E00298406BC0F34020D1
:10D760008DF806000EE00298406BC0F380208DF823
:10D77000060007E00298406BC0F3C0208DF8060059
:10D7800000E0FFE79DF8060003B0704780B582B067
:10D790008DF807008DF80610ADF804209DF80710ED
:10D7A00045F2BC40C0F2020050F821000090F3F7AF
:10D7B00039FB0098416B0120B0EBD17F19D1FFE715
:10D7C000BDF80420009948694FF6FF739843104450
:10D7D00048619DF8071040F6C060C2F2000030F8C2
:10D7E00031200099D1F8000162F30400C1F8000172
:10D7F00022E0BDF8042000989DF8061000EB81019E
:10D8000048694FF6FF739843104448619DF807102C
:10D8100040F6C060C2F2000000EBC1009DF80610A7
:10D8200030F81120009800EB8101D1F8000162F37B
:10D830000400C1F80001FFE7F3F7F8FA02B080BD79
:10D8400080B584B003908DF80B108DF80A20F3F7A3
:10D85000F9FA9DF80B000146019103283CD8019983
:10D86000DFE801F002101E2C9DF80A200399D1F880
:10D87000A00002F0010220F4807040EA0220C1F80A
:10D88000A0002AE09DF80A200399D1F8A00002F038
:10D89000010220F4007040EA4220C1F8A0001CE020
:10D8A0009DF80A200399D1F8A00002F0010220F4AB
:10D8B000806040EA8220C1F8A0000EE09DF80A20B6
:10D8C0000399D1F8A00002F0010220F4006040EAC0
:10D8D000C220C1F8A00000E0FFE7F3F7B7FA04B0F8
:10D8E00080BD00BF80B586B0844608988DF817C00B
:10D8F0008DF81610ADF81420ADF812308DF8110027
:10D900000020ADF80E00ADF80C009DF81610490887
:10D910008DF80B10ADF8080001208DF807008DF888
:10D920000600FFE79DF81700022809D3FFE745F23C
:10D930002A70C0F2020040F64441FDF7D5FC0BE12D
:10D940009DF81600082809D3FFE745F22A70C0F2B7
:10D95000020040F64541FDF7C7FCFDE09DF81710B9
:10D9600040F6AC50C2F2000000EBC1009DF816106A
:10D97000405C8DF80A009DF80A00062804D0FFE7F5
:10D9800000208DF80700FFE79DF8070048B9FFE782
:10D9900045F22A70C0F2020040F64E41FDF7A4FCA9
:10D9A000DAE09DF8171040F6DC50C2F2000000EB00
:10D9B000C1009DF80B1030F81100BDF8141088421A
:10D9C00035D0FFE7BDF8140088B3FFE7BDF81200BB
:10D9D0009DF8172040F6DC51C2F2000101EBC201B4
:10D9E0009DF80B2031F812100844BDF81410401AAD
:10D9F000ADF80800BDF80800BDF81210884211DD2E
:10DA0000FFE79DF8171040F6DC50C2F2000000EB73
:10DA1000C1009DF80B1030F81100BDF808108842C5
:10DA200004DCFFE700208DF80600FFE7FFE79DF824
:10DA3000060048B9FFE745F22A70C0F2020040F63E
:10DA40005841FDF751FC87E0BDF812009DF8172002
:10DA500040F6EC51C2F2000101EBC2019DF80B202F
:10DA600021F81200BDF814009DF8172040F68C51E3
:10DA7000C2F2000101EB02119DF8162021F81200FC
:10DA8000BDF8120020B9FFE70120ADF80E0004E058
:10DA9000BDF81200ADF80E00FFE79DF8171040F634
:10DAA000DC50C2F2000000EBC1009DF80B1030F812
:10DAB0001100BDF8141088420FD1FFE79DF8171030
:10DAC00040F6EC50C2F2000000EBC1009DF80B10D4
:10DAD00030F81100ADF80C002EE0BDF8140078B954
:10DAE000FFE79DF8171040F6DC50C2F2000000EB93
:10DAF000C1009DF80B1030F81100ADF80C001AE0D1
:10DB00009DF8173040F6EC50C2F2000000EBC30065
:10DB10009DF80B2030F8120040F6DC51C2F20001F3
:10DB200001EBC30131F812100844BDF81410401A7B
:10DB3000ADF80C00FFE7FFE79DF817009DF8161001
:10DB4000BDF80E20BDF80C309DF811C0EE46CEF8A1
:10DB500000C0FEF795F9FFE706B080BD80B586B03E
:10DB60008DF817008DF8161000200490FFE79DF83F
:10DB70001700022809D3FFE745F22A70C0F202001D
:10DB800040F68B41FDF7B0FBBAE09DF8160008287F
:10DB900009D3FFE745F22A70C0F2020040F68C413B
:10DBA000FDF7A2FBACE09DF8171045F2BC40C0F2B7
:10DBB000020050F8210003909DF8171040F6AC5079
:10DBC000C2F2000000EBC1009DF81610405C8DF819
:10DBD0000B009DF8160040088DF80A0003989DF888
:10DBE0001610FEF7A5FD002840F08980FFE7039896
:10DBF000416B0120B0EBD17F04D1FFE700208DF80D
:10DC0000090004E09DF80A008DF80900FFE7039879
:10DC10009DF80A10FFF77CFD012809D1FFE7039862
:10DC20009DF8091000EB8100406980B201900AE084
:10DC300003989DF8091000EB81004169012010FA5A
:10DC400081F00190FFE79DF80B00062834D1FFE733
:10DC500003989DF80A1000EBC100006E80B200909E
:10DC6000009803999DF80A2001EBC201C96D89B2A1
:10DC700088420BD9FFE7009803999DF80A2001EB31
:10DC8000C201C96D89B2401A009002E000200090E4
:10DC9000FFE700980199884203D9FFE701980090B7
:10DCA000FFE79DF81600C00728B9FFE70198009923
:10DCB000401A0090FFE71BE003989DF8161000EB58
:10DCC0008100C06D80B2009003989DF8091000F0AB
:10DCD0001BF801280BD1FFE79DF81600C00728B1FB
:10DCE000FFE701980099401A0090FFE7FFE7FFE780
:10DCF0000098C0030199B0FBF1F00490FFE7FFE743
:10DD0000BDF8100006B080BD83B002908DF80710FA
:10DD100000208DF806009DF80700014600910328B9
:10DD200024D80099DFE801F0020A121A0298D0F80C
:10DD30008800C0F380108DF8060018E00298D0F833
:10DD40008800C0F380308DF8060010E00298D0F80B
:10DD50008800C0F380508DF8060008E00298D0F8E3
:10DD60008800C0F380708DF8060000E0FFE79DF8A2
:10DD7000060003B0704700BF80B584B08DF80F0077
:10DD80008DF80E10ADF80C20FFE79DF80F0002286B
:10DD900009D3FFE745F22A70C0F2020040F6E441E1
:10DDA000FDF7A2FA6BE09DF80E00082809D3FFE703
:10DDB00045F22A70C0F2020040F6E541FDF794FA00
:10DDC0005DE09DF80F1045F2BC40C0F2020050F833
:10DDD0002100019001989DF80E104908FFF794FF6B
:10DDE000012809D0FFE745F22A70C0F2020040F690
:10DDF000E741FDF779FA42E001989DF80E104908D5
:10DE000000F040F8012809D0FFE745F22A70C0F27F
:10DE1000020040F6E841FDF767FA30E0BDF80C205B
:10DE200000210846B1EB123F009007D1FFE7BDF893
:10DE30000C00002818BF01200090FFE70098C007E1
:10DE400048B9FFE745F22A70C0F2020040F6E94106
:10DE5000FDF74AFA13E09DF80F1045F2B440C0F206
:10DE6000020050F821000290BDF80C0002999DF8C4
:10DE70000E2002F0FE0201EB42014862FFE704B00F
:10DE800080BD00BF83B002908DF8071000208DF890
:10DE900006009DF8070001460091032824D8009948
:10DEA000DFE801F0020A121A0298D0F88800C0F3E5
:10DEB00040008DF8060018E00298D0F88800C0F302
:10DEC00040208DF8060010E00298D0F88800C0F3DA
:10DED00040408DF8060008E00298D0F88800C0F3B2
:10DEE00040608DF8060000E0FFE79DF8060003B0F3
:10DEF000704700BF80B584B08DF80F000291FFE736
:10DF00009DF80F00022809D3FFE745F22A70C0F2FE
:10DF1000020040F60451FDF7E7F919E09DF80F10F3
:10DF200045F2B440C0F2020050F821000190F2F72F
:10DF300051FF0198D0F880000090029900980843A2
:10DF4000009000980199C1F88000F2F747FFFFE7C1
:10DF500004B080BD80B584B08DF80F000291FFE75A
:10DF60009DF80F00022809D3FFE745F22A70C0F29E
:10DF7000020040F62451FDF7B7F919E09DF80F10A3
:10DF800045F2B440C0F2020050F821000190F2F7CF
:10DF900021FF0198D0F880000090029900988843F2
:10DFA000009000980199C1F88000F2F717FFFFE791
:10DFB00004B080BD80B582B08DF807009DF80710D1
:10DFC00045F2B440C0F2020050F821000090F2F790
:10DFD00039FF0099D1F8A00040F47060C1F8A000AA
:10DFE000F2F734FF02B080BD80B584B08DF80F0029
:10DFF00002919DF80F1045F2B440C0F2020050F8B3
:10E0000021000190F2F7EEFE9DF808000290029ABE
:10E010000199486B90434863F2F7E8FE04B080BD75
:10E0200080B584B08DF80F0002919DF80F1045F275
:10E03000B440C0F2020050F821000190F2F7D2FE85
:10E040009DF808000290029A0199486B10434863BA
:10E05000F2F7CCFE04B080BD80B582B08DF8070029
:10E060008DF80610FFE79DF80700022809D3FFE7A7
:10E0700045F22A70C0F2020040F67D51FDF734F9F6
:10E0800052E09DF8071045F2BC40C0F2020050F883
:10E09000210000909DF80600012823D1FFE7F2F748
:10E0A000E1FE0099086820F003000860F2F7DEFE48
:10E0B000F2F7E8FE009948684FF6FF729043486017
:10E0C000009988686FF30F0088600099C8686FF343
:10E0D0000F00C860009908696FF30F000861F2F73C
:10E0E000D5FE20E0F2F7BEFE9DF8071040F61C605A
:10E0F000C2F20000425C0099086862F30100086007
:10E100009DF8071040F61E60C2F20000425C0099C4
:10E11000086802F0070220F01C0040EA8200086054
:10E12000F2F7A4FEFFE7FFE702B080BD81B08DF8F3
:10E1300003008DF802109DF8031040F6AC50C2F2B7
:10E14000000000EBC1009DF80210405C01B0704778
:10E1500081B08DF803008DF802109DF8031040F691
:10E16000BC50C2F2000000EBC1009DF80210405C00
:10E1700001B0704780B582B08DF807008DF80610A9
:10E180008DF80520F2F776FE9DF807C040F6BC51E9
:10E19000C2F2000101EBCC009DF80630C05C40F6F5
:10E1A0002062C2F2000202EBCC02D0549DF80500BE
:10E1B0009DF8072001EBC2019DF806208854F2F774
:10E1C0005DFE02B080BD00BF81B08DF803008DF808
:10E1D00002109DF8033040F62060C2F2000000EB10
:10E1E000C3009DF80220805C40F6BC51C2F20001E1
:10E1F00001EBC301885401B0704700BF81B08DF8B6
:10E2000003008DF802109DF8031040F67C50C2F216
:10E21000000000EBC1009DF80210405C01B07047A7
:10E2200081B08DF803008DF802109DF8031040F6C0
:10E23000DC50C2F2000000EBC1009DF8021001F0BA
:10E24000FE01405A01B0704780B584B08DF80F00D0
:10E250009DF80F1045F2BC40C0F2020050F82100BA
:10E2600002900299D1F89C0040F00400C1F89C0093
:10E270000299D1F89C0040F00800C1F89C00029877
:10E2800000210122019200F019F8019A029811462A
:10E2900000F014F8019A0298022100F00FF8019A98
:10E2A0000298032100F00AF80299D1F89C0040F08E
:10E2B0000100C1F89C0004B080BD00BF83B0029093
:10E2C0008DF807108DF806209DF807000146009193
:10E2D00003283CD80099DFE801F002101E2C9DF8BD
:10E2E00006200299D1F8880002F0010220F0040013
:10E2F00040EA8200C1F888002AE09DF806200299D1
:10E30000D1F8880002F0010220F4806040EA822007
:10E31000C1F888001CE09DF806200299D1F8880019
:10E3200002F0010220F4802040EA8240C1F8880017
:10E330000EE09DF806200299D1F8880002F0010253
:10E3400020F0806040EA8260C1F8880000E0FFE7CA
:10E3500003B0704780B582B08DF807009DF80710B4
:10E3600045F2BC40C0F2020050F821000090F2F7E4
:10E3700071FD0099D1F89C0040F00100C1F89C00AB
:10E38000F2F76CFD02B080BD81B08DF803008DF80E
:10E3900002108DF801209DF801009DF8032040F641
:10E3A000CC51C2F2000101EBC2019DF80220885459
:10E3B00001B0704781B08DF803008DF802108DF820
:10E3C00001209DF801009DF8032040F63061C2F263
:10E3D000000101EBC2019DF80220885401B0704792
:10E3E00081B08DF803008DF802109DF8031040F6FF
:10E3F000CC50C2F2000000EBC1009DF80210405C5E
:10E4000001B0704780B586B08DF817009DF81710E1
:10E4100045F2BC40C0F2020050F8210004909DF883
:10E42000171045F2B440C0F2020050F821000390EA
:10E430000498416B0120B0EBD17F63D1FFE70398D3
:10E44000406BC0F300508DF80B000398806BC0F355
:10E4500000308DF80A009DF80B00002851D0FFE72E
:10E460009DF80A0000284CD0FFE70399886B20F440
:10E470008050886300208DF80800FFE79DF80800B1
:10E4800007283DD8FFE79DF8171040F67C50C2F2F0
:10E49000000000EBC1009DF80810405C8DF80700FB
:10E4A0009DF807008007002823D5FFE79DF80700A7
:10E4B000400700281DD4FFE79DF8171040F6406084
:10E4C000C2F2000000EB41109DF8081050F8210046
:10E4D00070B1FFE79DF8171040F64060C2F20000EF
:10E4E00000EB41109DF8081050F821008047FFE72D
:10E4F000FFE7FFE79DF8080001308DF80800BDE751
:10E50000FFE7B4E000208DF80900FFE79DF809005F
:10E51000032800F2AB80FFE70398406B9DF80910D9
:10E520001431C84000F001008DF80B000398806B97
:10E530009DF809100C31C84000F001008DF80A0068
:10E540009DF80B00002800F08A80FFE79DF80A0084
:10E55000002800F08480FFE79DF8090000F10C011D
:10E56000012000FA01F20399886B904388639DF8BB
:10E57000090040008DF808009DF8171040F67C5007
:10E58000C2F2000000EBC1009DF80810405C8DF85D
:10E5900007009DF807008007002823D5FFE79DF8B6
:10E5A0000700400700281DD4FFE79DF8171040F62C
:10E5B0004060C2F2000000EB41109DF8081050F8D6
:10E5C000210070B1FFE79DF8171040F64060C2F2DD
:10E5D000000000EB41109DF8081050F82100804722
:10E5E000FFE7FFE79DF80900400001308DF80800C3
:10E5F0009DF8171040F67C50C2F2000000EBC100FD
:10E600009DF80810405C8DF807009DF80700800712
:10E61000002823D5FFE79DF80700400700281DD4F8
:10E62000FFE79DF8171040F64060C2F2000000EBD3
:10E6300041109DF8081050F8210070B1FFE79DF8D7
:10E64000171040F64060C2F2000000EB41109DF848
:10E65000081050F821008047FFE7FFE7FFE7FFE7DA
:10E660009DF8090001308DF809004FE7FFE706B07B
:10E6700080BD00BF80B586B08DF817009DF81710DB
:10E6800045F2BC40C0F2020050F821000490002086
:10E690008DF80D00FFE79DF80D00072800F2B3800C
:10E6A000FFE704989DF80D1000EB8100C06BC0F3EC
:10E6B00000108DF80F0004989DF80D1000EB8100FC
:10E6C000C06BC0F340108DF80E009DF80F000028BD
:10E6D00000F09280FFE79DF80E00002800F08C808B
:10E6E000FFE704989DF80D1000EB8101C86B20F046
:10E6F0002000C8639DF8171040F67C50C2F200005D
:10E7000000EBC1009DF80D10405C00F001008DF899
:10E710000C009DF80C00E8B1FFE79DF8171040F6DB
:10E720008060C2F2000000EB41109DF80D1050F81F
:10E73000210070B1FFE79DF8171040F68060C2F22B
:10E74000000000EB41109DF80D1050F821008047AB
:10E75000FFE7FFE79DF8171040F6AC50C2F200004B
:10E7600000EBC1009DF80D10405C062843D1FFE787
:10E770009DF80D00C00728B9FFE79DF80D00013096
:10E78000019004E09DF80D0001380190FFE7019829
:10E790008DF80B009DF8171040F67C50C2F2000077
:10E7A00000EBC1009DF80D10405C00F008008DF8F2
:10E7B0000C009DF80C00E8B1FFE79DF8171040F63B
:10E7C0008060C2F2000000EB41109DF80B1050F881
:10E7D000210070B1FFE79DF8171040F68060C2F28B
:10E7E000000000EB41109DF80B1050F8210080470D
:10E7F000FFE7FFE7FFE7FFE7FFE79DF80D000130C8
:10E800008DF80D0047E706B080BD00BF80B584B02D
:10E810008DF80F0002919DF80F1045F2BC40C0F238
:10E82000020050F821000090029842780099086890
:10E8300002F0070220F01C0040EA82000860029803
:10E8400002780099086862F30100086002988078F5
:10E85000E8B9FFE700208DF80700FFE79DF8070003
:10E8600002990979884211DAFFE79DF80F000299B1
:10E8700089689DF8072051F8221000F025F8FFE77D
:10E880009DF8070001308DF80700E7E70CE09DF8E0
:10E890000F0002998968096800F016F80099486B22
:10E8A00040F000404863FFE70298C2780099D1F831
:10E8B000800002F0010220F4807040EA0220C1F8DA
:10E8C000800004B080BD00BF80B584B08DF80F001B
:10E8D00002919DF80F1045F2BC40C0F2020050F8C2
:10E8E00021000190029A90889DF80F3040F6C06197
:10E8F000C2F2000101EBC301127821F812009DF869
:10E900000F1040F66C50C2F2000000EBC1000299FB
:10E91000097810F81100012809D1FFE79DF80F00D0
:10E92000029A117852885208FEF730FF09E09DF8EC
:10E930000F00029A11785288013A92B2FEF726FF30
:10E94000FFE70299CA880198097800EB8101486ABB
:10E9500062F30B0048629DF80F00029909784900A4
:10E96000C9B2002200F002F804B080BD80B584B0C6
:10E970008DF80F008DF80E108DF80D209DF80F10FA
:10E9800045F2BC40C0F2020050F8210002909DF810
:10E990000E0040088DF80700F2F724FA0298416B48
:10E9A0000020B0EBD17F3DD1FFE79DF80700014685
:10E9B0000091032834D80099DFE801F0020E1A26EE
:10E9C0009DF80D200299486B02F0010220F480109E
:10E9D00040EA0250486324E09DF80D200299486BFC
:10E9E00002F0010220F4001040EA4250486318E0AF
:10E9F0009DF80D200299486B02F0010220F480007E
:10EA000040EA825048630CE09DF80D200299486B63
:10EA100002F0010220F4000040EAC250486300E026
:10EA2000FFE70BE09DF80D200299486B02F0010210
:10EA300020F4801040EA02504863FFE7F2F7D6F96D
:10EA400004B080BD83B002908DF807108DF80620C9
:10EA50009DF8070001460091072862D80099DFE879
:10EA600001F0040C1824303C48549DF8062002990B
:10EA7000C86F62F30000C86754E09DF80620029951
:10EA8000C86F02F0010220F0020040EA4200C867AD
:10EA900048E09DF806200299C86F02F0010220F0BC
:10EAA000040040EA8200C8673CE09DF80620029915
:10EAB000C86F02F0010220F0080040EAC200C867F7
:10EAC00030E09DF806200299C86F02F0010220F0A4
:10EAD000100040EA0210C86724E09DF80620029961
:10EAE000C86F02F0010220F0200040EA4210C8671F
:10EAF00018E09DF806200299C86F02F0010220F08C
:10EB0000400040EA8210C8670CE09DF80620029998
:10EB1000C86F02F0010220F0800040EAC210C8670E
:10EB200000E0FFE703B0704783B002908DF8071054
:10EB30008DF806209DF8070001460091072866D849
:10EB40000099DFE801F004101C2834404C589DF86F
:10EB500006200299C86F02F0010220F4807040EA9A
:10EB60000220C86754E09DF806200299C86F02F0A1
:10EB7000010220F4007040EA4220C86748E09DF896
:10EB800006200299C86F02F0010220F4806040EA7A
:10EB90008220C8673CE09DF806200299C86F02F009
:10EBA000010220F4006040EAC220C86730E09DF80E
:10EBB00006200299C86F02F0010220F4805040EA5A
:10EBC0000230C86724E09DF806200299C86F02F061
:10EBD000010220F4005040EA4230C86718E09DF876
:10EBE00006200299C86F02F0010220F4804040EA3A
:10EBF0008230C8670CE09DF806200299C86F02F0C9
:10EC0000010220F4004040EAC230C86700E0FFE79C
:10EC100003B0704783B002908DF807108DF806207E
:10EC20009DF8070001460091072800F273800099C3
:10EC3000DFE801F0040E1C2A384654629DF80620D5
:10EC40000299D1F8800062F30000C1F8800062E010
:10EC50009DF806200299D1F8800002F0010220F010
:10EC6000020040EA4200C1F8800054E09DF806200E
:10EC70000299D1F8800002F0010220F0040040EA7D
:10EC80008200C1F8800046E09DF806200299D1F884
:10EC9000800002F0010220F0080040EAC200C1F842
:10ECA000800038E09DF806200299D1F8800002F03B
:10ECB000010220F0100040EA0210C1F880002AE0B2
:10ECC0009DF806200299D1F8800002F0010220F0A0
:10ECD000200040EA4210C1F880001CE09DF80620A8
:10ECE0000299D1F8800002F0010220F0400040EAD1
:10ECF0008210C1F880000EE09DF806200299D1F83C
:10ED0000800002F0010220F0800040EAC210C1F849
:10ED1000800000E0FFE703B0704700BF80B588B017
:10ED20008DF81F008DF81E108DF81D209DF81F1006
:10ED300045F2BC40C0F2020050F8210006909DF858
:10ED40001F1045F2B440C0F2020050F821000590B7
:10ED50009DF81E0040088DF813000698416B0120B5
:10ED6000B0EBD17F04D1FFE700208DF8130000E065
:10ED7000FFE79DF81D00013801460391052800F2C8
:10ED800091800399DFE801F00316334B8E759DF8EF
:10ED9000130000F10801012000FA01F20599486B07
:10EDA0009043486306989DF81E104908002200F021
:10EDB0000FF978E09DF8130000F10801012000FA36
:10EDC00001F3059A516B194351639DF8131000FA32
:10EDD00001F20599D1F8A0001043C1F8A0000698EF
:10EDE0009DF81E104908002200F0F2F85BE09DF843
:10EDF00013000830012202FA00F30599486B98438A
:10EE0000486306989DF81E10490800F0E1F806983E
:10EE10009DF81E104908002200F026F943E09DF8F5
:10EE200013000830012202FA00F30599486B1843D9
:10EE300048639DF8130002FA00F30599D1F8A00089
:10EE40001843C1F8A00006989DF81E10490800F06C
:10EE5000BFF806989DF81E1049080022029200F0A3
:10EE600003F9029A06989DF81E10490800F048F927
:10EE700019E09DF8130008300122019202FA00F314
:10EE80000599486B9843486306989DF81E104908F9
:10EE900000F09EF8019A06989DF81E10490800F0AF
:10EEA000E3F800E0FFE79DF81D009DF81F2040F605
:10EEB000AC51C2F2000101EBC2019DF81E20885442
:10EEC00008B080BD83B002908DF807108DF8062041
:10EED0009DF807000146009103283CD80099DFE81F
:10EEE00001F002101E2C9DF806200299D1F888002E
:10EEF00002F0010220F0020040EA4200C1F888005E
:10EF00002AE09DF806200299D1F8880002F001025B
:10EF100020F4007040EA4220C1F888001CE09DF80F
:10EF200006200299D1F8880002F0010220F4003096
:10EF300040EA4240C1F888000EE09DF806200299A0
:10EF4000D1F8880002F0010220F0007040EA42602F
:10EF5000C1F8880000E0FFE703B0704784B0039079
:10EF60008DF80B109DF80B0040088DF80A0000206A
:10EF700001909DF80A0001460091032820D80099CD
:10EF8000DFE801F0020910170398D0F88800C0F3F9
:10EF90008010019015E00398D0F88800C0F380300D
:10EFA00001900EE00398D0F88800C0F380500190E3
:10EFB00007E00398D0F88800C0F38070019000E06B
:10EFC000FFE70198002818BF012004B0704700BF78
:10EFD00083B002908DF807108DF806209DF8070089
:10EFE0000146009103283CD80099DFE801F00210A7
:10EFF0001E2C9DF806200299D1F8880002F001022B
:10F0000020F0400040EA8210C1F888002AE09DF814
:10F0100006200299D1F8880002F0010220F4804015
:10F0200040EA8230C1F888001CE09DF80620029971
:10F03000D1F8880002F0010220F4800040EA8250FA
:10F04000C1F888000EE09DF806200299D1F88800EA
:10F0500002F0010220F0804040EA8270C1F888008E
:10F0600000E0FFE703B0704783B002908DF807100F
:10F070008DF806209DF807000146009103283CD832
:10F080000099DFE801F002101E2C9DF8062002997D
:10F09000D1F8880002F0010220F0200040EA42107E
:10F0A000C1F888002AE09DF806200299D1F888006E
:10F0B00002F0010220F4005040EA4230C1F888001A
:10F0C0001CE09DF806200299D1F8880002F00102A8
:10F0D00020F4001040EA4250C1F888000EE09DF88C
:10F0E00006200299D1F8880002F0010220F00050B9
:10F0F00040EA4270C1F8880000E0FFE703B07047C3
:10F1000083B002908DF807108DF806209DF8070057
:10F110000146009103283CD80099DFE801F0021075
:10F120001E2C9DF806200299D1F8880002F00102F9
:10F1300020F0080040EAC200C1F888002AE09DF8EB
:10F1400006200299D1F8880002F0010220F4006044
:10F1500040EAC220C1F888001CE09DF80620029910
:10F16000D1F8880002F0010220F4002040EAC240F9
:10F17000C1F888000EE09DF806200299D1F88800B9
:10F1800002F0010220F0006040EAC260C1F888008D
:10F1900000E0FFE703B0704780B582B08DF807004C
:10F1A0008DF80610F1F70EFE9DF8071040F67C5022
:10F1B000C2F2000000EBC1009DF80610405C800721
:10F1C00000280FD5FFE79DF8071040F67C50C2F2EB
:10F1D000000000EBC1019DF80620885C40F00400AF
:10F1E0008854FFE7F1F7F2FD9DF807009DF806103F
:10F1F000FDF7E2F802B080BD80B584B08DF80F0055
:10F200008DF80E109DF80F1045F2BC40C0F20200C0
:10F2100050F8210002909DF80F1040F6AC50C2F259
:10F22000000000EBC1009DF80E10405C8DF8070057
:10F230009DF80E00C00730B9FFE79DF80E000130C1
:10F240008DF8060005E09DF80E0001388DF80600E7
:10F25000FFE7F1F7B7FD9DF80F1040F67C50C2F2C2
:10F26000000000EBC1009DF80E10405C80070028F4
:10F2700018D5FFE79DF80F1040F67C50C2F2000051
:10F2800000EBC1019DF80E20885C00F0FB00885463
:10F29000F1F79CFD9DF80F009DF80E100122FFF77D
:10F2A00065FB02E0F1F792FDFFE7F1F7ABFD9DF89A
:10F2B0000F1040F67C50C2F2000000EBC1009DF838
:10F2C0000E10405CC00750B1FFE702989DF80E1089
:10F2D00000EB8101C86B40F01000C863FFE79DF8A8
:10F2E0000700062823D1FFE702989DF8061000EBDF
:10F2F0008101C86B20F02000C8639DF80F1040F614
:10F300007C50C2F2000000EBC1009DF80610405C8A
:10F31000000700280AD5FFE702989DF8061000EBC9
:10F320008101C86B40F01000C863FFE7FFE7F1F709
:10F330006DFD04B080BD000080B582B0019000205A
:10F340000090019800F01CF8012817D1FFE7009AFF
:10F3500043F2E470C0F2020050F8220040F6E0618F
:10F36000C2F2000141F82200009800F033F820B901
:10F37000FFE7009800F074F8FFE7FFE702B080BDF8
:10F3800080B584B00390002002908DF807000299A8
:10F3900040F6E460C2F20000405C38B1FFE75C2058
:10F3A00000220623114612F0BDF90EE0039838B191
:10F3B000FFE75C2000220923114612F0B3F903E0B5
:10F3C00001208DF80700FFE7FFE79DF8070004B074
:10F3D00080BD00BF80B582B0019000208DF8030091
:10F3E0008DF802008DF80200FFE79DF80200019AF7
:10F3F00040F6E061C2F2000151F8221089688842AB
:10F4000029D2FFE7019940F6E060C2F2000050F80F
:10F410002100C0699DF8021050F82100A0B1FFE75B
:10F420009DF8021040F6E560C2F20000405C50B169
:10F43000FFE75C2000220623114612F073F9012039
:10F440008DF8030007E0FFE7FFE79DF802000130B9
:10F450008DF80200C9E79DF8030002B080BD00BF2F
:10F4600080B584B0039000208DF80B0001218DF849
:10F470000A1001908DF80B00FFE79DF80B00039A2E
:10F4800040F6E061C2F2000151F82210896888421A
:10F490005AD2FFE7039940F6E060C2F2000050F84C
:10F4A0002100C0699DF80B1050F82100002844D0BD
:10F4B000FFE7039940F6E060C2F2000050F8210037
:10F4C000C0699DF80B1050F8210001900198C07898
:10F4D000012831D1FFE70198008B9DF80B2040F601
:10F4E000F261C2F2000121F812009DF80B2040F6F3
:10F4F000E861C2F20001002041F822009DF80B20D3
:10F5000040F6F061C2F2000188549DF80B00019AA8
:10F51000917801F0E9FD8DF80A009DF80A0048B9DC
:10F52000FFE79DF80B2040F6E561C2F200010220E2
:10F53000885400E008E0FFE7FFE7FFE79DF80B00D5
:10F5400001308DF80B0098E79DF80A00012830D1B2
:10F55000FFE700208DF80B00FFE79DF80B00039AF2
:10F5600040F6E061C2F2000151F822108968884239
:10F570001ED2FFE7039940F6E060C2F2000050F8A7
:10F580002100C0699DF80B1050F8210048B1FFE739
:10F590009DF80B2040F6E561C2F20001002088547E
:10F5A000FFE7FFE79DF80B0001308DF80B00D4E773
:10F5B00007E0039A40F6E461C2F20001012088549A
:10F5C000FFE704B080BD00BF80B584B000208DF897
:10F5D0000F000290019000F05BF8012855D1FFE781
:10F5E000029A40F6E461C2F20001002088548DF8CE
:10F5F0000F00FFE79DF80F00029A40F6E061C2F2AB
:10F60000000151F822108968884235D2FFE702993B
:10F6100040F6E060C2F2000050F82100C0699DF899
:10F620000F1050F8210000B3FFE7029940F6E060A8
:10F63000C2F2000050F82100C0699DF80F1050F888
:10F64000210001900198C07801280DD1FFE79DF8B5
:10F650000F2040F6E561C2F20001002088540198B5
:10F66000807803F073F8FFE7FFE7FFE79DF80F00EE
:10F6700001308DF80F00BDE7029A40F6E061C2F25A
:10F680000001002041F82200FFE704B080BD00BF68
:10F6900080B586B001208DF81700002004908DF809
:10F6A0000F00049940F6E460C2F20000405C0128BB
:10F6B0000BD0FFE75C20002202920623114612F0D5
:10F6C00031F802988DF817003CE000208DF80F000B
:10F6D000FFE79DF80F00049A40F6E061C2F20001D6
:10F6E00051F82210896888422BD2FFE7049940F62E
:10F6F000E060C2F2000050F82100C0699DF80F10D0
:10F7000050F82100B0B1FFE79DF80F1040F6E5601A
:10F71000C2F20000405C01280BD1FFE75C20002111
:10F7200001911022062311F0FDFF01988DF81700BA
:10F7300007E0FFE7FFE79DF80F0001308DF80F00AD
:10F74000C7E7FFE79DF8170006B080BD80B582B01F
:10F750008DF807008DF8061001208DF805000320B4
:10F7600000F01AF8012812D1FFE79DF807100320D6
:10F7700000F032F8012809D1FFE79DF807009DF855
:10F78000061000F051F88DF80500FFE7FFE79DF83F
:10F79000050002B080BD00BF80B582B08DF80700C3
:10F7A00000208DF806000090009940F6E460C2F257
:10F7B0000000405C40B9FFE79DF807205C20002175
:10F7C000052311F0AFFF03E001208DF80600FFE7ED
:10F7D0009DF8060002B080BD80B584B08DF80F00A2
:10F7E0008DF80E1001208DF80D00002002909DF87C
:10F7F0000E00029A40F6E061C2F2000151F82210B8
:10F80000896888420CD3FFE79DF80F205C20002117
:10F810000191042311F086FF01988DF80D00FFE798
:10F820009DF80D0004B080BD80B586B08DF817003E
:10F830008DF8161000200490039001208DF80B0025
:10F84000049940F6E060C2F2000050F82100C0695F
:10F850009DF8171050F8210003909DF816000146FE
:10F860000191012808D0FFE7019802282ED0FFE778
:10F870000198032831D037E09DF8171040F6E56075
:10F88000C2F20000405C022807D0FFE75C200021A4
:10F890000322062311F046FF17E0039908788978C0
:10F8A00001F05EFF80B9FFE79DF8172040F6E560A4
:10F8B000C2F200000121815403984078F0F768FDFE
:10F8C00000208DF80B00FFE7FFE714E09DF817001C
:10F8D00001F0CEFF8DF80B000DE09DF8170002F04F
:10F8E0001DF88DF80B0006E05C20002103220423A4
:10F8F00011F018FFFFE79DF80B0006B080BD00BFB8
:10F9000080B584B08DF80F00002002900190042093
:10F91000FFF742FF01282BD1FFE79DF80F100420CD
:10F92000FFF75AFF012822D1FFE7029940F6E06075
:10F93000C2F2000050F82100C0699DF80F1050F885
:10F9400021000190F1F7FEF89DF80F2040F6E861E4
:10F95000C2F2000151F82200013041F82200F1F713
:10F96000F5F801990878897800F004F8FFE7FFE7D7
:10F9700004B080BD80B582B08DF807008DF8061008
:10F980009DF8071040F6EC60C2F2000050F821002C
:10F9900000909DF8071040F6F460C2F20000405C51
:10F9A00001284FD1FFE79DF8060003F075FB009892
:10F9B000007B012807D1FFE79DF806000121002206
:10F9C00003F0E2FFFFE7009890F8360000070028F8
:10F9D00007D5FFE79DF806000A21002203F0D4FFB7
:10F9E000FFE7009890F836004007002807D5FFE7AA
:10F9F0009DF806000B21002203F0C6FFFFE70098E8
:10FA000090F83600C00738B1FFE79DF806000C21DA
:10FA1000002203F0B9FFFFE70098007A8007002872
:10FA200007D4FFE79DF806000022114603F0ACFF63
:10FA3000FFE79DF8072040F6F461C2F200010020C4
:10FA40008854FFE702B080BD80B584B08DF80F0008
:10FA50000020029001900520FFF79EFE012841D171
:10FA6000FFE79DF80F100520FFF7B6FE012838D1FB
:10FA7000FFE7029940F6E060C2F2000050F8210072
:10FA8000C0699DF80F1050F821000190F1F75AF865
:10FA90009DF80F1040F6E860C2F2000050F8210017
:10FAA00060B1FFE79DF80F2040F6E861C2F2000167
:10FAB00051F82200013841F82200FFE7F1F746F83B
:10FAC0009DF80F1040F6E860C2F2000050F82100E7
:10FAD00030B9FFE701990878897800F005F8FFE769
:10FAE000FFE7FFE704B080BD80B582B08DF8070066
:10FAF0008DF806109DF8071040F6EC60C2F2000089
:10FB000050F8210000909DF8071040F6F460C2F212
:10FB10000000405C00284FD1FFE79DF8060003F08D
:10FB20002FFA0098007B012807D1FFE79DF8060017
:10FB30000122114603F028FFFFE7009890F83600F5
:10FB40000007002807D5FFE79DF806000A210122DB
:10FB500003F01AFFFFE7009890F8360040070028EE
:10FB600007D5FFE79DF806000B21012203F00CFFEB
:10FB7000FFE7009890F83600C00738B1FFE79DF81E
:10FB800006000C21012203F0FFFEFFE70098007A37
:10FB90008007002807D4FFE79DF806000021012216
:10FBA00003F0F2FEFFE79DF8072040F6F461C2F291
:10FBB000000101208854FFE702B080BD80B586B007
:10FBC0008DF81700049101208DF80F00002002909D
:10FBD00001901120FFF7E0FD012828D1FFE79DF8F3
:10FBE00017101120FFF7F8FD01281FD1FFE7049837
:10FBF00000F022F8012818D1FFE7029940F6E060F2
:10FC0000C2F2000050F82100C0699DF8171050F8AA
:10FC10002100019001990878897800F025F804996D
:10FC2000087000208DF80F00FFE7FFE7FFE79DF861
:10FC30000F0006B080BD00BF80B584B003900120E6
:10FC40008DF80B00039858B9FFE75C200021019163
:10FC50001122012311F066FD01988DF80B00FFE7DA
:10FC60009DF80B0004B080BD80B586B08DF81700FC
:10FC70008DF8161000208DF815009DF8172040F61D
:10FC8000EC61C2F2000151F822100491029001903F
:10FC90009DF8160003F098FA02909DF8160003F004
:10FCA000BBFA01909DF8160003F066FA03900398E2
:10FCB00020B9FFE700208DF8150014E00398012813
:10FCC0000CD1FFE701208DF8150004984078BDF8AD
:10FCD0000810BDF80420F0F7E5FE03E002208DF8DF
:10FCE0001500FFE7FFE79DF8150006B080BD00BFD7
:10FCF00080B586B08DF81700049101208DF80F00B3
:10FD00000020029001903020FFF746FD012828D105
:10FD1000FFE79DF817103020FFF75EFD01281FD187
:10FD2000FFE70499302000F021F8012817D1FFE700
:10FD3000029940F6E060C2F2000050F82100C0696C
:10FD40009DF8171050F8210001900198807803F079
:10FD50003BFA0499087000208DF80F00FFE7FFE7D9
:10FD6000FFE79DF80F0006B080BD00BF80B584B0EE
:10FD70008DF80F00029101208DF80700029860B9FC
:10FD8000FFE79DF80F205C2000210091012311F076
:10FD9000C9FC00988DF80700FFE79DF8070004B044
:10FDA00080BD00BF80B586B08DF81700049101209A
:10FDB0008DF80F000020029001903120FFF7ECFC3D
:10FDC000012828D1FFE79DF817103120FFF704FD27
:10FDD00001281FD1FFE704993120FFF7C7FF012851
:10FDE00017D1FFE7029940F6E060C2F2000050F838
:10FDF0002100C0699DF8171050F82100019001986A
:10FE0000807803F009FA0499087000208DF80F003B
:10FE1000FFE7FFE7FFE79DF80F0006B080BD00BFDA
:10FE200080B584B08DF80F00029101208DF8070095
:10FE30001220FFF7B1FC01281DD1FFE79DF80F103C
:10FE40001220FFF7C9FC012814D1FFE7029800F047
:10FE500017F801280DD1FFE79DF80F1040F6E56077
:10FE6000C2F20000405C0299087000208DF8070083
:10FE7000FFE7FFE7FFE79DF8070004B080BD00BF84
:10FE800080B584B0039001208DF80B00039858B919
:10FE9000FFE75C20002101911222012311F042FCB6
:10FEA00001988DF80B00FFE79DF80B0004B080BDB2
:10FEB00080B588B08DF81F00069101208DF81700DD
:10FEC00000200490039002908DF807000620FFF7B1
:10FED00063FC012855D1FFE79DF81F00069900F04B
:10FEE00055F801284CD1FFE7049940F6E060C2F2D2
:10FEF000000050F8211049699DF81F20895C8DF899
:10FF00000710049950F82100C0699DF8071050F8B7
:10FF100021000290029890B3FFE7049940F6E06058
:10FF2000C2F2000050F8210080699DF81F1001EB1B
:10FF3000810100EB8100039002980399069A00F07A
:10FF400069F801281AD1FFE79DF8071040F6E5602F
:10FF5000C2F20000405C012810D1FFE70299087846
:10FF600089789DF81F20039BDDF818C0EE46CEF877
:10FF700000C000F0B9F88DF81700FFE7FFE7FFE7D2
:10FF8000FFE79DF8170008B080BD00BF80B586B0C0
:10FF90008DF81700049101208DF80F0000200290C9
:10FFA0009DF81700029A40F6E061C2F2000151F894
:10FFB0002210096988420DD2FFE79DF81700029AC6
:10FFC00040F6E061C2F2000151F82210097988423E
:10FFD0000BDAFFE75C20002101910622022311F0D9
:10FFE000A1FB01988DF80F000FE0049858B9FFE7C6
:10FFF0005C20002100910622012311F093FB009860
:020000040001F9
:100000008DF80F0000E0FFE7FFE79DF80F0006B056
:1000100080BD00BF80B584B00390029101920020A2
:100020008DF803008DF80200ADF800000398017808
:1000300040F6F260C2F2000030F81100ADF80000A6
:100040000398C069BDF8001001EB410100EBC1004D
:10005000807A012819D1FFE7019880780299097AFE
:1000600088420DDCFFE70198807809280CD3FFE770
:100070000198406800F08040B0F1804F04D0FFE765
:1000800001208DF80300FFE709E001988078092836
:1000900004D3FFE701208DF80300FFE7FFE79DF899
:1000A0000300012807D1FFE75C200021062203237B
:1000B00011F038FB13E00198806858B9FFE7029807
:1000C000407938B9FFE75C2000210622012311F0B6
:1000D00029FB03E001208DF80200FFE7FFE79DF810
:1000E000020004B080BD00BF80B588B0DDF828C034
:1000F0008DF81F008DF81E108DF81D20069301202D
:100100008DF80F0000208DF80E0006989DF81D2038
:1001100040F67871C2F2000141F822000698007C96
:10012000012853D1FFE70A984068C00F8DF81000EE
:100130000A9880788DF8110000208DF81200FFE7F2
:100140009DF81E000699497C9DF80E201144C9B205
:1001500003F088F88DF80F009DF80F00C8B9FFE78D
:100160009DF81F009DF81E109DF81D20069B5B7CCE
:100170009DF80EC06344DDF828E0EC46CCF804E0BE
:10018000DBB2CCF8003004AB01F094FC8DF80F002A
:10019000FFE79DF80E0001308DF80E00FFE79DF897
:1001A0000E100698C27900209142029008DAFFE70B
:1001B0009DF80F000238B0FA80F040090290FFE786
:1001C0000298C0070028BBD1FFE7FFE79DF80F00AA
:1001D00048B1FFE79DF80F00022804D0FFE7012097
:1001E0008DF80F00FFE79DF80F0008B080BD00BF3D
:1001F00080B586B08DF8170000200490039002901F
:100200008DF807001420FFF7C7FA012837D1FFE760
:100210009DF8170000F036F801282FD1FFE7049968
:1002200040F6E060C2F2000050F8211049699DF8E4
:100230001720895C8DF80710049950F82100C069D7
:100240009DF8071050F8210002900298A8B1FFE72E
:10025000049940F6E060C2F2000050F82100806985
:100260009DF8171001EB810100EB810003900298CB
:100270008078039900F038F8FFE7FFE7FFE706B062
:1002800080BD00BF80B584B08DF80F0001208DF8CF
:100290000E00002002909DF80F00029A40F6E061E7
:1002A000C2F2000151F82210096988420DD2FFE71D
:1002B0009DF80F00029A40F6E061C2F2000151F889
:1002C0002210097988420BDAFFE75C2000210191B6
:1002D0001422022311F026FA01988DF80E00FFE790
:1002E0009DF80E0004B080BD80B584B08DF80F007D
:1002F000029100208DF807008DF80700FFE79DF8B8
:1003000007000299C979884211DAFFE79DF80F00CA
:100310000299497C9DF807201144C9B201F07AFD89
:10032000FFE79DF8070001308DF80700E7E704B00C
:1003300080BD00BF80B584B00020039002908DF88E
:1003400007008DF80600039940F6E060C2F2000055
:1003500050F82100002866D0FFE7039940F6E060DE
:10036000C2F2000050F8210000798DF80600FFE786
:100370009DF80600039A40F6E061C2F2000151F8D0
:100380002210096988424DD2FFE7039940F6E060E8
:10039000C2F2000050F8211049699DF80620895CDE
:1003A0008DF80710039950F82100C0699DF80710D7
:1003B00050F821000290029870B3FFE70298C078CD
:1003C000012828D1FFE7039940F6E060C2F200005F
:1003D00050F8210080699DF8061001EB810100EBC7
:1003E00081000079012816D1FFE79DF807000299E6
:1003F00089789DF80620DDF80CC040F6E063C2F273
:10040000000353F82C309B6902EB820C03EB8C0346
:1004100000F00CF8FFE7FFE79DF8060001308DF8CB
:100420000600A5E7FFE704B080BD00BF80B584B03B
:100430008DF80F008DF80E108DF80D2002930298A4
:100440009DF80D2040F67871C2F2000141F82200BB
:1004500000208DF807008DF80700FFE79DF80700E2
:100460000299C979884247DAFFE79DF80F1045F2F3
:10047000C440C0F2020050F821000299497C9DF866
:100480000720114400EB0110007B02282DD1FFE76B
:100490009DF80E000299497C9DF807201144C9B2CD
:1004A00002F0A2FF9DF80E000299497C9DF80720FA
:1004B0001144C9B202F0D6FE8DF806009DF8060080
:1004C00090B9FFE79DF80F1041F2A430C2F200008E
:1004D00000EB01200299497C9DF80720114430F877
:1004E0001100EFF75DFFFFE7FFE7FFE79DF807006B
:1004F00001308DF80700B1E704B080BD80B584B04D
:100500000020039002908DF807008DF806000399F3
:1005100040F6E060C2F2000050F8210000285CD0F4
:10052000FFE7FFE79DF80600039A40F6E061C2F29C
:10053000000151F82210097988424DDAFFE703994A
:1005400040F6E060C2F2000050F8211049699DF8C1
:100550000620895C8DF80710039950F82100C069C6
:100560009DF8071050F821000290029870B3FFE741
:100570000298C078012828D1FFE7039940F6E0608F
:10058000C2F2000050F8210080699DF8061001EBCE
:10059000810100EB81000079012816D1FFE79DF869
:1005A0000700029989789DF80620DDF80CC040F616
:1005B000E063C2F2000353F82C309B6902EB820C1B
:1005C00003EB8C0300F00CF8FFE7FFE79DF8060053
:1005D00001308DF80600A5E7FFE704B080BD00BF3D
:1005E00080B582B08DF807008DF806108DF80520D3
:1005F000009300989DF8052040F67871C2F2000142
:1006000041F822009DF8060003F0FAFDF0B9FFE77B
:100610000098007C48B9FFE79DF807009DF8061098
:100620009DF8052001F088FA0FE00098007C022870
:1006300009D1FFE79DF807009DF806109DF80520F9
:1006400001F0B0FA00E0FFE7FFE7FFE702B080BD8E
:10065000704700BF80B584B00020039002908DF8F1
:100660000700039940F6E060C2F2000050F8210054
:10067000E0B3FFE700208DF80700FFE79DF80700D3
:10068000039A40F6E061C2F2000151F82210896835
:1006900088422AD2FFE7039940F6E060C2F20000E8
:1006A00050F82100C0699DF8071050F82100029011
:1006B000029898B1FFE70298C07801280DD1FFE7B2
:1006C0000299087889789DF8073040F6E562C2F211
:1006D00000021A4400F00CF8FFE7FFE7FFE79DF87F
:1006E000070001308DF80700C8E7FFE704B080BDC0
:1006F00080B584B08DF80F008DF80E1002929DF831
:100700000F1040F6EC60C2F2000050F8210001909A
:100710000298007801280FD1FFE79DF80E0003F042
:1007200035FD40B9FFE70298022101700198407839
:10073000EFF72EFEFFE716E002980078022810D1AE
:10074000FFE79DF80E0003F021FD012808D1FFE727
:1007500002980121017001984078EFF719FEFFE738
:1007600000E0FFE7FFE704B080BD00BF80B586B0C2
:100770008DF817008DF816108DF8152000200490C4
:1007800003908DF80B00049940F6E060C2F200007F
:1007900050F82100002866D0FFE7049940F6E06099
:1007A000C2F2000050F82110C9689DF81720895C3A
:1007B0008DF80B10049950F82100C0699DF80B10BA
:1007C00050F821000390039800284BD0FFE79DF8D4
:1007D000150001460191B8B1FFE70198012804D046
:1007E000FFE7019802281FD03AE003980078049AA6
:1007F00040F6E061C2F2000151F8221089699DF8CB
:10080000162000F033F82CE0039908788978049BCF
:1008100040F6E062C2F2000252F8232092699DF88D
:10082000163000F067F81CE09DF81600072807D185
:10083000FFE75C2000210822012310F07FFFFFE783
:10084000039908788978049B40F6E062C2F20002BE
:1008500052F8232092699DF8163000F04BF800E022
:10086000FFE7FFE7FFE706B080BD00BF80B584B0BB
:100870008DF80F0002918DF8072000208DF80600FA
:100880009DF80F1040F6F560C2F2000000EBC110B9
:100890009DF80710405C8DF806009DF80600FF28C3
:1008A00025D0FFE702989DF8061001EB810100EBCF
:1008B00081000079D8B9FFE702989DF8061001EB96
:1008C000810100EB8100007C01280FD1FFE79DF83A
:1008D0000F1041F2A430C2F2000000EB01209DF89D
:1008E000071030F81100EFF75BFDFFE7FFE704B0FA
:1008F00080BD00BF80B58EB08DF837008DF8361002
:100900000C928DF82F309DF8371040F6EC60C2F253
:10091000000050F821000A90002009908DF80F0087
:1009200002909DF8371040F6F560C2F2000000EB2F
:10093000C1109DF82F10405C8DF80F009DF80F003E
:10094000FF2800F09080FFE70C989DF80F1001EB56
:10095000810100EB81000079002840F08480FFE7EE
:100960000C989DF80F1001EB810100EB81000290C3
:100970000298007C8DF807009DF8070008BBFFE790
:100980009DF8371045F2C440C0F2020050F8210033
:100990000299497C0901405809909DF83700029955
:1009A000C978099A6B461A6007AA04AB01F0BAF934
:1009B0009DF8360002990B79497C002202F0DCF8A0
:1009C00050E09DF8070002284AD1FFE79DF82F006C
:1009D00007280BD1FFE70A984068806828B1FFE735
:1009E0000A98406880688047FFE738E09DF82F004C
:1009F00006280BD1FFE70A984068C06828B1FFE7D6
:100A00000A984068C0688047FFE727E09DF83710E4
:100A100045F2C440C0F2020050F821000299497C1E
:100A20000901405809909DF837000299C978099A40
:100A30006B461A6007AA04AB01F074F90A98406883
:100A4000006928B1FFE70A98406800698047FFE71E
:100A50009DF83600002102F0FBF8FFE7FFE700E019
:100A6000FFE7FFE7FFE70EB080BD00BF80B584B0B1
:100A70008DF80F008DF80E100020029001908DF877
:100A80000300029940F6E060C2F2000050F8210035
:100A9000B0B3FFE7029940F6E060C2F2000050F800
:100AA0002110C9689DF80F20895C8DF80310029908
:100AB00050F82100C0699DF8031050F82100019002
:100AC0000198E0B1FFE79DF80E00122807D1FFE77B
:100AD0005C2000210822012310F030FEFFE701997D
:100AE00008788978029B40F6E062C2F2000252F870
:100AF000232092699DF80E3000F004F8FFE7FFE72D
:100B000004B080BD80B58CB08DF82F008DF82E100C
:100B10000A928DF827309DF82F1040F6EC60C2F253
:100B2000000050F82100089000208DF80B009DF87F
:100B30002F00C10140F6F560C2F20000405C8DF864
:100B40000B009DF80B00FF2841D0FFE70A989DF8A5
:100B50000B1001EB810100EB81000079B8BBFFE7CE
:100B60000A989DF80B1001EB810100EB81000190C8
:100B70009DF82700112813D1FFE79DF82F00019958
:100B8000C978089A126B6B461A6006AA03AB01F08B
:100B9000C9F89DF82E000899096B02F059F815E084
:100BA0009DF8270012280FD1FFE70898C06A20B1EE
:100BB000FFE70898C06A8047FFE79DF82E00089974
:100BC000096B02F045F800E0FFE7FFE7FFE70CB034
:100BD00080BD00BF80B584B08DF80F00002002906A
:100BE00001908DF80300029940F6E060C2F2000027
:100BF00050F8210078B3FFE7029940F6E060C2F2B6
:100C0000000050F82110C9689DF80F20895C8DF80C
:100C10000310029950F82100C0699DF8031050F8A4
:100C2000210001900198A8B1FFE70199087889781F
:100C300000F014F868B9FFE79DF8032040F6E5617D
:100C4000C2F200010220885401984078EFF79AFB25
:100C5000FFE7FFE7FFE704B080BD00BF80B584B0C9
:100C60008DF80F008DF80E1000208DF80C008DF817
:100C700007009DF80F1040F6EC60C2F2000050F83B
:100C8000210000909DF80F1040F6F460C2F20000C1
:100C9000405C012847D1FFE79DF80E0002F0FCF907
:100CA0000098007B012807D1FFE79DF80E00012185
:100CB000002202F069FEFFE7009890F83600000776
:100CC000002807D5FFE79DF80E000A21002202F058
:100CD0005BFEFFE7009890F836004007002807D534
:100CE000FFE79DF80E000B21002202F04DFEFFE70A
:100CF000009890F83600C00738B1FFE79DF80E0065
:100D00000C21002202F040FEFFE70098007A8007E5
:100D1000002807D4FFE79DF80E000022114602F0DC
:100D200033FEFFE7FFE700208DF80C00FFE79DF89A
:100D30000C00009991F82010884237DAFFE70098FC
:100D4000406A9DF80C1050F8210002900298007C37
:100D500001281DD1FFE700208DF80700FFE79DF86F
:100D600007000299C979884211DAFFE79DF80E0061
:100D70000299497C9DF807201144C9B201F04AF854
:100D8000FFE79DF8070001308DF80700E7E706E070
:100D90009DF80E000299497C01F03CF8FFE7FFE75F
:100DA0009DF80C0001308DF80C00C0E79DF80E0096
:100DB00003F088FA8DF80D009DF80D0004B080BD99
:100DC00080B586B08DF817008DF8161004920020BB
:100DD000039002908DF80700039940F6E060C2F29C
:100DE000000050F82100B8B3FFE7039940F6E06037
:100DF000C2F2000050F82110C9689DF81720895CE4
:100E00008DF80710039950F82100C0699DF807106C
:100E100050F8210002900298E8B1FFE7029840786C
:100E2000049900F01BF89DF81600012809D1FFE78E
:100E30000298406920B1FFE7029840698047FFE7C8
:100E400008E00298006920B1FFE702980069804736
:100E5000FFE7FFE7FFE7FFE706B080BD80B582B0A0
:100E60008DF8070000919DF801004007002806D585
:100E7000FFE79DF807000921EFF71EFEFFE79DF849
:100E800001000007002806D5FFE79DF807000821AC
:100E9000EFF712FEFFE79DF80100C006002806D517
:100EA000FFE79DF807000A21EFF706FEFFE79DF830
:100EB00001008006002806D5FFE79DF80700042101
:100EC000EFF7FAFDFFE79DF801004006002806D580
:100ED000FFE79DF807000221EFF7EEFDFFE79DF821
:100EE00001000006002806D5FFE79DF80700012154
:100EF000EFF7E2FDFFE702B080BD00BF80B586B02E
:100F00008DF81700049103920020029001908DF853
:100F10000300029940F6E060C2F2000050F82100A0
:100F2000002845D0FFE7029940F6E060C2F20000D9
:100F300050F82110C9689DF81720895C8DF80310BE
:100F4000029950F82100C0699DF8031050F8210063
:100F50000190019858B3FFE704980A2809D1FFE7E8
:100F60000198806B20B1FFE70198806B8047FFE715
:100F70001CE004980B2809D1FFE70198C06B20B151
:100F8000FFE70198C06B8047FFE70EE004980C284C
:100F900009D1FFE70198006C20B1FFE70198006CD0
:100FA0008047FFE700E0FFE7FFE7FFE7FFE7FFE736
:100FB00006B080BD80B584B08DF80F0001208DF89B
:100FC0000E009DF80F1040F6EC60C2F2000050F8E1
:100FD000210002901520FEF7DFFB012836D1FFE744
:100FE0009DF80F101520FEF7F7FB01282DD1FFE724
:100FF000029890F84400012826D1FFE702988078F3
:1010000003F062FE8DF80E009DF80E00D8B9FFE7E0
:101010009DF80F2040F6F061C2F20001019101201D
:1010200088540298807803F049FF014601988DF8B2
:101030000E109DF80F10405C20B1FFE701208DF8E5
:101040000E00FFE7FFE7FFE7FFE7FFE79DF80E0071
:1010500004B080BD80B582B08DF8070001208DF806
:1010600006009DF8071040F6EC60C2F2000050F850
:10107000210000901620FEF78FFB01282FD1FFE7FB
:101080009DF807101620FEF7A7FB012826D1FFE7E1
:10109000009890F84400012812D1FFE79DF807104E
:1010A00040F6F060C2F20000405C012807D1FFE783
:1010B0000098807803F07EFF8DF80600FFE7FFE7D9
:1010C0009DF8060048B9FFE79DF8072040F6F0615B
:1010D000C2F2000100208854FFE7FFE7FFE79DF818
:1010E000060002B080BD00BF80B586B08DF8170045
:1010F0008DF81610049201208DF80F0004989DF8C9
:10110000172040F6EC61C2F2000141F822000020F5
:101110008DF80E008DF80D008DF80C0002909DF8F2
:1011200016009DF8172045F2C441C0F2020151F8A3
:101130002210049A926A126801F0C6F98DF80F0025
:101140009DF80F00002840F0BA80FFE79DF81600D8
:1011500001F0ACFC9DF8172040F6F461C2F20001EA
:10116000012088549DF81600049AD169128B02EB75
:10117000420211F8321003F0D5FC00208DF80C006B
:10118000FFE79DF80C007F2813DCFFE79DF81710A0
:1011900040F6F560C2F2000000EBC1119DF80C2092
:1011A000FF208854FFE79DF80C0001308DF80C00FB
:1011B000E7E700208DF80E00FFE79DF80E00049988
:1011C00091F82010884273DAFFE70498406A9DF88E
:1011D0000E1050F8210002900298C27840F6787103
:1011E000C2F2000141F822000298007C8DF807004D
:1011F0009DF807000146009140B1FFE700980128E3
:1012000011D0FFE7009802282FD049E0029A9DF8FC
:10121000171040F6F560C2F2000000EBC111D07863
:10122000527C88543DE000208DF80D00FFE79DF8CA
:101230000D000299C979884216DAFFE7029A9DF8F3
:10124000171040F6F560C2F2000000EBC111D07833
:10125000527C9DF80D301A448854FFE79DF80D002C
:1012600001308DF80D00E2E71BE0029B9DF81700AE
:1012700040F6F561C2F2000101EBC012D8785B7C48
:10128000D0540298C0789DF8172001EBC2129071DB
:101290000298C0789DF8172001EBC211C87100E0D8
:1012A000FFE7FFE79DF80E0001308DF80E0084E7A0
:1012B0009DF817009DF8161000F006F8FFE79DF85E
:1012C0000F0006B080BD00BF80B586B08DF8170056
:1012D0008DF816109DF8171040F6EC60C2F2000071
:1012E00050F821000490002000908DF80F009DF828
:1012F0001600012102F0C0FE00988DF80F00FFE7F4
:101300009DF80F00049991F82010884243DAFFE716
:101310000498406A9DF80F1050F82100029002983E
:10132000007C08BBFFE70298807820B9FFE7002027
:101330008DF8070003E001208DF80700FFE79DF816
:101340001600029B597C9DF80720DB681B6800F0A3
:101350006FFF9DF816009DF80710029B5A7CDB6812
:101360005B6803F069FA0FE00298007C022809D15B
:10137000FFE79DF817009DF816109DF80F2000F06C
:1013800017F800E0FFE7FFE7FFE79DF80F000130E7
:101390008DF80F00B4E79DF8160002F093FF0028C7
:1013A00018BF01208DF815009DF8150006B080BD0E
:1013B00080B5ADF5846D8DF81F048DF81E148DF881
:1013C0001D249DF81F1440F6EC60C2F2000050F896
:1013D0002100CDF8180400208DF817048DF81604AC
:1013E000DDF81814496A9DF81D2451F82210CDF833
:1013F00010148DF80F048DF80E0403A84FF48061CB
:101400000FF0BCFEDDF81004417A062000EB9100DD
:10141000202809D8FFE7DDF81004417A062000EB08
:1014200091008DF80F0403E020208DF80F04FFE7F2
:1014300000208DF81704FFE79DF817149DF80F247E
:101440000020914202900BDAFFE79DF81714DDF8B7
:101450001004427A00209142B8BF01200290FFE7B9
:101460000298C007C0B1FFE79DF81F049DF81E1445
:101470009DF81734DDF81024EC46CCF800200DF26E
:101480000E4200F053F88DF81604FFE79DF817049C
:1014900001308DF81704CFE79DF81E04DDF818140D
:1014A0004968496803F028FA00208DF81704FFE71F
:1014B0009DF817049DF8161488422DDAFFE7DDF831
:1014C0001004C0689DF8172450F8320003A901EBFE
:1014D000C2014860DDF81004807840B1FFE79DF854
:1014E000171403A800EBC1010120487007E09DF824
:1014F000171403A800EBC10100204870FFE79DF816
:10150000172403A9002001F83200FFE79DF8170413
:1015100001308DF81704CBE79DF81E049DF80E14DA
:1015200003AA02F0FBFE0DF5846D80BD80B588B086
:10153000DDF828C08DF81F008DF81E1006928DF87A
:10154000173000208DF8160004909DF81F1040F60B
:10155000EC60C2F2000050F821000390039840684C
:1015600000788DF80B009DF80B000146019140B109
:10157000FFE7019801282BD0FFE70198022869D0E6
:10158000DFE00A98407A8DF816004FF04040049052
:101590000699002008700A98807860B1FFE70A98E1
:1015A000C0689DF8171000EBC1004168049840EA3C
:1015B000410004900BE00A98C0689DF8171000EBFA
:1015C000C1004168049840EAC1400490FFE7BCE0D4
:1015D0000A98407A40008DF816004FF04040049081
:1015E0000699012008700A988078D8B1FFE70A9818
:1015F000C0689DF8171000EB0110406840004FF6DE
:10160000FF7120EA01010498084304900A98C06819
:101610009DF8171000EB0110C168049840EAD13022
:10162000049016E00A98C0689DF8171000EB0110AE
:101630004168049840EAC14004900A98C0689DF847
:10164000171000EB0110C168049840EAC100049033
:10165000FFE77AE00A98407A80008DF81600069934
:10166000022008700A988078A8B3FFE70A98C0683B
:101670009DF8171000EB411041684FF07F4000EAE1
:10168000C10004900A98C0689DF8171000EB411043
:10169000C1680020C0F2FF7000EA511104980843AD
:1016A00004900A98C0689DF8171000EB411041693A
:1016B0006FF0FF0000EA51310498084304900A9843
:1016C000C0689DF8171000EB4110C169049840EA0A
:1016D0005150049034E00A98C0689DF8171000EB50
:1016E000411041684FF07F4000EA415004900A9851
:1016F000C0689DF8171000EB4110C06840034FF61A
:10170000FF7120EA01010498084304900A98C06818
:101710009DF8171000EB411041696FF0E00000EAFE
:1017200041110498084304900A98C0689DF8171066
:1017300000EB4110C169049840EAD1000490FFE732
:1017400003E0069903200870FFE79DF81E009DF84E
:101750001710049A03F050F99DF8160008B080BDE8
:1017600080B586B08DF817008DF816109DF817100B
:1017700040F6EC60C2F2000050F821000490002016
:101780008DF80F00029001218DF807108DF80F00E1
:10179000FFE79DF80F00049991F82010884257DA6E
:1017A000FFE70498406A9DF80F1050F8210002905E
:1017B0000298807820B9FFE700208DF8060003E04A
:1017C00001208DF80600FFE70298007C58B9FFE77A
:1017D0009DF81600029B597C9DF80620DB681B686B
:1017E00000F026FDFFE70298007950BBFFE7029862
:1017F000007C0146009120B1FFE70098022809D043
:101800001DE09DF8160002990B79497C002201F039
:10181000B3F915E00498806A00688079012807D13F
:10182000FFE79DF816000499096B01F011FA05E035
:101830009DF81600002101F00BFAFFE700E0FFE73A
:10184000FFE7FFE79DF80F0001308DF80F00A0E7DC
:101850009DF817009DF8161000F0ACF820B9FFE7CE
:1018600000208DF80700FFE79DF8070006B080BD57
:1018700080B586B08DF817000020049003900121F8
:101880008DF80B100490049940F6E060C2F200005D
:1018900050F82100C0699DF8171050F821000390FE
:1018A0009DF8171040F6E560C2F20000405C01466A
:1018B0000191012805D0FFE701980238022818D3CA
:1018C00027E0039908788978FFF7C8F980B9FFE71E
:1018D0009DF8172040F6E560C2F200000221815415
:1018E00003984078EEF754FD00208DF80B00FFE7D9
:1018F00010E09DF8172040F6E560C2F200000221DA
:10190000815403984078EEF743FD00208DF80B00DA
:1019100000E0FFE79DF80B0006B080BD80B584B005
:101920008DF80F0000200290019001218DF8031026
:101930000290029940F6E060C2F2000050F82100E7
:10194000C0699DF80F1050F8210001909DF80F100C
:1019500040F6E560C2F20000405C022810D1FFE7CB
:101960009DF80F2040F6E560C2F20000032181548B
:1019700001984078EEF70CFD00208DF8030015E08B
:101980009DF80F1040F6E560C2F20000405C0328AD
:1019900004D1FFE700208DF8030006E05C20002161
:1019A000032206230FF0BEFEFFE7FFE79DF80300CA
:1019B00004B080BD80B582B08DF807008DF80610A8
:1019C00001208DF805009DF8071040F6EC60C2F28A
:1019D000000050F8210000909DF8060002F03EFC47
:1019E0008DF805009DF806000621C0F23B0101F0CC
:1019F000A3FA9DF8071040F6F460C2F20000405CC4
:101A0000012847D1FFE70098007B012807D1FFE7B5
:101A10009DF806000122114601F0B6FFFFE700988D
:101A200090F836000007002807D5FFE79DF806006C
:101A30000A21012201F0A8FFFFE7009890F8360084
:101A40004007002807D5FFE79DF806000B2101227B
:101A500001F09AFFFFE7009890F83600C00738B110
:101A6000FFE79DF806000C21012201F08DFFFFE742
:101A70000098007A8007002807D4FFE79DF8060049
:101A80000021012201F080FFFFE79DF8060001F030
:101A900077FAFFE79DF8050038B9FFE79DF80600E3
:101AA00001F034FC8DF80500FFE79DF8050002B059
:101AB00080BD00BF10B586B08446099808988DF89F
:101AC00017C08DF816108DF8152004938DF80F00AF
:101AD00001208DF80E009DF8151040F67870C2F2C6
:101AE000000050F821000290099800889DF8172006
:101AF00041F2A431C2F2000101EB02219DF80F2056
:101B000021F812009DF816009DF80F10049A029B10
:101B10001B79DDF824E0DEF804C0DEF80840EE466C
:101B2000CEF80440CEF800C002F0B8FC8DF80E00EC
:101B30009DF80E0006B010BD80B59CB08DF86F000A
:101B40008DF86E108DF86D209DF86D1040F6787050
:101B5000C2F2000050F8210001909DF86E0001993A
:101B60000B79497C07AA01F007F89DF86E000199EE
:101B7000497C01F0F9FC9DF86E000199497C01F067
:101B800071FB60B9FFE79DF86F009DF86D106B4623
:101B900007AA1A6005AA02AB00F0C4F8FFE71CB060
:101BA00080BD00BF80B5A0B08DF87F008DF87E109D
:101BB0008DF87D209DF87F1040F6EC60C2F20000A9
:101BC00050F821001E909DF87D1040F67870C2F20A
:101BD000000050F821001D90002002908DF80F00A9
:101BE0008DF80E008DF80D009DF87E00052102F0A5
:101BF00089FA014602988DF80E108DF80F00FFE764
:101C00009DF80F101E9890F820200020914201901E
:101C100008DAFFE79DF80E000138B0FA80F04009BD
:101C20000190FFE70198C007002879D0FFE79DF8F1
:101C30007E00062102F066FA8DF80D009DF80D0079
:101C4000012810D1FFE71E984068C06828B1FFE75F
:101C50001E984068C0688047FFE79DF87E00062117
:101C600002F076FAFFE79DF87E00072102F04AFABB
:101C70008DF80D009DF80D00012816D1FFE75C20BE
:101C80000021082201230FF059FD1E98406880684A
:101C900028B1FFE71E98406880688047FFE79DF8FD
:101CA0007E00072102F054FAFFE79DF87E0009A9A3
:101CB00000F0CEFF9DF87E001D99497C01F054FC98
:101CC0009DF87E001D99497C01F0CCFA8DF80C003E
:101CD0009DF80C00B0B9FFE79DF87F009DF87D10DE
:101CE0006B4609AA1A6007AA04AB00F01BF81E98FD
:101CF0004068006928B1FFE71E9840680069804786
:101D0000FFE7FFE79DF87E00052102F0FBF98DF863
:101D10000E00FFE79DF80F0001308DF80F006FE710
:101D200020B080BD80B586B0DDF820C08DF81700EA
:101D30008DF81610049203939DF8171040F6EC608E
:101D4000C2F2000050F8210002909DF8161040F6F3
:101D50007870C2F2000050F82100019008984068A5
:101D600004990860089880788006002806D5FFE767
:101D70000499086840F000400860FFE70198007C83
:101D800080B9FFE70898006800F07060B0F1C06F9C
:101D900007D1FFE75C200021082201230FF0CEFCD1
:101DA000FFE7FFE70198007C02280DD0FFE70898C5
:101DB000C0780006002806D5FFE70499086840F0BF
:101DC00080400860FFE7FFE70198C0780499096840
:101DD000089B93F848200833EEF75AFE012816D1E5
:101DE000FFE70198C0780499087102980078049977
:101DF0004871089890F8480003998860089808305E
:101E00000399086004980399EEF7D6FAFFE706B045
:101E100080BD000080B582B08DF807008DF80610F7
:101E200000208DF80500FFE79DF80700082809D37A
:101E3000FFE746F21E10C0F2020041F2A60100F0D8
:101E40005FF859E09DF8071041F2A440C2F200008B
:101E500050F8210000909DF807009DF8061000F052
:101E600055F820B1FFE701208DF8050043E0009808
:101E70009DF8061000EB0110007B012804D1FFE75C
:101E800003208DF8050035E09DF807009DF8061049
:101E9000009A92F80234002200F064F800989DF84D
:101EA000061000EB0110007B022809D1FFE79DF826
:101EB00007009DF8061000F0B9F88DF8050011E054
:101EC00000989DF8061000EB0110007B032807D155
:101ED000FFE79DF807009DF8061000F02DF900E0DF
:101EE000FFE7FFE700989DF8061000EB01110120C5
